:10000000E010002015040000BD030000E303000021
:10001000EF0300002F040000310400000000000086
:100020000000000000000000000000003304000099
:10003000350400000000000037040000390400000F
:100040003B0400003D0400003F04000041040000A8
:100050004304000045040000470400004904000078
:100060004B0400004D0400004F0400005104000048
:100070005304000055040000570400005904000018
:100080005B0400005D0400005F04000061040000E8
:1000900063040000650400006704000069040000B8
:1000A0006B0400006D0400006F0400007104000088
:1000B0007304000075040000770400007904000058
:1000C0007B0400007D040000DFF800F07D000020CC
:1000D000DFF800F02F000020F8B5040025005FF0E5
:1000E000FF30002604E00100FF2000F0A1F8761C9C
:1000F000802EF8D38034002605E00100207800F03F
:1001000097F8641C761CB6F5F06FF6D3B5F8481076
:100110004F1C09E00100207800F08AF8641C761C6E
:10012000B6F5006FF6D37F1CB5F8481089B2090AFE
:1001300089B2FFB2B94201DB0026F1E7002604E0F4
:100140000100FF2000F074F8761CB6F5205FF7D3AD
:10015000696CC043814201D1012000E00020F2BD62
:10016000F8B504000D00160010E02800FFF7ACFF02
:100170003700B7F5006F01DD4FF40067220039004A
:100180002800FFF7A5FF3D443C44F61B012EECDAA6
:10019000F1BD0000F8B54FF480442148006850F0EC
:1001A00020001F4908604FF4904502E04FF40060C2
:1001B0000544B5F5802F2AD22800018A40F6A722EF
:1001C0009142F3D190F8481001F0FF014FF4006222
:1001D00002FB01F6B0F8480080B2000A80B24FF48A
:1001E000006101FB00F7B6F5804FDFD12800FFF773
:1001F00073FF002808D04FF400603844821B4FF48E
:1002000080412800FFF7ACFF2800FFF75DFF606921
:10021000044908602068854660688047F1BD000099
:10022000B0400E4008ED00E080B5FFF7B3FF01BD20
:100230000A0AC0B2484000F0FF01002001E049086E
:10024000401CC0B2082805DACB07F8D5034B93EA67
:100250005101F5E791EA0200704700002083B8EDF4
:100260002E4A106001202E4A10602E48016008209E
:100270002B4908602C480068C007FBD4704770B554
:1002800004000D0016002948006850F001002749BD
:10029000086006E031682000FFF7E2FF241D361DEC
:1002A0002D1F042DF6D2002D09D031685FF0FF30EC
:1002B000EDB2EA00904001432000FFF7D1FF1B4858
:1002C0000068400840001949086070BD5FF0FF31C8
:1002D000164A126852F00102144B1A60020002E042
:1002E00013681940121D10F500639A42F8D311F1FA
:1002F000010F0BD00949086001200949086002205C
:100300000749086008480068C007FBD40748006830
:1003100040084000054908607047000010000E408A
:100320000C000E4018000E401C000E4008000E404D
:1003300010B450F8041B79B10268436802440830D5
:10034000DC0744BFA9F10104E31852F8044B43F859
:10035000044B091FF9D1ECE710BC704710B50749F1
:1003600079441831064C7C44163404E00A68081DB0
:10037000114488470146A142F8D110BD2C0000006D
:100380003C0000004EF68851CEF20001086840F4AF
:1003900070000860BFF34F8FBFF36F8F4FF0007096
:1003A000E1EE100A7047000089FFFFFFD000000057
:1003B000B0FEFFFF1000002000000000FEE700007C
:1003C00000F00BF8002801D0FFF7C8FF0020AFF3C2
:1003D0000080FFF729FF00F002F80120704700F0CD
:1003E00001B8FEE70746384600F002F8FBE7FEE7F3
:1003F00080B5AFF30080024A11001820ABBEFBE7C6
:10040000260002000248016841F470010160704753
:1004100088ED00E080B5FFF7F5FFBDE8014000F092
:1004200000B8AFF30080FFF7ADFFFFF7C9FFFEE7AD
:10043000FEE7FEE7FEE7FEE7FEE7FEE7FEE7FEE794
:10044000FEE7FEE7FEE7FEE7FEE7FEE7FEE7FEE784
:10045000FEE7FEE7FEE7FEE7FEE7FEE7FEE7FEE774
:10046000FEE7FEE7FEE7FEE7FEE7FEE7FEE7FEE764
:10047000FEE7FEE7FEE7FEE7FEE7FEE7FEE7000039
:10048000000000000000000000000000000000006C
:10049000000000000000000000000000000000005C
:1004A000000000000000000000000000000000004C
:1004B000000000000000000000000000000000003C
:10400000F87B00204B0A020087CE000093F30000EB
:10401000A70A00010041000000000080000000002D
:10402000C335E1AC0000000000000000000000000B
:104030000000000000000000000000000000000080
:1040400000000000206D73B10000000000000000BF
:1040500000000000FFFFFFFF000000000000000064
:104060000000000000000000000000000000000050
:104070000000000000000000000000000000000040
:104080000000000000000000000000000000000030
:104090000000000000000000000000000000000020
:1040A0000000000000000000000000000000000010
:1040B0000000000000000000000000000000000000
:1040C00000000000000000000000000000000000F0
:1040D00000000000000000000000000000000000E0
:1040E00000000000000000000000000000000000D0
:1040F00000000000000000000000000000000000C0
:10410000F87B00204B0A020087CE000093F30000EA
:10411000E70701009F1401003315010000000000B3
:10412000000000000000000000000000FF16010079
:10413000E3220100000000005F4001007741010020
:1041400089950000ED7701003B500100F5770100F3
:1041500021780100FF770100FD7701001978010047
:1041600033530100235F0100B75F01008760010046
:10417000E7610100676E0100CF800100FBAC010028
:10418000CBAE01001FCB01007BCB01000FCC0100A7
:104190002FF10100AF010200E3060200E70902006F
:1041A000070A0200650A0200670A02000978010096
:1041B000117801002B080100690A02006B0A020055
:1041C000AD0902006D0A02000000000000000000BE
:1041D00000000000000000000000000000000000DF
:1041E00000000000000000000000000000000000CF
:1041F00000000000000000000000000000000000BF
:104200000298380002983E000298A002029800032B
:1042100002985C0002986A0002985C000298F20022
:104220000298A0010298C0010298F40102980202CB
:1042300002986E0202988A020698660700F80698AD
:10424000660700C59C0F00210698EC080698F60A40
:104250000698600B00C5A00F002100F806986607BD
:104260000698840B0698AA0A00F80698660710B903
:1042700002BA06982C0600C5A00F002100F8911282
:10428000033288B903DE52727179811002D8FC7250
:10429000A11020D812710698EC080698F60A069824
:1042A000600B00B95E7000C3000F0021341380DB87
:1042B0001C7100C3A8100840A1141034024C48130C
:1042C00000BC481391140764FF3448138CBB627B15
:1042D00040D80E71517900BA7079811001D8FC7202
:1042E000076A00C0A00008400698480E0420029803
:1042F000480E0698660700BD0698F20710B903DC61
:10430000047100B902BA06982C0604D9067101D8C6
:10431000207106988001FFD8087288B847783670F7
:10432000911008D8067100B8617820B802A800F88A
:1043300000C0000F0021041320DB1A71911008D86F
:1043400008718CB84378BC7008DBB872A11308DB25
:10435000B27203BD069874010698840B00C5A40FC1
:1043600000210698F20703DC0472042506987609FA
:104370000298CE0C9110015503355150011900A03F
:1043800001B8811180D9187100C10C500840141077
:1043900004300C7200C1A45008401410013000A079
:1043A000069866070698840B00BD0698740188B8C5
:1043B000477800C5AC0F0021069876090298CE0C0C
:1043C0000698660706988001FFD8067208B86078DC
:1043D00000C20000020206982A0600F80698540E51
:1043E00088B850785178911104D9047248788CB803
:1043F000427800A0069866070698DC010698AA0A8B
:1044000000F8069866070698F20707DC0A7200C5EE
:10441000A00F002100F80698AA0A03B9911004D849
:10442000047100B900C20000020006982C0601D8F1
:10443000207200C0000F0021041120D914710761FF
:1044400001D9E0728110076001D8D8728CB8637806
:104450000698DC0100C5B00F00210698EC0806980C
:10446000F60A0698600B00C5B40F002100F8069804
:1044700066070698DC0100BD0698740188B8477885
:1044800000C5B80F00210298CE0C06986607069862
:10449000F60D0698840B0698AA0A0698DC0100F827
:1044A000B110076001D80A7108B87F78020C7E78D5
:1044B0000698660701F8911008D8347100C0080FFB
:1044C00000210410015800C2905008402414415C9F
:1044D000A0222413E8222411412931390129F87539
:1044E00018B874788CB8437801B802A800F802981C
:1044F000AA0B0698B20800C024000840207800F8F3
:104500000698660700B8011A91100F30011900C211
:104510000202000006982A0604D9067101B802A812
:1045200000C0000F0021041380DB06720298B20461
:104530000763076301DB0A7190B963790298A405E8
:10454000076300B902EC00CD114502EC00CC41112B
:1045500003B804D91E720731911208DA087102DD1E
:104560001272147002B807600698660E303808722E
:1045700008B80298F20202EC00CA05B801DB127119
:1045800020DA0E7110DAEC7201DA0A71ADB80A7035
:1045900023DAE07202EC00C8076891110F31114074
:1045A0002111C0311140011990B820DA04716178ED
:1045B000411108D90471627820D9047263782731D7
:1045C00023DD0872C0DA0471607803B84111073145
:1045D0000872A11508359C7102DD2872A11108D955
:1045E000927102D91E72CCDA8A7206B802DB0C71A3
:1045F000026D5111FFD952720765054D4C72029838
:10460000A40521114049C0D93E71A0314115403562
:1046100001655141036108DA207204DA2A721049F7
:10462000A1150235067108DB107201340C71076B9D
:1046300080DB147190B8677800C00D0F0C0D0698E0
:10464000680E01D8087207B80298F202CC32204AEC
:1046500000C0051708500698680E113001422088E6
:104660000DDA06720298760500C1C618000020BB5C
:1046700004DA0E7208DA087242B90369F823E823F3
:104680003114056B01DA06710649024B076B076BA3
:1046900000C0540F00213810BC2002DA107100B99C
:1046A000FF21A11380DB06717CB9076918100298FD
:1046B000F20401DB34710698E20502DB1871FC227A
:1046C0002410112811280698A00E00C218000840D6
:1046D000FF20081200C05A0F002104100760076075
:1046E0000698760E01D8087120BC10DB067202987D
:1046F000A40500BB00C1540F00211415511207621C
:104700000762C021112CFF320E71408851140698A7
:10471000AE054143009441115112076AFF320E71F8
:10472000511407640698AE05076C414300C1580F49
:1047300000211410013BB82114113110FF300C710D
:1047400004610112006001DAF87131100760FF3076
:104750000C7100610112006001DAF87101D90C726C
:1047600088B8787804B80298F20200C0000F0021DF
:10477000041380DB307100920362DDDA0671029867
:104780005E04A11101D91E7100C238100840241224
:104790000420281002EC00C804D90A7204DC067256
:1047A00018B873780698B00C00B8477800F83088CD
:1047B0005088FF34087102ECFF24F87002EC00CD41
:1047C000141001BB5150FFD8047131440760006BD5
:1047D00010DBF2710421FF22E4720F4C009500936C
:1047E00000A000C25C0F002124111114FF3402EC60
:1047F00000C8FF24FA760761113807610698760E23
:10480000011108222410112806988A0E00DC087273
:1048100003B80298F20200A088BA727A811204DA10
:10482000FC7200A088BA527A00A0187006988A0814
:1048300010D906710CDB087200B8103C067201B882
:10484000076A00BB00C10C0F002100C4B45008402F
:10485000141120391272417B007CB82400C2000080
:104860000101281400A00698180600C2000F0021BC
:10487000241240DA0672617B007C02982406B11093
:1048800001D8047200A000C02870084004111088EC
:1048900000C1001800401810442004111088A820FE
:1048A000041110884CBA757A18103DB11088F4B80C
:1048B000427844207278D8207378E82073784FB219
:1048C00000C4FFFF8080413A4FAA01BC016441133C
:1048D000076300C06C70084003B918100110011084
:1048E00001B91810011001100110011098200411D5
:1048F000076101B80160003A0471044904D90472E7
:1049000041520760003A0471084908D904723152D3
:104910000460003B0E7200630064314241424FAAC2
:10492000B2704FAA44B801685378F8B85378402061
:10493000527800913DA9009100C0147008401810F1
:104940000091582018100091BC20181000A000C041
:10495000FFFF0000013C1DB00220015840280675F1
:104960001EAC01EC00A0009000C6C00F0021008822
:1049700001B0076800C3680F00213414036C415074
:104980000F30415008130F3003640F340111C04839
:10499000069800080698240603DD1C7204BA00C0BD
:1049A0006C000840041110D9047106BA10232813B2
:1049B000047802989E0801DD0C7200C04400084093
:1049C0002578267809DD067202989E08411303DFD8
:1049D00006720298160C00DD06720698960C53B00B
:1049E00080BB006B30380A7109DD06710298BE0C7D
:1049F00000A000C0680F0021041003600F3000A069
:104A00001088B111076980D90A7100C1800008407F
:104A10000811009100A0B111076940D906720298EF
:104A2000860800C1700F0021141200BC01DC207147
:104A300006988A084034087101B80698BA08F0DA76
:104A40000C720CDB087102B80698BA0848BC00C3A7
:104A500080000840FFB80120042114155145087159
:104A600001455813082400C138300840141100C50E
:104A70000060084054153035016D51410141181353
:104A800001422813481300B82A7000C4600008408F
:104A900000C06C0F002144140410014400A000C0A9
:104AA0006C0F002100B90698180618100698240605
:104AB00000A000C1700F0021141203682150F030D3
:104AC0000152281100A000C020300E400411041033
:104AD0001050F47200A000C028400E400412215172
:104AE00007610C3107691152281000A00698BE0A10
:104AF00000C0F80F002104112EA900C004300840A6
:104B00002178227800C0980F00211DB11810069856
:104B1000A6090111FF300769FF3151B300C4F3FF4B
:104B2000FFFF413B115900290675084B027051AB3C
:104B3000A4BB00C07C300E40041100C20080010004
:104B400020391E71B11204DA18716E7B6F7BE4207C
:104B500004114CBA7C7A181014200411607A1810D1
:104B6000B11002D81071707B30B8627860780DB0E7
:104B700001D8FC7100A00698BE0A00C0FC0F0021FD
:104B800004112EA9F82004110698D60800C004309C
:104B90000840217823780698A60900C0880F0021D4
:104BA0001DB1181000A0541400C0BC0F0021041047
:104BB000012C0A7500B826A806984E0700C0840F7D
:104BC00000211DB1181028B000C1F0FFFFFF1138FF
:104BD0000EB9114028A880B800C14430084008111F
:104BE00000C0006F000026A800C0043008402178F3
:104BF000050C2020267800C063EF000026A8050CD5
:104C000020EC00C004300840247820EC217800C05B
:104C10007BEF000026A828B000C1F0FFFFFF11388D
:104C200000C10A000000114028A8050C00C0043093
:104C30000840207820EC0F0C00C0984008404678CF
:104C40004178B11020D84A7100C04C30084000C1F2
:104C50007D00000018100D0E0D0E00C070300840D1
:104C6000041130311A7100C078300840257824785A
:104C7000960C00C07030084004113031EA7200C058
:104C80004C30084000C106000000181000B9181090
:104C90000698C60800C27C0F0021241000C300FF44
:104CA000FFFF31381140081200A00698BE0A00B874
:104CB00026A800C08C0F00211DB1181000A030B82C
:104CC00040780DB101D9FC72427800C074300E40BA
:104CD000041100C2FEFFFFFF21391810EC2004115F
:104CE00000C2FFFFFFEF213918101C78A4BB707BB6
:104CF0004E7B4F7B00A008B86E784EB010D818726B
:104D000000C00E0000003EA8140C00C00F00000000
:104D10003EA802982E0B00C00E00000044A8140C00
:104D200000C00100000000C1B0300E40081100C0FA
:104D300077801F003DB201423DAA00C1EC0F002167
:104D4000141054A8140C00C077E01F0001423DAAC3
:104D500051B801687D7800C00000004002A800A0A2
:104D60000698180606987E06069824065414069897
:104D70004E07F4B84578090C00C0940F00211DB10E
:104D8000181000A051B801685D7800B844A83EA88A
:104D900000C1B0300E40081100C0001000003DB14D
:104DA00001393DA908B86F7800A001F8541000DC63
:104DB0001271011406984E0718B8707800B841783F
:104DC00000F80298C60B00C57C0F00215415511441
:104DD000FF3507644113FF3407633112FF33076265
:104DE000FF323110212B0158012A0698C6080158BC
:104DF0005128047501584128187551B00CD8067116
:104E0000215806703110115901290675FF0FB8702D
:104E100018B8727800F800C3780F0021341300C46A
:104E2000E0100840441200C000010400013A26715D
:104E300008242814084B00C458100840237C00C4E0
:104E4000700F00214414F034447200C46400084020
:104E5000257C3A7004DBE0720DDDDA7100C1401090
:104E600008401410F821141101581128207100C1B4
:104E7000781008400811076008119110081100C04F
:104E8000006008400410076007600811308800B80F
:104E900006981608009300C0780F0021041102D96B
:104EA0000A7100C16C000840247900B9181000A0F4
:104EB00000C0780F002104110449181000A00698C2
:104EC000F60D11510698D60801B802981608541428
:104ED00041150764076406984E07508806987E00BF
:104EE0000095B110076820D80C7108B8657818B81B
:104EF000717800F808B86C7820B85A7859785B78DF
:104F000000C1F00F0021141054A84EB010D8067143
:104F10000298660D4DB100C09FFFFFFF113840B1F0
:104F200002D91472604800C1040000401112104AF6
:104F300004BB41540C70204802B903BA02BB02BC46
:104F40004DA840A9F8B87078190C3EB141413EA96E
:104F5000F4B973797378717800C1E80F002100C447
:104F600000410840287000C20000010044AA230C40
:104F700000C200000B0044AA00C1E80F002100C2DB
:104F80002000004000C41841084004BB00C0C83FD6
:104F900000001411113821400814050C11400814A8
:104FA00004240F0C2FAB050CB11008D814711CB8D9
:104FB00079787B787A7820B879787B787A78607C91
:104FC000F4244113511406984E07727B53B80168BC
:104FD000050C687840EC00C0900F00211DB118103E
:104FE00000F800C06860084004110761076180D9BB
:104FF000047240EC00A0015053A80698E20D4EB098
:1050000010D80A7200C4F8400840087000C410416B
:10501000084041130C23527C407B01502FA8050C03
:10502000FC23341200C1FF3FC0E0113A28130A0CE0
:1050300000C000000100081406322813050C0150BE
:10504000081408B86D7800A0087809780411214187
:10505000181000A000B900C09C10084018101C20B7
:105060000AB9181000A0115910D90671076007601D
:1050700008D90471076004D90471036002D904716E
:10508000016001D90471006000A010880411033090
:1050900008710761FF20FC721110FF30009100A021
:1050A000108804110230067107610761111000C1F8
:1050B000FFFF00001138009100A00000AF030000C6
:1050C0000028012803280118052A0018002A012AAF
:1050D0000A18292A02290000F01921B4478FA4BF19
:1050E000A14F63FDEED6141D636032E0375EA488E5
:1050F000534E6DFB6435BFF753A1811F582CD0A5CB
:105100004540FC34F32742980C027B0074050020D4
:10511000130C110053A1811F582CD0A54540FC341D
:10512000F3274298080100000000000013080F0058
:10513000636032E0375EA488534E6DFB6435BFF781
:1051400010F01921B4478FA4BFA14F63FDEED61410
:105150001D0000000C53696C69636F6E204C616226
:105160007300000005020C00292A0000020A180042
:105170000240030005020900012A000000000000AF
:1051800005020700002A00000200180020000400A9
:10519000F005002005200300052A00000201180088
:1051A00000000108000000009C51000002000108FE
:1051B00000000000945100000400000800010000FD
:1051C0008C5100000A0007080003000002000000E4
:1051D00000000108000000008851000002000108E2
:1051E00000000000805100000600010800000000DF
:1051F0007C51000002000108000000007451000012
:1052000007000108000000007051000000000108C4
:10521000000000006C5100000200010800000000C6
:105220006451000009000108000000005451000012
:1052300000000108000000004051000002000108C9
:10524000000000002C51000001800208000700004F
:10525000245100000200010800000000105100006D
:1052600002800608000100000851000003000F0042
:1052700011000000A0510000110000000B00000010
:10528000C050000003000000D850000003000000E0
:105290006C520000080B020000000000090B020025
:1052A0000000000000000000A00042010A600706A4
:1052B000020A060700000000636032E0375EA4883F
:1052C000534E6DFB6435BFF753A1811F582CD0A5F9
:1052D0004540FC34F3274298200100009902020067
:1052E00020040001D302020020010002E5020200B6
:1052F000200000030D03020020000100A5060200AB
:1053000020010101DD06020020000103E505020085
:105310002002010A770602002001010B1906020093
:105320002001010C5F06020020070300D9040200DF
:105330002002030185040200200103023D05020052
:105340002000030351050200200503046305020049
:1053500020080305950502002005030677050200D5
:10536000200203079B04020020010308C504020079
:10537000200908004304010020010801770401000E
:10538000200208029D04010020020803E504010038
:105390002002090007660100200109011F660100C3
:1053A00020020902536601002005090395660100E9
:1053B00020060904B166010020040905D567010033
:1053C00020030906ED67010020030907E1660100DB
:1053D0002006090815670100200409096D6701000E
:1053E0002004090A836701002006090B9967010060
:1053F0002002090CBF6701002001090D6969010045
:105400002003090E036801002004090F1968010038
:105410002005091077660100200209114567010087
:1054200020070912FB66010020040A003968010008
:1054300020020A017168010020050A02F7680100D4
:1054400020050A031169010020040A043B690100D8
:1054500020040A055369010020030A06C7680100F9
:1054600020040A077D69010020020B0007050100E6
:1054700020020B019705010020010B02EB05010042
:1054800020050B034306010020050B04450601001F
:1054900020010B054706010020060C008770010063
:1054A00020000C0BE3700100200A0C0CAB70010013
:1054B00020010C0D0F71010020000D0035030200CA
:1054C00020000D01B903020020030D02DD030200DC
:1054D00020020D03F703020020020D043104020034
:1054E00020030E00E506020020010E01FD06020069
:1054F00020000E022307020020040E0C35070200D4
:1055000020010F005D72010020020F01BD72010039
:1055100020020F029573010020010F044572010063
:1055200020010F067572010020000F07A57201000F
:1055300020050F08E772010020020F09197301000E
:1055400020010F0A2F73010020000F0B27720100AA
:1055500020020F0EB573010020000F0FE173010050
:1055600020040F100573010020010F115B7301006F
:1055700020010F124573010020011100B507020040
:105580002004110131080200200200014104010041
:105590002002000241040100200200034104010036
:1055A0002002010041040100200601034104010022
:1055B0002002010A410401002003010B4104010003
:1055C0002002010C410401002003030041040100FA
:1055D00020020301410401002002030241040100F2
:1055E00020020303410401002002030441040100DE
:1055F00020020305410401002002030641040100CA
:1056000020020307410401002002030841040100B5
:1056100020020800410401002002080141040100A9
:105620002002080241040100200208034104010095
:105630002002090041040100200209014104010087
:105640002002090241040100200209034104010073
:10565000200209044104010020020905410401005F
:10566000200209064104010020020907410401004B
:105670002002090841040100200209094104010037
:105680002002090A410401002002090B4104010023
:105690002002090C410401002002090D410401000F
:1056A0002002090E410401002002090F41040100FB
:1056B00020020910410401002002091141040100E7
:1056C000200209124104010020030A0041040100E4
:1056D00020030A014104010020020A0241040100E2
:1056E00020020A034104010020020A0441040100CF
:1056F00020020A054104010020040A0641040100B9
:1057000020020A074104010020030B0041040100AC
:1057100020030B014104010020030B02410401009E
:1057200020030B034104010020030B04410401008A
:10573000200B0B054104010020020C004104010074
:1057400020060C0B4104010020020C0C4104010056
:1057500020020C0D4104010020020D004104010053
:1057600020020D014104010020020D02410401004C
:1057700020030D034104010020020D044104010037
:1057800020020E004104010020020E01410401002C
:1057900020020E024104010020060E0C410401000B
:1057A00020020F004104010020020F01410401000A
:1057B00020020F024104010020020F0441040100F5
:1057C00020020F064104010020020F0741040100DE
:1057D00020020F084104010020020F0941040100CA
:1057E00020020F0A4104010020020F0B41040100B6
:1057F00020020F0E4104010020020F0F410401009E
:1058000020020F104104010020030F114104010088
:1058100020020F1241040100200411004104010084
:105820002001110141040100A00400004104010015
:10583000A002000141040100A00C0100410401008C
:10584000A004010341040100A0000104410401007F
:10585000A002010541040100A00B03004104010066
:10586000A000030141040100A00A08004104010056
:10587000A003080141040100A0080802410401003E
:10588000A003080341040100A00208044104010030
:10589000A003090041040100A00609014104010020
:1058A000A005090241040100A0040903410401000C
:1058B000A007090441040100A006090541040100F4
:1058C000A003090641040100A0070A0041040100E9
:1058D000A0060A0141040100A0070A0241040100D8
:1058E000A0060A0341040100A0030A0441040100C8
:1058F000A0030B0041040100A0020B0141040100C0
:10590000A0070B0241040100A0010C0041040100AA
:10591000A0080C0141040100A0030D004104010096
:10592000A0040E0041040100A0080E024104010081
:10593000A0050F0041040100A0010F014104010076
:10594000A0050F0241040100A0020F034104010061
:10595000A0030F0441040100A0080F054104010049
:10596000A0000F0641040100A0020F09410401003C
:105970000000000000000000000000000100020024
:1059800015005400A9005301A7024F059F0A00000B
:10599000020000000100000008070F000A00C80014
:1059A00020000000A0000000000000000000000037
:1059B000A00042010A200706020A040700000000B6
:1059C000000207000000000000000000A0004201EB
:1059D0000A200706020A0407000000000002070070
:1059E00000000000000000000100000009000000AD
:1059F0000000000001000000100000000100000095
:105A00000000000004000000010000000800000089
:105A10000100000010000000010000000001000073
:105A200001000000000800001D000000000200004E
:105A30001D000000000400001D0000000000010027
:105A40001D00000001000000000000000000000038
:105A50000000000000000000000000000200000044
:105A60000000000000000000030000000000000033
:105A70000000000000000000030000000100000022
:105A80000000000002000000010000000200000011
:105A9000030000000C0804010800000000010602D9
:105AA00001000000000103FF04FF02003B000000B2
:105AB00000F04902000000003C008A003C008C001D
:105AC000F4010000FA0000009600000064000000ED
:105AD0004B000000320000001E0000001400000017
:105AE00000000000070000000200000004000000A9
:105AF000000000000400000000000000050000009D
:105B000000000000611C0100BF1C0100CB1C010053
:105B10006C888391AAF5A53860370BDB5A6083BE89
:105B20003F49F6D4A3C55F3874C9B3E3D2103F50E0
:105B30004AFF607BEB40B7995899B8A6CD3C1ABD97
:105B4000E69D350E480103CCDBFDF4AC1191F4EF7A
:105B5000B9A5F9E9A7832C5E2CBE97F2D203B02039
:105B60008BD28915D08E1C742430ED8FC24563769C
:105B70005C15525ABF9A32636DEB2A65499C80DCF2
:105B80000000000000000000010000000000000014
:105B90000100000000000000000000000100000003
:105BA00000000000010000000200000002000000F0
:105BB00003000000000000000200000000000000E0
:105BC00000000000000000000000000000000000D5
:105BD00002000000020000000100000000000000C0
:105BE00002000000000000000000000001000000B2
:105BF000000000000100000000000000050000009F
:105C0000010000000000000005000000020000008C
:105C1000020000000300000000000000020000007D
:105C20000000000000000000000000000000000074
:105C3000000000000200000005000000010000005C
:105C40000000000005000000FFC1FBE84C90728BD3
:105C5000E7B3518963AB232302841872AA612F3BF7
:105C600051A8E53749FBC9CA0C18532CFD45E39AE6
:105C7000E6F15DB0B61BB4BE2A50EAE90E9C4B5E5D
:105C80005724CCA1B759B8874648050359450000A9
:105C900078464805035964000545000000000000EF
:105CA00078056400000000000645000000000000C8
:105CB0007806640000000000000200000000000000
:105CC00000010000000000000002000000000000D1
:105CD00000010000000000000002000000000000C1
:105CE00000010000000000000002000000000000B1
:105CF000000100000000000000000F40190000003B
:105D000002000000081400200C140020F851054582
:105D1000F946510545034805590000000000000000
:105D20007846510545F90348055964FB0448055177
:105D300000000000F8510545F9984603480545580C
:105D40005283465105455800F903480546785A6480
:105D5000F878FE510545FB0448055100F946034813
:105D600005590000000000000000000000000000D5
:105D700078F946034805596400000000000000005F
:105D80000000000000000000000000000000000013
:105D9000000000E10000270080841E00809C2B8F03
:105DA000FFFFFFFFFFFFFFFFFFFFFFFF00000000FF
:105DB000000000000000000001000000FFFFFFFFE6
:105DC0004B60D2273E3CCE3BF6B053CCB0061D65AF
:105DD000BC86987655BDEBB3E7933AAAD835C65A38
:105DE00096C298D84539A1F4A033EB2D817D037775
:105DF000F240A463E5E6BCF847422CE1F2D1176B10
:105E0000F551BF376840B6CBCE5E316B5733CE2BE2
:105E1000169E0F7C4AEBE78E9B7F1AFEE242E34F11
:105E2000512563FCC2CAB9F3849E17A7ADFAE6BC3C
:105E3000FFFFFFFFFFFFFFFF00000000FFFFFFFF6E
:105E4000F40F010100000000F80F010100C0030081
:105E5000FC0F01010BC003000400010001610100FF
:105E600008000100300000001800010000000000E0
:105E70001C000100010000002800010000000000DB
:105E80002C000100000000003000010000000000B4
:105E900034000100000000003C0001000000000090
:105EA00040000100A00700004800010000000000C1
:105EB0005400010000000000580001000000000034
:105EC000A000010001480000A4000100FF4C0000F8
:105ED000A800010001490000AC000100FF4D0000D6
:105EE000002001000807000010200100FFFFFF0054
:105EF000182001000060DA00083001003FAC00000B
:105F000030300100AA2A10003430010001000000E6
:105F10004030010000000000A04001007A27000F7F
:105F2000F44001002010000034410100800800000E
:105F300038410100E6870000404101004800880028
:105F400044410100C0E6531114600100100000003C
:105F500018600100000000841C6001001FC00100E7
:105F600020600100C8200000246001000000000043
:105F700028600100000000032C6001000000000008
:105F800030600100C804FF0034600100A208000076
:105F9000386001000A0000013C600100920004002A
:105FA00040600100D6BE898E446001000000000000
:105FB000486001008C00D40A4C6001000000000021
:105FC00050600100D1032A0054600100000000006D
:105FD00058600100000000005C600100040A132208
:105FE0006060010032414A4F64600100000000001F
:105FF00014700100F8700200187001000003000026
:106000001C7001006000D081287001000000800138
:10601000487001003C3D00004C700100BC190000BC
:106020007070010005810000747001001301000010
:106030007870010000235500FFFFFFFFF40F0101FE
:1060400000000000FC0F01010BC00300083001003C
:106050003FAC0000F440010020100000FFFFFFFFF4
:10606000F40F010100080000FC0F010108C003004B
:106070000830010037AC0000FFFFFFFFFC0F0101FB
:1060800009C003000830010037AC0000F4400100F3
:1060900020000000FFFFFFFFF4400100200000008F
:1060A000FFFFFFFFFC0F010109C0030008300100E2
:1060B00037AC0000FFFFFFFF80B5C0490A685060A1
:1060C0000868BF4A02602AE038B5BC4D044628681B
:1060D000047122462868401D00F0B0F92868B949CB
:1060E0000DE038B50C46B54D11462A689080947184
:1060F00022462868C01D00F0A1F92868B24901EBCA
:1061000004210160296800F013F8B0480068001D00
:1061100032BD80B5A9490A689080AD481060096811
:1061200000F006F8A9480068001D02BD0160316852
:1061300051F8040B00F00EBAA6488008800000F267
:10614000FF70C00AC00200F1100140F6A7230A88C0
:106150009A4209D1098F0A0008D0C9029E4A01F467
:10616000FF218142116001D000207047012070475B
:106170002DE9F04FADF5606DA9B082A8E42100F0E3
:1061800049FAC4208290ACAC00208DF8A90201210C
:1061900001208DF8AC024FF0010B40F6B830A08022
:1061A0004FF00057BBA8AC908C48A061894880088C
:1061B000800000F2FF70C60A894800F08DFB894814
:1061C0000168F602490505D53968012904BF4FF079
:1061D000000B4160FFF7B0FF834D10B9012038601C
:1061E0000AE0BBF1000F07D000203860706928601A
:1061F0003068854670688047022038604FF48271AD
:106200007A486E4E7A4FDFF8EC81DFF8EC91286027
:1062100040F2811B02A800F0FDF93022774976A8F0
:1062200000F01CF9CC22764943A800F017F943A8E6
:1062300076900DF5867A02A8579000208DF8080018
:1062400076A8206182A801F093F80DF5DB7001902B
:106250006C4C09E0002008716B49306801603168BE
:1062600051F8040B00F0ABF901F0B8F9674B026884
:1062700031681A40A02A09D0654B9A4252D0654B2A
:106280009A42E7D0644B9A4254D0EDE73620FFF7AC
:1062900040FF018841B981788DF80810C11C8278CF
:1062A0000DF1090000F0CAF83520FFF732FF018830
:1062B00081B9C11C0422684600F0C0F8BAF8AA00EF
:1062C00000990843AAF8AA0001980099008B084396
:1062D000019908837E21306881805049FFF726FFAD
:1062E0004F4A10210020FFF7FCFE018809B94088C1
:1062F000386010214B4A0020FFF7F3FE018809B9EE
:1063000040882060386800281CBF20680028ABD077
:106310003168022008713168487130684249FFF7DE
:1063200005FFA1E7B0F80510226891429CD100F06A
:1063300081F899E70279C9F800200025B0F8052016
:10634000C8F800203B689A421DD1C07A20B10228CB
:1063500003D0032808D024E000E00020FFF7ACFEC3
:10636000008858451DD11BE030480860FFF7DFFE6C
:10637000164800688088584512D040F6033188429C
:106380000FD180250DE021688A420AD100F052F831
:106390000088B0EB0B0003D00D3808BF822500E069
:1063A00081253268D8F80000D9F8001011713168E1
:1063B000A1F80500CD7130681D49B0E72400002028
:1063C000200400012001000220030A06280000200A
:1063D00020020D03020D0200D8040020A452000088
:1063E0000055080004500E4008ED00E00041000098
:1063F000D0040020CC040020C80400207452000007
:10640000A0510000D404002020010101F800FFFF8A
:10641000A0000A00A0000801A0000A022002090052
:10642000B8520000C85200002002030120000003FF
:1064300020040A0400F10B01807A45E662B38B0761
:1064400008D0521E11F8013B00F8013B00F02480F7
:106450008B07F6D1830740F0208000BF103A07D3A6
:1064600030B4B1E83810103AA0E83810F9D230BC96
:10647000530724BFB1E80810A0E8081044BF51F842
:10648000043B40F8043BD20724BF31F8022B20F82C
:10649000022B44BF0B7803707047083A07D3B1E86A
:1064A0000810083A40F8043B40F804CBF7D25307F1
:1064B000E4E7002A4B490860704700F11C0251696B
:1064C000802900D1704710B582B011684FF0FF33BA
:1064D00009B191F93E303C30434984780C715269DE
:1064E000C1F805204B72002300783E4C88720022D0
:1064F0003E480860012000900B2087E010B53A4C20
:1065000082B0A180214690F83E00A0710023384857
:1065100020600120334C2468009000220720A0470F
:1065200013BD10B5034682B008462F4993F83E309C
:106530002C4C48710B71801C030243EA10202D4B38
:10654000184308601346012000904A792468062009
:10655000A04713BD31B584B00C46012001F0B3F85B
:10656000052817DA9DF813109DF812001D4C2468B9
:10657000090641EA004040F40870019000234FF4FE
:10658000C170ADF8080000220120009001A906208A
:10659000A04712E0049801F0B7F8010003D0496861
:1065A0002046884709E01448056804E004982A68F2
:1065B000214690476D68002DF8D105B030BDC9E780
:1065C00010B50446082001F0CFF810B94FF4C1709F
:1065D00010BD094904600A6842600860002010BDCF
:1065E0000000000050050020FC070020A0070B025F
:1065F000A0030B00A0000B014805002010B582B0DD
:10660000049C0094004C01E0500500202468A04741
:1066100013BD0028002201F0BBB80028890001EB5F
:10662000401000F1844002607047890001EB401087
:1066300000F184400068704700F1806300F1C060A1
:10664000196002607047401CB0FA80F0C0F11F0072
:10665000704710B58142A441E20F1021DFF8400AD3
:10666000FFF7DCFFE20FBDE810401821DFF8640BF4
:10667000D4E7DFF8301ACA6B02B1012241F6713358
:10668000CB63D2B20B68DFF8203A1818DFF8483B2A
:1066900098420B6834BF4FF08070002023F04073A5
:1066A000184308600AB10020C8637047C01C0F2857
:1066B00001D2000770474FF07040704738B504466C
:1066C000002500F073FADFF8F02ADFF8741A94421C
:1066D00008D0DFF8E82A944206D0DFF8E42A944292
:1066E00004D006E0086802E0486800E0886800F02E
:1066F0000700401E032819D8DFE800F002050C0847
:1067000001F09EF804E001F0A1F801E001F09BF82F
:1067100005460BE0DFF8BC0A0068C00103D501F0B4
:1067200051F8850802E001F04DF84508284632BDD1
:10673000DFF8A81A4A68D20702D40A680242FCD1DC
:106740007047DFF89C0A0068704738B5DFF8942A74
:10675000044694421FBFDFF8902A9442DFF88C2A47
:106760009442DFF88C0A2AD0DFF8882A944224D099
:10677000DFF8842A94421ED0DFF8802A944218D091
:10678000DFF87C2A944212D0DFF8782A94420CD0A9
:10679000DFF8742A944206D0DFF8702A94420CBFC6
:1067A000056B00250CE0C56A0AE0856A08E0056A09
:1067B00006E0C56904E0856902E0C56800E0056897
:1067C000DFF81C0A04601921DFF8100AFFF72DFF1B
:1067D0000028F8D1DFF80C0A84420AD0DFF8080A52
:1067E000844208D0DFF8040A844208BF25F0C0655F
:1067F00004E0022000E0012060F35A65DFF8100A8F
:10680000056031BD10B50429DFF8084A17D8DFE864
:1068100001F0030E101214000121216060600120BC
:10682000606100F04DF80028FBD0606810BD0321C6
:10683000F3E70021F1E70221EFE70421EDE7002073
:1068400010BD000010B5DFF8CC391C68042924F015
:10685000770412D8DFE801F00306090C0F0044F0BA
:1068600020040AE044F0400407E044F0100404E08F
:1068700044F0300401E044F05004042A58600FD87A
:10688000DFE802F003060E090C0044F0010407E003
:1068900044F0030404E044F0020401E044F0040482
:1068A0001C6010BD10B5DFF86C4908212046FFF7C9
:1068B000BCFE18B900F004F80028FBD0606810BDD9
:1068C0001021DFF85409B0E680B500F0B1F8401CA3
:1068D00002BD491EE0E00000F8B50446201200F0B9
:1068E0000F000026401E09280D46DFF8307914D825
:1068F000DFE800F0051E141307202313262ADFF813
:10690000A077C4F3043416B13046FFF711FF2A46CE
:1069100021463846BDE8F84080E6F1BDDFF80009C1
:1069200000F015F8DFF8E018FFF793FE0837E8E706
:106930001037E6E730370126E3E738371026E0E77F
:1069400040374FF48036DCE7DFF8D878D9E770B508
:10695000DFF88C18DFF8D0480E68DFF85C28DFF825
:106960005C18012510F478105AD0B0F5003F27D0FC
:10697000B0F5802F1ED0B0F5002F51D0B0F5202FEC
:1069800024D0B0F5402F43D0B0F5602F4DD0B0F5F6
:10699000901F38D0B0F5A01F21D0B0F5B01F27D080
:1069A000B0F5D01F19D0B0F5E01F1FD0B0F5001F13
:1069B00029D039E000F015FF6168C1F308210AE031
:1069C00000F00FFF2168C1F3082104E000F009FF87
:1069D000E168C1F30421491C12E0104615E010469D
:1069E000FFF76CFEA16901F00F0107E008460CE01B
:1069F0000846FFF763FE216A01F0030105FA01F181
:106A0000B0FBF1F611E0DFF8B807FFF757FE09E039
:106A1000DFF8180800F0CAF8072806D0082803D1C4
:106A200000F0DFFE064600E00026304670BD0000A4
:106A3000031103F00F0301225B1E072BDFF89417ED
:106A400028D8DFE803F004060A0E10141C27086893
:106A500000E04869C0F3042070470868C0F3006094
:106A60007047C86800E08868C0F308207047DFF806
:106A7000C03798420ED1086A00F00F0006E0DFF838
:106A8000B437984206D1886A00F0030002FA00F099
:106A9000401E7047002070472DE9F8458A460111D5
:106AA00001F00F01491E0729DFF82877DFF870573A
:106AB000DFF88467DFF88487DFF84C4773D8DFE8B6
:106AC00001F004131A21273F546500F088FEFFF7F8
:106AD000D0FD21464046FFF7BCFD386820F4F85051
:106AE00040EA0A20386020E0786920F4F85040EA53
:106AF0000A20786157E0386820F0807040EA0A6028
:106B0000386050E0F868304040EA0A20F8604AE017
:106B100000F065FEFFF7ADFD21464046FFF799FD09
:106B2000B868304040EA0A20B86000F04BFEFFF73A
:106B3000A0FD2846FFF70BFF2146BDE8F44588E598
:106B4000DFF8FC16884225D0DFF8E41688422AD107
:106B50005046FFF778FD04460420FFF7E9FD386A48
:106B6000000944EA001038621DE0DFF8C8168842C8
:106B700019D15046FFF767FD04464020FFF7D8FDC6
:106B8000B86A800844EA8000B8620CE0DFF8B0160A
:106B9000884208D14FF48020FFF7CAFD386B000906
:106BA0004AEA00103863BDE8F185000000F00F00EC
:106BB0000121401E0528DFF88C263BD8DFE800F0D5
:106BC0000311153A2230506A00F00700022804D061
:106BD00005D3042807D01FD301E004212BE00521B1
:106BE00029E010690FE0022125E0506900F007005C
:106BF000401E03281FD8DFE800F00F020311F2E760
:106C0000062118E0906900F00700012804D002284E
:106C1000E9D0042802D00EE003210CE009210AE0AB
:106C2000106810F0010003D0012804D1082102E00F
:106C3000072100E00021084670472DE9F0410326B6
:106C4000032700F00F000128DFF85444DFF8B8856F
:106C5000DFF8EC5406D0022836D0032833D00528BC
:106C60002FD03EE00229DFF8D40506D003291ED03C
:106C700004291ED0052922D03DE004260027012248
:106C80000121384600F070F900F0A9FDFFF7F1FC92
:106C90006667DFF88C05FFF75AFE4146FFF7D9FC1F
:106CA00000F00FFF00F08EFDFFF7E3FC19E0012775
:106CB000E5E7022602274146FFF7CBFCDFE7012686
:106CC000F9E7083500E02D1D012908D0022914D06C
:106CD000032919D006291ED0092929D00BE000204C
:106CE000286010212046FFF7A0FCBDE8F0411821E4
:106CF000DFF8E00499E4BDE8F081012201210020E1
:106D000000F032F90220EBE701220121012000F01E
:106D10002BF90120E4E700F055FD4146FFF799FC0F
:106D200001220021DFF8F404FFF778FC0320D7E705
:106D30000420D5E7DFF8A41418B108680028FCD1B6
:106D4000012048607047DFF800050068704770B5A3
:106D5000DFF89024044694421FBFDFF88C2494424D
:106D6000DFF888249442DFF8E4042AD0DFF8842492
:106D7000944224D0DFF8802494421ED0DFF87C2493
:106D8000944218D0DFF87824944212D0DFF87424AB
:106D900094420CD0DFF87024944206D0DFF86C24C3
:106DA00094420CBF056B00250CE0C56A0AE0856AB9
:106DB00008E0056A06E0C56904E0856902E0C56887
:106DC00000E00568DFF88004046000F0B0F80528F2
:106DD00003D100F004FDFFF74CFC1821DFF8FC03A1
:106DE000FFF723FC0028F8D1DFF8F8138C420AD013
:106DF000DFF8F4138C4208D0DFF8F0138C4208BFA0
:106E000025F0C06504E0022000E0012060F35A652F
:106E100000F08DF80528DFF8F06303D131462046F5
:106E2000FFF717FCDFF82804056000F080F805285C
:106E300003D100F0C7FCFFF71CFCDFF8E403FFF709
:106E400086FD3146BDE87040FFF703BC38B5DFF87A
:106E500004341C6800F0804040F04055AC4309B158
:106E60004FF08051150014BF4FF00055002504432A
:106E700021432943002808BF002A19600BD000F0E5
:106E8000CBFC0446FFF7F5FB2046BDE83440DFF8B5
:106E90007813FFF7DEBB31BD10B500F047F80122D3
:106EA0000021022000F060F82069002202282078EA
:106EB00008BF012208B142F4807240F20111DFF8EC
:106EC0009403FFF7B9FBE27ADFF88C030721FFF7A1
:106ED000B3FBA088617A41EAC022DFF88013DFF8B3
:106EE0008003FFF7A9FB207AFFF7E0FB227AE18815
:106EF000D20142EAC121A27A114340EA01026FF0B5
:106F00007F61DFF86003FFF797FB617B207B09035C
:106F100041EA0040A17B40EA0110E17BBDE810405E
:106F200041EA0002D049D148FFF786BB0446112050
:106F30003CE600207047704710B5FFF7F7FF0022CE
:106F40000021002000F010F82078617840EAC1208C
:106F5000A17840EA01606168BDE8104040EA012282
:106F6000C349C448FFF768BB2DE9F84F04288046A1
:106F7000924674D8DFE800F04B463C0341000126FE
:106F80000220012700240029DFF88C92B14D5DD04A
:106F9000B8F1020F04BF286810F0300F4FF0000B5B
:106FA0000AD12868C0074FF0010B05D5286820F0EA
:106FB000300040F010002860EE6300F052F8002826
:106FC000FBD0BAF1000F46D0394600F04BF800284C
:106FD000FAD0B8F1020F3ED1BBF1000F3BD02868C8
:106FE000C0071BD501222021022000F0CBF819E0B8
:106FF0000426082003270224C5E7102620200527A1
:107000000424C0E74026802007270624BBE74FF46E
:1070100080764FF4007009270824B4E7002102208D
:1070200000F090F8022000F021F80446012200212F
:107030000220FFF799FF2146022000F037F8EE63A7
:10704000394600F00FF80028FAD004E0E86300F0B9
:1070500008F80028FBD1BDE8F14F00F032BDBDE8D3
:10706000F18F21464846FFF7E0BA0000401E032892
:10707000774912D8DFE800F0020C06080869C0F36F
:1070800008007047086800E0886800F07F007047DB
:1070900079480068C0F30A0070470020704700007C
:1070A00000400E4004000E407F4573FE70B5401E48
:1070B0000C46032804F07F01654D484E3FD8DFE8B9
:1070C00000F0022A101DC4F308041A213046FFF70D
:1070D000ACFA0028F9D12869400A44EA4020286126
:1070E00070BD0C4618213046FFF79FFA0028F9D1F1
:1070F0002868C00944EAC010286070BD0C461921F8
:107100003046FFF792FA0028F9D1A868C00944EA8E
:10711000C010A86070BD534E306E686920F030001A
:1071200040F010006861C4F3C310FFF7BFFA40EAF3
:1071300004023046BDE870405049FFF77DBA70BD8B
:1071400080400E404348026812F0300F18BF0029FB
:1071500007D0202902D0302903D005E04FF40001E8
:1071600003E04FF4400100E04549C26E0A408A4204
:10717000FBD1490204D5C06F800A00F001007047BE
:107180000120704710B5022809D121B13D4B4FF4C1
:1071900080645C64196012B1BDE81040D2E7012040
:1071A00010BD30B91F48006810F0020002D0012065
:1071B000704700207047000002001A0003001C0006
:1071C00005002000002201B101224000411C1548A9
:1071D000FFF724BA00410E40809FD50040410E4089
:1071E0002000002040420F0080841E0000093D0066
:1071F0009082E00FC0CF6A00405DC6000024F4001A
:10720000C0EA210180BA8C010048E80180D5430220
:1072100018400E4050400E4090400E40B0400E408E
:107220000005080050410E4008410E4006000C00C9
:107230006006140070071600FF00FEFF0148E80119
:107240008009120070400E40180000203082E00FCC
:1072500010400E4024400E4028400E407FF80F00A2
:107260002C400E4030400E40FFF00F0034400E40E6
:107270007F1B000738400E409C400E40FF0700F087
:10728000FF03F10764400E400146DFF8880390F9E0
:10729000000000F0C4BF10B582B01868DFF87813A2
:1072A000DFF8784348600023DFF8740308600120AA
:1072B0000090002224680820A047002016BD10B5C9
:1072C0000446002200210020FFF7C0FD0521112007
:1072D000FFF7B3FC002200210220FFF745FED14852
:1072E000D14A01686FF3D321016002EAC422016828
:1072F00011430160012201210220FFF735FE042124
:107300001120FFF79AFCBDE8104001220021002067
:10731000FFF79CBD80B56A460021322001F0ABF931
:1073200018B9BDF80000FFF7CAFF01BD70B50446EB
:10733000BE480078A8B1BE4DBE492E680968301914
:10734000884201D3002070BD22460021304601F062
:1073500009FA28682018C01C800880002860304680
:1073600070BD2046BDE8704000F0EFB901F006BAEC
:107370002DE9FE4F044601F0AEFB04F1A80504F12F
:10738000A106002C2868DFF8AC92DFF8A4A21ABF8F
:10739000F778002F04274FF01E0830B1CAF800001C
:1073A000A9880844C9F800000120DFF880B2A2498A
:1073B0008BF80000062000F074F900230022002161
:1073C000002000F043F900233A466821022000F033
:1073D0003DF9384601F006FC9BF8000040B1D9F8B1
:1073E0000000DAF80010001F401A5C21B0FBF1F831
:1073F00000235FFA88F25521012000F027F900F000
:10740000E4FE01F0C6FC34B9002001900090012395
:10741000002200210DE0206800F0080101918008A1
:10742000296A009100F0010080F00103EA69A9696E
:10743000686901F048FF00F06BFF207800060ED469
:1074400004F1D80304220021352000F0D3FF04F119
:10745000DC00436802780021362000F0CBFF02F008
:1074600058F9FFF757FF2068800900F001076D48C1
:1074700000680003C00DADF802006A460021342008
:1074800001F0F9F848B9BDF80000BDF802108842D3
:107490000AD017B1FFF713FF06E00DF10203022235
:1074A0000021342000F0A6FF00275CB130784007AF
:1074B000207848BF01274007286948BF002708B146
:1074C00001F05CF902F0FDF90020029002AB01AA84
:1074D00000212C2001F08EF800281FBF9DF8040029
:1074E000062800200290686A02F02DFA1CB90020DC
:1074F0000023012108E021682B6A490801F00101FD
:1075000004F1D00081F0010100902046029A01F0C0
:1075100076FE02F037FA49484949006808601CB114
:1075200004F1B30001F04EFF0021464800F068FE70
:1075300038490870002F0CBF0220032002F0EFFB37
:10754000BDE8F78F80B500F04DF808B1002002BD0E
:107550003A48006802F055FC10F1010F02D14FF0DB
:10756000FF3002BD4FF47A71A1FB0001C00B40EA6D
:10757000414002BD80B510F1010F0FBF4FF0FF3049
:10758000C0034FF47A71B0FBF1F002F063FD4FF4E9
:107590007A714843C00B02BDF8B5044602F04AF9BF
:1075A000274D08E002F0A2FD0646384602F052FDE3
:1075B000304602F09FFD214800682860286802F0EC
:1075C000C9FD074602F03FF938B901F019FC00F097
:1075D0003EFE0028F2D1002CE4D1F2BD0120DBE711
:1075E0000020D9E780B500F060FE20B9134800689C
:1075F00002F0FAFB00B1012002BD80B512490B7800
:10760000984202D140F2811002BD087002F0CCFD18
:10761000002002BD3C140020FC0700205005002083
:10762000A004010330400E4000F80F003D1400207C
:1076300040050020440500202D7300000820044070
:10764000DC040020977200003E14002070B5144640
:10765000C91C4FF6FC721140C91C02EA01052849F9
:1076600001EB00160020274935807480F06004FB90
:1076700005F009688847706015FB04F1318189B213
:10768000706802F099FD002007E0716800FB05F2C8
:107690001144F2680A60F160401CA042F5DB74807E
:1076A00070BD184A1160506001011548FEF7B2BF65
:1076B000134901EB0011C86820B10268CA604A880A
:1076C000521E4A8070470E4901EB00104088C0B23C
:1076D00070470B4A02EB0010C2680A60C160418823
:1076E000491C41807047000105490A5A2AB10A180D
:1076F000085A128992FBF0F0704700207047000092
:10770000E0040020F407002001B40E4800E0083037
:10771000416899B101789DF8002001F0F80102F06C
:10772000F802914202BF81789DF80220914202BF87
:10773000C1789DF803209142E9D100E0002001B01A
:1077400070470000D8520000704738B5C01C84084C
:10775000A00002F035FD050001D1002032BDA100DE
:1077600002F02AFD284632BD38B50446FFF7EDFF8A
:1077700005001CBF214602F01FFD284632BD4843CC
:10778000F2E702F075BD022862F30F2262F31F4296
:1077900000B500BF130096469446103928BFA0E8F4
:1077A0000C50FAD85FEA417C28BF0CC048BF40F8B3
:1077B000042BC90728BF20F8022B48BF00F8012B73
:1077C00000BD022880B500F00CF82749274A096857
:1077D000C1F30821491CB0FBF1F0106002BD244840
:1077E00070472448016801F00701022909D00AD333
:1077F000042901D002D306E01F4905E04FF40041FF
:1078000003E01E4900E01E490968C06EC0F3042071
:10781000401CB1FBF0F070471848006870471749EA
:1078200008601448006800F00700022808BFFFF74E
:10783000C9BF70471348016841F470010160704787
:107840004FF4004070474FF47A7070470A48006860
:107850007047094908600748006800F007000428DD
:1078600008BFFFF7AFBF704708410E404C0500202E
:1078700000F0490294400E40140000201000002047
:107880001800002088ED00E0890001EB401000F1B5
:10789000844002607047890001EB401000F1844091
:1078A0000068704710B5DFF87C08016845F60E02E5
:1078B00002600023DFF870281268D40748BF012354
:1078C000D40648BF43F01003540648BF43F04003BA
:1078D000540748BF43F00403D205DFF8502848BFDF
:1078E00043F48073D363DFF848381B7803F0070351
:1078F000022B10D01ED3042B08D01BD213689B0080
:1079000018D4D36E1B06FCD5032312E0D36E9B055F
:10791000FCD504230DE0D36E1B07FCD5136813F0D0
:10792000300F05D1D36E03F44003B3F5400FF9D106
:1079300002231365C90744BF0021016010BDDFF8B1
:10794000F417DFF8F42738B110680860106820F4E5
:107950007F4040F4EE4000E008681060E2E0DFF8AD
:10796000DC070168012918BF02290BD1DFF8D01705
:107970000A6802F00302012A02D1CA6BD203FCD5C5
:1079800003210160704738B50446DFF8B807DFF817
:1079900098270168DFF8985711604068288000F048
:1079A00039F8FFF7DCFF30BF0020FFF7C8FF04B154
:1079B00038E0287800F00700012800D035E031BD1C
:1079C00038B50446DFF88007DFF85C27016BDFF885
:1079D0006057116045F60E03416B2980DFF84417AC
:1079E0000A680B604FF420730360D00744BF002087
:1079F000086000F00FF8FFF7B2FF30BF0020FFF77C
:107A00009EFF04B10EE0287800F00700012800D0A6
:107A10000BE031BDDFF83407016841F0040101607B
:107A200001208CE7BDE831403CE7BDE83140FFF77D
:107A3000C9BEF8B5DFF81847206920F4403040F49B
:107A4000003520694AF6E85740F44036276020693F
:107A5000C00708D4A06B00F00300012812BF022861
:107A6000002000F09DF82069C0070DD572B6DFF840
:107A7000E4060760816841F080018160DFF8D80684
:107A8000016841F4807101600120FFF758FFFFF7A2
:107A900066FF04202561401E2661FBD12561F1BDF2
:107AA00080B5012201E080B500220021DFF8AC069C
:107AB000FFF7EAFEBDE80140BBE7DFF8A416086067
:107AC0007047DFF88006DFF86026016811604068C3
:107AD000DFF85C16088070470078DFF88816002809
:107AE000086812BF40F0010040084000086070477D
:107AF00070B5DFF868160A680378920903B10423A9
:107B0000447804B10224857805B10825466806B199
:107B1000012643EA821222432A43806832431043FB
:107B2000086070BDDFF84026DFF80C060168128897
:107B300002F12803C1F3032103EBD373491C02EBC9
:107B40006302283201EB8103B2FBF3F2521E036899
:107B5000072A34BF12064FF0E06223F0EE631A43A7
:107B600042F480120260DFF80426B2F90020002AF5
:107B700015D492B202F1280303EBD37302EB630234
:107B80004B08283203EB4101B2FBF1F142680729AF
:107B900034BF0901702122F0700211434160704727
:107BA00070B5DFF89C550446286800F00306A6422D
:107BB00017D0DFF8BC05416AC907FAD4220018BF04
:107BC00001220D21FFF760FE002E08BF012C03D11A
:107BD000DFF86815022008602868800844EA800001
:107BE000286070BDF8B50446DFF888152068086085
:107BF000096801F00F01814240F09880DFF87805B4
:107C0000006810F1010F13D0DFF8700541680268B9
:107C10001160C16882681160416902691160C169BF
:107C200082691160416A026A1160C16A806A0160FA
:107C3000A0894B28B8BF00200DDBB0F5FA7FB8BF94
:107C40004FF0805007DB40F6C4118842B4BF4FF0BC
:107C500000504FF04050DFF82855DFF828352969EB
:107C6000B4F91420DFF8D0641940D243084340EA45
:107C7000D270286100213046FFF70DFE316A41F0D5
:107C80008071316200B1042000F05DF9706920F06C
:107C9000C0407061306840F006003060DFF8E804F2
:107CA0000068C0F30747684602F022FBA7F1100006
:107CB0000C2803D3512F18BF532F19D19DF8010061
:107CC000012815D19DF80000032811DADFF86C04B3
:107CD000016869B9A968DFF8B42441F00101A9601D
:107CE00071691140DFF8A82411437161012101601D
:107CF000E089DFF874140880A08ADFF87014088027
:107D00006089DFF89014088000F0EAF8A06920B1DB
:107D1000012805D1DFF8800401E0DFF88004F0607D
:107D200020890122012100F00FF808B90020F2BDDE
:107D3000226902B1012205212846FFF7A5FD6068EE
:107D4000FFF72EFF0120F2BD2DE9F74FDFF82404E5
:107D5000016801F00F0100260229B44640F0B2800C
:107D60000099A1F5E161B1F5966FF7D80021DFF830
:107D7000302400E041B99DF80430002B09D051B9FE
:107D800000F12C03012409E0012904BF9DF808300B
:107D9000002B00F09E8000F124030824009DB5F51F
:107DA000E16F0ED94FF0010E4FF4E16840F6B8399B
:107DB00059B315684FF0020A4FEA156CC5F3074630
:107DC00071E04FF0000E4FF496684FF4E169F2460F
:107DD000E9B9456905F0405555EA0A0723D07F1EE9
:107DE00011D06FF0704BB7EB0B071ED07F1E14D075
:107DF000B7EB0B071BD07F1E11D0B7EB0B071CD0C6
:107E00007F1E0ED01EE0D66812E0F246E1E715684C
:107E1000C5F3072C05F0FF0645E0D6680EE01669AD
:107E200006E016690AE0566802E0566806E09668C1
:107E3000C6F3072C06F0FF0604E096684FEA166CBE
:107E4000C6F30746DFF85C733F68FFB2042F08DA19
:107E50005569BEF1000F0CBF05F0FF0EC5F3072EEC
:107E600015E097698DB1B5F1805F0BD0B5F1005F7A
:107E700005D0B5F1405F25D14FEA176E07E0C7F393
:107E8000074E04E0C7F3072E01E007F0FF0E4FEAAC
:107E90000E3737F4704515D1456B25F470453D43D9
:107EA000C84545630ED2009DA5EB0807ACEB06055F
:107EB0007D43A9EB0808B5FBF8F8B044C44528BFDA
:107EC000B04501D2002009E008FA04F44AEA0404AB
:107ED0001C60491C0229FFF64DAF0120BDE8FE8F52
:107EE00010B595494B6A0C68E4074FF0FF3203F078
:107EF000070312D5022B10D3142815D314381428D5
:107F00001FD30F22086820F47F4040EA022040EA95
:107F100002300860BDE8104004E60C68E40709D4AC
:107F2000022B07D20A2801D20322EBE70A380A28DB
:107F300007D3E6E70C68E407E4D5022BE2D2282851
:107F4000DFD20722DEE738B504467B4D0021284604
:107F5000FFF7A1FC686AC00844EAC0006862BDE897
:107F600032408C480088BBE7824802210160016CE6
:107F7000C907FCD4032181608068032801D1012056
:107F8000704700207047A0F59660C82202FB1100E0
:107F90001421B0FBF1F07047B0B500F066F8276827
:107FA00081490302032F43EA053214D8DFE807F0C2
:107FB00002141B22227A02B10422677A07B1082731
:107FC000000440EA055040EA053018431043A27A05
:107FD000384310430860B0BD207A00B1042000F09F
:107FE00019F84860B0BD207A00B1042000F012F802
:107FF0008860B0BDE07A00B11020237A03B1042379
:10800000657A05B1082510431843A27A2843104326
:10801000C860B0BD637A03B108231043A27A184345
:1080200010437047F8B500F020F80646A068A0F5A8
:108030009661C82291FBF2F73946FFF7A4FF216849
:1080400091B9217B01B10421627B02B10822330482
:1080500043EA055343EA073343EA00200843A17B80
:108060001043084350490860F1BD0446C8226068C7
:10807000A0F5966191FBF2F5294684E703284A4B67
:1080800008D8DFE800F002080A0C0A46002118466A
:10809000FFF7FABB70471B1DF7E70833F5E70C3312
:1080A000F3E7000080B503280BD8DFE800F00204F6
:1080B0000608012106E0022104E0032102E0042178
:1080C00000E000213948FFF7E6FB00B10120C0B213
:1080D00002BD10B50221002300B90021344AD46A40
:1080E000012C03D14AF6E8540123D4620228106817
:1080F0000CBF20F0740040F074001060906B40F0F2
:10810000080090632B48046824F4406444EA812109
:108110000160906B20F0080090630BB10020D062EA
:1081200010BD000080410E406405002024400E4038
:1081300028140020680500204C300E406005002007
:1081400040300E4090400E4060400E4010ED00E088
:1081500008300E4090310E4088300E4018300E40EE
:108160000C300E4000300E402A1400202E14002047
:1081700054300E4038300E401C83E00F3880E00F42
:108180003C300E40FEFFFFCFFC81E00F000F0EF0F1
:10819000B4C0400B2C140020372110B77740205773
:1081A0001883E00F0082E00F90300E4004300E4044
:1081B00064310E403C400E40890001EB401000F15C
:1081C0000850026070470122F6E73A480021C0E9F2
:1081D000001139482821FEF71DBA36494A68D043B4
:1081E00090FAA0F0B0FA80F0C0B2052802DB4FF0A0
:1081F000FF307047012383401A434A6040B2704702
:1082000070B504460D46FFF7E8FF06462A482A46A1
:10821000214600EBC60001F08BFE304670BD10B564
:10822000052809D200F009F852E8003F0B4342E864
:108230000034002CF8D105E010BD1F4B03EBC00249
:10824000121D7047BDE81040C1B21A48BBE770B5B7
:1082500082B01A4C174D00E02070286820B32678B1
:108260000121B140084219D0002231462846FFF7CB
:10827000A3FF114800EBC600011D002351E8002FA9
:1082800041E8003CBCF1000FF8D11100009205D08C
:108290006A460B4901F093FE012076BD686886426C
:1082A00034BF701C0020D7E776BD0248006800B1DB
:1082B00001207047B4070020BC07002040140020B4
:1082C0007856341210B5044602F031F80021201D12
:1082D00002F032F8012104F1080002F02DF8221D0D
:1082E000082100F083F90146204602F025F800201D
:1082F00010BDC0F30A010831B1F5006F04D28088C7
:108300004FF6FF71884201D101207047002070476D
:1083100010B502F007F802F015F8DFF84044A0F5B8
:108320008050206002F00EF8A0F500606060082127
:108330002068021D00F05AF92168096888421CBFB4
:108340002068FFF7BFFF6068021D082100F04EF9AA
:108350006168096888421CBF6068FFF7B3FF206846
:1083600040686168496888428041DFF8F413C00FB3
:10837000087010BD2DE9FC4104464FF6FF75AC4274
:1083800014BF002840F212200E462AD000F0D7F881
:1083900050F8218008F10C073846FFF7AAFFF8B91A
:1083A000B888304006EA040188420ED1D7E90001BE
:1083B000CDE90001ADF80650BDF804006840ADF805
:1083C0000400381D019901F0B7FFB87900F005F9F4
:1083D00007EB800000F10807F80A00F004F8DBD092
:1083E0000020BDE8F68108F10C01C002C90AB0EB1B
:1083F000C12F70472DE9F84D80460EB44FF6FF703F
:10840000804514BF5FEA080040F212200D469346F3
:108410001F461FD000F093F850F8210000F10C0423
:10842000002600F10C0A2046FFF763FF00282DD13B
:1084300000F0D9F82168884204BFA08840451CD1CB
:10844000A079834507D102985A4604F1080101F04A
:1084500083FF00286AD0D4E90001CDE90001BDF80E
:1084600004004FF6FF714840ADF80610ADF8040067
:10847000201D019901F060FF064600F0F0F800F0C1
:1084800058F808BF002ECED0002E4AD15FEA0B006C
:1084900048D004EB0B000830C00A00F04AF80ED0B8
:1084A00000F004F90446C4F30A00002804D058443C
:1084B0000830B0F5006F02D940F2015036E04BEAC7
:1084C0000520ADF80480ADF80600251D019926466B
:1084D000284601F031FF2C1D00250FE0387879780F
:1084E00040EA0120B97840EA0140F97840EA0161A8
:1084F000204601F021FF3F1D241D6D1C38B90BF1F2
:108500000300411000EB9170B5EBA00FE6DB321DCC
:108510000BF1040100F06AF80146304601F00CFF4F
:1085200006460EB9002001E04FF4C67004B0BDE865
:10853000F08DC0024FEADA21B0EBC12F70478849B5
:10854000864891F9001070472DE9F0470C468449A0
:1085500091F900100746814850F821A01546994628
:108560000AF10C0846463046FFF7C3FEE0B9B07981
:10857000011D321D00F03AF83168814218BF7F1C9E
:10858000F088FF2190FBF1F1C1EB0121401A00F0CE
:1085900024F808EB800000F108084FEAD8200AF11F
:1085A0000C01FFF722FF02D040F2025012E03846E1
:1085B000471EC0B20028D5D1B088208015B1F08800
:1085C000000A2870F08889F8000006F10800089970
:1085D00008600020BDE8F087A879C01C411000EBBE
:1085E000917080107047A079011D221D4FF0FF305F
:1085F00001F0E4BE2DE9F8430D46594991F9001008
:108600008146564850F8218016461F4608F10C0452
:108610002046FFF76EFEC8B9FFF7E5FF21688842E4
:1086200004BFA08848450CD184B115B1E088000A88
:108630002870E088307004F1080038600020BDE840
:10864000F28300F00CF8FFF7CEFEE1D00DB1002070
:10865000287000203070386040F20250EFE7A079B7
:10866000C01C411000EB9170801004EB800000F101
:108670000804E00A70471CB514466B4601AAFFF7D0
:10868000B9FF10B99DF8040010B940F2025016BDB0
:108690000098007820809DF80410022904DB0099DE
:1086A000497840EA01202080002016BD2DE9F047DE
:1086B0002B4C2A4994F9000051F8209080F00100D9
:1086C00051F82070384601F032FE09F10C0A07F12A
:1086D0000C0805E0FFF780FF0AEB800000F1080AB4
:1086E0004FEADA2009F10C01FFF77FFE1BD1554656
:1086F0002846FFF7FEFDB0B9A879011D2A1DFFF736
:1087000075FF29688842E5D10026FFF765FF801CC8
:108710008642E5DA5AF8041B404601F00DFE08F1E6
:108720000408761CF1E7D9F80400411C381D01F05B
:1087300003FE012107F1080001F0FEFD3A1D0821AA
:10874000FFF754FF0146384601F0F6FD207880F02F
:10875000010020704046BDE8F0870000900800202E
:108760005B02002010B5044610460A46014620462A
:1087700001F03CFE204610BD01F076BE01F08EBE39
:1087800080B501F081FF00B9C6E0BDE8024002F00B
:1087900003B938B500F047F8050000D17AE020466B
:1087A00002F04EFE10B94FF4C07032BD214628468B
:1087B0002269BDE83840D2B202F07AB910B500F0B3
:1087C00032F800B90EE02146BDE8104002F096B93B
:1087D00010B500F028F800B904E02146BDE81040CB
:1087E00002F01FBA40F2011010BD70B500F04EF853
:1087F000060000D125E0284602F022FE00B937E04D
:108800002A46214630462B69BDE87040DBB202F0B3
:1088100097BA10B500F007F800B9E3E72146BDE8C4
:10882000104002F0ABBA0C4601F02EBF70B500F05C
:108830005BF800B905E000F046F8BDE8704002F0D2
:1088400026BB40F2011070BD70B500F01FF80600A5
:1088500000D1F6E7284602F0F3FD00B908E02A4609
:10886000214630462B69BDE87040DBB202F034BBD4
:108870004FF4C07070BD38B500F008F800B909E0D9
:108880002A462146BDE8384002F044BB0C46154656
:1088900001F0FABE40F2011032BD70B500F024F8CC
:1088A00000B9CEE700F00FF8BDE8704002F048BB19
:1088B00070B500F019F800B9C3E700F004F8BDE89E
:1088C000704002F053BB33462A462146704770B5CC
:1088D00082B000F009F800B9AEE006990091FFF708
:1088E000F2FF02F051FB76BD0C4615461E4601F024
:1088F000CBBE10B5FFF797FF00B973E72146BDE87F
:10890000104002F058BB80B501F0BEFE00B903E094
:10891000BDE8024002F082BD40F2011002BD10B578
:10892000FFF781FF00B95DE72146BDE8104002F086
:10893000CBBB70B5FFF7D8FF00B982E7FFF7C3FFE5
:10894000BDE8704002F0D2BB38B5FFF79FFF00B919
:10895000A0E72A462146BDE8384002F03CBB7CB582
:108960000E4615461C46014601AB6A46002003F040
:1089700007F80146019828B100202080019800F5F1
:10898000806076BDBDF80000B04204D20020208097
:1089900040F2074076BD801BADF8000031442088CE
:1089A000BDF80030984238BFADF80000BDF80000B7
:1089B00018B102462846FDF741FDBDF800002080B1
:1089C000002076BD38B50C46154603F0FDF84FF68D
:1089D000FF71884204D10020288040F2014032BD5E
:1089E00001044CBF102102212980214602F060FDC4
:1089F000002032BD38B504460D46D9B2104603F00A
:108A000031F9030002D14FF4C17032BD2A4621462C
:108A1000002002F0F0FF08B100F5806032BD70B5B3
:108A200082B0FFF761FF00B906E0069B0095324671
:108A3000214604F061F976BD40F2011076BD38B5EB
:108A4000FFF724FF00B925E72A462146BDE8384054
:108A500004F06FB9F8B50024FF280D4616461F46EE
:108A600006D001F011FE040002D140F20110F2BD67
:108A70003B4632462946204601B0BDE8F04004F0AE
:108A800000B970B50C4615461E4688B10146204611
:108A900002F0DFFC02464FF6FF70824208D0290048
:108AA00008BF01250146284603F04BF8010002D11A
:108AB00040F20A4070BD16B940F2014070BD3080EE
:108AC000002070BD41F0010104F075BA204A02EBAC
:108AD00080000164704700B583B01E490020FFF795
:108AE000F5FF1D490120FFF7F1FF1C490320FFF7A7
:108AF000EDFF1B490420FFF7E9FF1A490520FFF7A6
:108B0000E5FF19490620FFF7E1FF18490720FFF7A5
:108B1000DDFF17491920FFF7D9FF16491B20FFF782
:108B2000D5FF15491C20FFF7D1FF14491D20FFF781
:108B3000CDFF13491E20FFF7C9FF1248044A006801
:108B40000021019100913223322104F03AFA07BD4D
:108B50000003002089950000ED770100F577010002
:108B600021780100FF770100FD77010019780100ED
:108B7000650A020009780100117801002B08010044
:108B8000690A020008ED00E070B5040048BF04F077
:108B900080FA600048BF05F072F9A00048BF06F0F7
:108BA00022FAE00048BF06F074FD200419D0A4B2F8
:108BB000002594FAA4F0B0FA80F0012101FA00F641
:108BC000C0B205F0D0FCB44318B105F0E8FC00B920
:108BD0003543002CEDD125B12846BDE8704000F0AA
:108BE000A7BE70BD05F049BF80B506F0FCFE04F0DD
:108BF0004CFA06F0DCFC05F03AF805F064FFBDE83D
:108C0000014007F04DB80228002105E0827A511892
:108C1000427A0068891AC9B20028F7D1084670471D
:108C200080B500F0EDF8012002BDDFF8C40490F932
:108C300000000121FFF7F3BA2DE9F04786B0804626
:108C40000E4692461D468DF804800296ADF80CA0A3
:108C500004950E9CDFF89C04DFF89C948DF814407A
:108C6000076806E001AADFF89414384607F026F9F1
:108C70003F68A7B197F83C0000F00A000A28F7D136
:108C8000D7F804C0BCF1000FECD000942B4652463C
:108C900031464046E047D9F800000028E8D006B049
:108CA000BDE8F087416A00291CBF243003F040B9B9
:108CB000704738B50446E069002837D000F014F951
:108CC000A0B3002003F046F8009078B3807A0099B2
:108CD000DFF82C543C308872002004E0009B1944DB
:108CE00001440A74401C0099009A497A927A521AF7
:108CF00090420AD218B9009B5E221944F1E7521E35
:108D000090420CBF21222A78E8E76946204600F00D
:108D10000AF9009810B1684603F00AF92878401C57
:108D20002870C0B23A28A4BF3020287031BDDFF8C7
:108D3000D40300784FF48071401CC0B2FF2804BFF8
:108D4000401CC0B2DFF8AC2303E092F83E3083420F
:108D500003D01268002AF8D17047491EECD1FF20D9
:108D6000704738B5FFF7E3FFFF2801D1002032BD7F
:108D70004420FEF7EAFC040009D0442101F01CFA6B
:108D800004F13E05FFF7D3FF2870012068702046EC
:108D900032BD80B50021DFF87003FFF731FADFF84C
:108DA0005013087000F01CF9FFF7DBFFC0B1011D84
:108DB00000220A604A600623DFF850238A60DFF849
:108DC0005023CA6000F13C0213701023CB621F23B2
:108DD000937000230B620121D170BDE8024000E0D6
:108DE00001BDDFF810130A680260086010F83C1F2C
:108DF00041F0010101708078DFF8081308707047B6
:108E000010B5DFF8F00204682DE0204600F084F988
:108E100094F83C00C00744BF2046FDF74EFB94F891
:108E20003C0000F0FE00810784F83C001AD54007A2
:108E30000BD5216908001CBF20468847606A20B115
:108E4000E16808001CBF2046884794F83C000007F2
:108E500008D5A068010005D0804718B1014620461A
:108E6000FDF74CFB2468002CCFD1002010BD38B595
:108E70000446251D0020E861A86184F83C00686074
:108E80002860A860686A28B104F1280003F050F84F
:108E900000206862286A28B104F1240003F048F831
:108EA00000202862934809E08169A14204BF0021A3
:108EB0008161C169A14204BF0021C161006800282D
:108EC000F2D131BD10B50446FFF7D1FF894800E06B
:108ED0000846016819B1A142FAD121680160204613
:108EE000BDE81040FEF74DBC08B90120704700F105
:108EF0003C010A7802F00603062B11D150F80C3F12
:108F000073B1C97801B901218069002201E00068CC
:108F1000521C0028FBD1D2B28A428041C00F704758
:108F200002F0020070472DE9F04704460D46E6695D
:108F3000FEB196F83C10301D01F0060106290FD154
:108F4000816869B12868FFF75FFEA16B0818A0630C
:108F500006F12400296803F0BFF800F095F80FE04F
:108F60000068010005D0FDF7A5FA02E0304602F0E6
:108F700044FF284603F09DF8060003D100F030F8C6
:108F800000202BE0707AB17ADFF86C9100F076F86F
:108F900009E0A06B5044A063A7EB0A07707A504425
:108FA0007072D044BFB2002FE0D0FD2FACBF4FF0A5
:108FB000FC0ABA4642465FFA8AF12046FDF7B1FA4A
:108FC000D9F800000028E4D03146284603F0D5F84F
:108FD0000020C9F8000000F003F80120BDE8F08788
:108FE0004C48FDF767BA2DE9F8435FEA00090D46E2
:108FF00006D1284602F09CFF00202860BDE8F283DD
:1090000009F1040699F83C0000F00600062810D18A
:10901000B06870B12868FFF7F7FD316B081830634E
:1090200009F12400296803F057F800F02DF800201A
:10903000E4E73068010005D0FDF73CFA02E0304675
:1090400002F0DBFE284603F034F8060002D1FFF7F9
:10905000C7FFECE7707AB17A00F010F807E04246FB
:10906000E1B24846FDF75DFA3F1BA044BFB2002FB6
:10907000E5D0FD2FACBFFC243C46F0E70F1A30448E
:10908000BFB200F110087047002028600121184885
:1090900090F90000FFF7C3B8164A12683AB1136B93
:1090A000834204BF136A8B42F7D1104670470020F9
:1090B00070471049096800291CBF91F83E20824280
:1090C000F8D10846704710B5044694F83C00626930
:1090D00020EA0101100002D02046904701E084F808
:1090E0003C1094F83C0040F0010084F83C0010BDB6
:1090F00041140020800800208408002002000100A4
:109100005A02002042140020218C0000A58C00008F
:10911000B38C0000398C000038B5044604F13C05DE
:109120006878C00713D52878400610D52046FFF789
:10913000DBFE60B1287800F0BF002870402168781D
:1091400000F0FE0068702046BDE83440BBE731BD4A
:1091500070B588B006460C46154602A8DFF8B8136D
:109160001422FDF77BF9DFF8B403D0E90023CDE941
:10917000002316B31422314602A806F0CDFE0420C7
:109180008DF8160002A8FDF787FE04211120FDF7D7
:1091900054FD002200210320FDF7E6FE0121DFF847
:1091A0008003FDF799FB0121DFF87803FDF794FBBD
:1091B000012200210020FDF749FEE4B108222146EA
:1091C000684606F0A9FE6846FDF7B6FE002D14BFFE
:1091D000022403242146DFF85003FDF72EFD21462B
:1091E000D248FDF72AFD2146D148FDF726FD012191
:1091F000D048FDF771FB08B070BD70477047F0B5FF
:109200008FB0054614980C4600281CBF0178002931
:1092100016461F4601D0407800B10120C6490860BB
:109220005020ADF80C0003AA00213120FFF723FAEB
:10923000BDF90C0000F02EF93FB12422394604A8F4
:1092400006F06AFE04A806F074FE0021705C10B9F6
:10925000491C0629FADB0629B8480AD00021725CAD
:10926000FF2A02D1491C0629F9DB062918BF002E66
:1092700017D1B349D1E90023CDE900239DF80010AF
:1092800001709DF8011041709DF8021081709DF8E9
:109290000510C1709DF8061001719DF8071041710D
:1092A00003E00622314606F037FEB5F8AE00ADF811
:1092B000080002A8FFF798FC204606F0C2FE07F05F
:1092C000B6F80FB0F0BD2DE9F04107460C4690B05E
:1092D000154698469B499C4800F0EDFC9B48006869
:1092E000060E684601F004F88F2E13DA9848994E5E
:1092F000016841F0040202604FF0501300224FF069
:10930000300E0EFB02FE521C46F80E30062AF6D333
:10931000016001E0902E06DA8F480168C909C90191
:1093200041F0200101609DF80100012804D18B4823
:10933000016841F00401016008A889491C22FDF779
:109340008DF857B117F1100F02D10020099004E0F9
:109350001C22394608A806F0DFFD08A8FEF742FCEB
:109360001798D8B103A87F491422FDF777F87E48F3
:10937000D0E90023CDE9012324B11422214603A81A
:1093800006F0CAFD25B10822294601A806F0C4FD51
:10939000424601A903A8FFF7DBFE04E04246294646
:1093A0002046FFF7D5FE01217048FDF795FAFEF73C
:1093B000CBF900F048FD07F0ABF907F015FA10B053
:1093C000BDE8F08138B50446207800285CD094F9D7
:1093D0000110674D11F1010F28D000F056F842F24C
:1093E0000200286694F90100801F05281AD8DFE8DA
:1093F00000F00305090D1115286912E0286940F4F1
:1094000080300EE0286940F400300AE0286940F41A
:10941000403006E0286940F4802002E0286940F4EA
:10942000A0202861286840F48060286094F9021028
:1094300011F1010F28D000F028F842F2010068660F
:1094400094F90200801F05281AD8DFE800F003070E
:10945000090D1115286940F0A06010E028690EE0A0
:10946000286940F080700AE0286940F0007006E04A
:10947000286940F0407002E0286940F0806028616F
:10948000286840F40060286031BD002304220220D7
:1094900007F012BA30B585B00446ADF80C0004F1FF
:1094A0007D007E288041C00F019023480068029013
:1094B0000020ADF80E000420ADF8100001A807F060
:1094C00038FA204607F0E6FD04B242F60720ADF870
:1094D00002000DF10201022001F0BBFF02464FF62F
:1094E000FF71012002F02DFB050012D0012CACBF52
:1094F000601D601F0A2190FBF1F08DF80000012132
:10950000684602F0AFFB034600222946002002F025
:1095100072FA204605B030BDAC590000C0590000B9
:10952000002508000055080002001A0003001C0076
:1095300005002000000508002C000020E4070020A2
:10954000F081E00FFD910000FB910000FC81E00F35
:10955000B0400E4000A000402C400E4064310E4050
:1095600090590000C8590000DC590000003508007F
:1095700008600E40012100F01F029140DFF86822D0
:10958000400942F82010704700BF38B5DFF85C4250
:10959000E068216808400CD5DFF8540200680568CF
:1095A000290003D000F017F80021A8474FF0004031
:1095B0000DE040000CD5DFF83C020068056829008A
:1095C00003D000F008F80121A8474FF08040A060C8
:1095D000BDE831404CE00021C0E90011F6E000BFD9
:1095E00038B5DFF81442216801290CBF0125002598
:1095F0004128B8BF002003DB5028B4BF012002205F
:10960000DFF8F81101EBC001D1E90023DFF8F01118
:10961000C1E90023DFF8EC1101EBC001D1E900231F
:10962000DFF8E411C1E9002329001CBF4AF6E85124
:109630002160002818BF022801D002D20120FEF7C5
:1096400048FD0DB10020206031BD7049096800EB74
:109650008000A1EBE00080F30800C0B270476C48C6
:109660004FF040410160416821F040414160704746
:10967000F0B56049624B0A68002053F8304044B1AD
:10968000156803EBC0041DB115792679B54200D2E7
:109690002246401C0628F0DB0A6011465D480A6835
:1096A0005AB10268120A1202026002680979114373
:1096B0000160416941F0804102E0416921F080414F
:1096C0004B4A514C41610021136854F8315045B167
:1096D0001E6804EBC1051EB12E791F79BE4200D26F
:1096E0002B46491C0629F0DB13601A6862B1026838
:1096F00022F47F4202600268197942EA0121016086
:10970000416941F0004102E0416921F000414161BD
:10971000F0BDF8B540490120087000F053F800F0A2
:109720004DF834493D48394B0860314908603C48A0
:109730000168406DC1F3074100F0FF00FF2912BF2F
:10974000FF281921902001EB810200EBD2021A6060
:10975000C0000522B0FBF2F04018324908606846AC
:1097600000F0C6FD9DF8010001281BD14120234CCB
:109770002D4D244FFFF769FF207125603920FFF739
:1097800064FF06465020FFF760FF3E73BD60207304
:10979000A5604820FFF759FF38753D6100F016F8C5
:1097A000FFF71EFFFFF75BFF0020FFF7E3FE1F49F7
:1097B00001200860FFF75CFF0020F2BD3021124855
:1097C000FCF728BF30210E48FCF724BF1848154984
:1097D000006809680006400D052290FBF2F0081AA7
:1097E00000F307007047000080E200E024300E40E4
:1097F000780700207407002008300E409C070020E6
:109800000C070020840700203C0700207C07002074
:109810002C300E401C300E403F1400206C070020FE
:10982000B081E00F80070020DF95000000E100E03C
:1098300020300E4030490A68100003D012680A60D8
:10984000FDF79FBF70472C48006800B1001D7047AE
:109850002DE9FC410D460746287800061446984637
:109860000FD5E019001DFDF770FF234E38B300211E
:10987000016000E00E4631680029FBD13060061D12
:1098800001E01E4806683A462946304606F044FB89
:10989000200014D00898F619022808D1E2B24146F7
:1098A000304602B0BDE8F041002302F008BB22467A
:1098B0004146304602B0BDE8F04106F02DBBBDE8A0
:1098C000F38180B5FFF74DFAA8B1011D0C4A0A607B
:1098D0000A2300224A608A60CA600A6100F13C02E1
:1098E00013704FF48073CB6200239370CB61BDE89B
:1098F0000240FFF776BA01BDFC06002028000020D8
:109900005198000050E8002F40E80013002BF9D1D7
:109910001046704780B500211548FFF7F3FFBDE8FA
:109920000240FFF731B913494FF08050086070478B
:109930000F4951E8002F024341E80023002BF8D1E2
:109940000D480068004780B502000B490DD10B4857
:1099500008606FF001000A49FFF7B4F84EF27C216D
:109960004FF0804008604EF2FC01086001BD00002D
:109970008808002004ED00E08C08002027990000F2
:1099800015990000B14942F60110086070472DE9B1
:10999000F84F044600F049F9AD49DFF8B8A200FBE2
:1099A0000410AD4CAD49D4F80080B0FBF1F000F1EB
:1099B000020BA069009000274FF0FF390025002618
:1099C00030015AF8001001F00301012910D1504470
:1099D0000125C168009807F0BCFBE16D06F10802A3
:1099E000D140C90748BFB94602D4484598BF81460F
:1099F000761C052EE4D308F44030B0F5003F11D1B9
:109A0000E06A421C08F44050B0F5805F07D1A06ABC
:109A100000F58070A0FB02864046314606E0110E3C
:109A2000100203E0A06A00F580700021A0FB098607
:109A300028468B4DD5F800A001FB096689490968C5
:109A400011F0706F04BFE16811F0060F64D10028B7
:109A500061D00BF1040000F013F9B1425CD828BFCB
:109A6000404559D24FEA182040EA066800F0DDF878
:109A70004246330AA0FB028600FB03661120FCF776
:109A800066FF0246002340463146B94607F090FC87
:109A9000C5F838907449626F4A60744A626702225E
:109AA000AA614FF480726266A36EA7662F687F1C5E
:109AB000EF630227AF63EF6B8F6004E0BF1C8F6022
:109AC0004FF00109EF632E68E76DFF0519D5626657
:109AD000A36600EB0A02A2EB0B02EA63ABEB000009
:109AE0000222AA61EA6942F00202EA612A68EB6B8B
:109AF000D21A82420DD30120087001275C49086008
:109B00000AE08F6807F1010E7645DCD1B9F1000F4C
:109B1000D4D0002001E001273846BDE8F28F52483A
:109B2000007800B970472DE9F04D52484A4CD0F802
:109B300000B0A0684A4D4C4940F4E400A060E869D8
:109B400020F00200E8612868801CE863E86B8968FF
:109B5000401A00F095F80646206810F4883F8A46BF
:109B600025D0A06AA76F00F58078304642460023D2
:109B700007F01EFC120A42EA0362D719304651462A
:109B80004246002307F014FC0646B7EB182F24BF0B
:109B9000761CA7EB18272761E06FE16A00F03EF81A
:109BA000606134480068216B00F038F8A061E06D16
:109BB000C00104D42868E96B081A0328F7D34FF0D2
:109BC000807060660220A86127492748214A4068C2
:109BD0006067A06820F4E400A06000200870002105
:109BE000A0690B01D558ED0713D5E66D01F1080505
:109BF000EE40F6070DD413445845DB6802D39B456D
:109C000007D201E09B4501D3984202D30123AB4028
:109C10002366491C0529E4DBBDE8F08D3018491C9A
:109C2000B0FBF1F201FB1200704710B51248016859
:109C30000124C90404D40068000A00F00F00844025
:109C40000E48FCF784FEB0FBF4F010BD5C600E40E3
:109C500020A10700745008400050084040420F0007
:109C600008200440044008400007002003000700CB
:109C700084000A43805008400020044080091200FC
:109C800038B504461120FCF762FEA0FB0445FFF73F
:109C9000CCFF024600232046294607F089FB090233
:109CA00041EA1061000234BD890001EB401000F16F
:109CB00084400260704710B5464A474C10602160EE
:109CC00000214648018007F0EFFBC00308D507F0EC
:109CD000E7FB2168080003D0BDE8104004200847D6
:109CE00010BD38B500F002FA044600F03FF8054612
:109CF000681E032803D2284600F042F800E0002541
:109D0000204600F0F7F9284632BD80B50022012137
:109D10003348FFF7C9FFBDE80240042030E00228C5
:109D200018BF03280BD12D490A18014412F8022C40
:109D3000521C022801F8022C01D1012213E07047C5
:109D4000022818BF03280DD124490A1812F8022C42
:109D5000130003D00844521E00F8022C087808B9FA
:109D6000002200E0704701211D489DE71B490A7849
:109D70000120002A01BF02204978002903207047F2
:109D800010B504461348016808001CBF20468847E8
:109D9000601E032814D8DFE800F002090D111148F5
:109DA000016821F00401016030BF09E00120FDF7E6
:109DB000EAFD05E00120FDF703FE01E0FDF739FEB5
:109DC00005480168080003D02046BDE81040084758
:109DD00010BD00006C05002070050020301400202C
:109DE00000300E4010ED00E099490A680AB90020E1
:109DF0007047D2680021101A00D400D10121084612
:109E0000704710B5924A12684FF0FF3109E0D368ED
:109E100014695268E3181B1A23F000438B4298BF61
:109E20001946002AF3D1084610BD10B504466069F2
:109E300020B1A168002958BFFDF7A3FC2046BDE86A
:109E40001040FDF79EBC82490020086070472DE954
:109E5000F84F7F4C25688046894692469B460026EF
:109E600004E06F682846FFF7E0FF3D46BDB1286873
:109E7000404502BFA86820F0004048450CD15FEA89
:109E80000B0003D068695146D84728B96868002E8E
:109E900014BF70602060E4E72E466D68E6E7BDE819
:109EA000F18F00230022D2E7F8B505001CBF286817
:109EB00000280E4617461C4608D127B1002E5CBF6D
:109EC0003846FDF75EFC4FF4C670F2BD1820FDF772
:109ED0003CFC78B100214161866047610560002249
:109EE00006995B4B0161594909686118C1601C689A
:109EF00025460AE027B1002E5CBF3846FDF741FC3D
:109F00004FF4C170F2BD2A466D6815B1EE68B142DA
:109F1000F9D212B94460186002E0516841605060A3
:109F20000020F2BD80B500230093FFF7BDFF02BD06
:109F300070B504460D4616460C20FDF706FC10B918
:109F40004FF4C17070BD456086602168016020607B
:109F5000002070BD2DE9F0410546002728680E4617
:109F60009046002801E0074620000ED042680168B4
:109F7000B24204BF826842450C46F4D1002F0CBFA8
:109F800029603960FDF7FDFBEEE7BDE8F08138B5EB
:109F900004462F492068096807E00A68A24203D1F5
:109FA0008A6802F000428A6049680029F5D120B130
:109FB0000568FDF7E6FB2846F9E7206031BD2DE98D
:109FC000F04104000D4690460DD0276800E037466A
:109FD0004FB13E68B8687F6843462A462146B84775
:109FE0000100F4D000E00020BDE8F0812DE9F0414F
:109FF000164C174D20601AE070682860B068400069
:10A000001CBF306800280FD007686FB1B2685000DD
:10A010000AD0D7F80080B868736931687F68B8479C
:10A0200010B95FEA0807F1D13046FFF7FEFE266857
:10A030003046FFF7D9FE18B12E68002EDCD1F6E7C6
:10A040003046BDE8F041DCE600000000EC070020EF
:10A05000F007002070B50546FEF727F940B915F165
:10A06000010F1E4C0DD01E48007850B9022D01D2B0
:10A07000002070BD20684019E064E06940F00400F1
:10A08000E061FFF773FE0025022812DB1548164A2F
:10A0900001680068C1F3031100F00F0032F81110DD
:10A0A00032F810004018B43080B2FFF770FC0500A1
:10A0B00002D10220FFF733FE2668FFF712FE206868
:10A0C000861BE06920F00400E061FFF728FD15B968
:10A0D0000220FFF735FE304670BD00BF0820044067
:10A0E0003E14002034400E4078590000EFF31080F9
:10A0F00072B6704700B962B67047032880B5214A2E
:10A10000002111602049086000200968887307F069
:10A1100009FA07F00DFA07F0E5FA07F005FB01F080
:10A1200098FD08F0F2F808F08BFA08F037FF00F01D
:10A1300097F9BDE8014007F0E6BD1CB504460622CC
:10A1400012496846FCF78AF9204669460622FCF760
:10A1500075F913BD10B5044603E0FFF747FF07F09C
:10A16000D0FD07F04AFD00282046F6D1BDE810409A
:10A17000FFF73CBF002818BF08F088BD4FF4C0703F
:10A1800070470000980800209C080020B00B0020B9
:10A1900080B507F06BFA20B1C08DBDE8024008F031
:10A1A0001BB84FF4C07002BD80B50146012008F015
:10A1B00052F8002002BD0328002200F01BB903283A
:10A1C00070B5054605F10F00C408AFF30080E40048
:10A1D000A54232D2082C04D2082402E0083000F054
:10A1E00047F82248026811000CD1011D0A6802B329
:10A1F0001368A34238BF111DF8D310E01D68A542B3
:10A200000DD2191D0B68002BF8D11268011D00E05A
:10A21000191D0B6893420CD01D68A542F8D361B19B
:10A220000D682A68A2F10803A3420AD26A680A608C
:10A230000FE009F027F80028D0D1AFF3008000200C
:10A2400070BD2B190B60121B6E685E600B681A6084
:10A250002C60096800291DBF4A68002A091D0021D9
:10A260000160AFF3008005F1080070BD1C140020F0
:10A2700000B9704738B5A0F108042068082833D326
:10A2800010F0070F30D1AFF300801848416809B1D2
:10A290008C4203D26160446017E019464B680BB1F1
:10A2A000A342FAD30B68CD18AC421BD3A54204D10C
:10A2B0002268D2180A600C4607E04A681AB123687F
:10A2C00023449A420ED362604C60616851B12268A7
:10A2D000A3188B4206D10023036008688018206011
:10A2E00048686060AFF3008031BD00001C1400209E
:10A2F0000B494A680B68920002F03C02C3F38113D9
:10A300001A4382700A6802F03F0242708A68C96884
:10A3100002F0F002C1F30311114301707047000015
:10A32000E0FF0FE080B508F0DCFF002002BD09F07F
:10A330003DB892B208F0D8BF02B504226946FFF7D3
:10A34000F8FF02BD02480349006801EA8020704717
:10A35000F881E00F00FCFF030300002013F0030F5F
:10A3600009D0521E22BF13F8010B11F801CBB0EB3C
:10A370000C00F3D07047121F22BF53F8040B51F8A2
:10A3800004CB6045F7D0121D0AD200BA9CFA8CFCAF
:10A39000B0EB0C0038BF6FF0000088BF01207047A1
:10A3A000521E22BF13F8010B11F801CBB0EB0C00C9
:10A3B000F6D0521C08BF10467047FEE710B50A4B96
:10A3C00040F201141C6098600120586002E012F80D
:10A3D000010B98610846411E0028F8D1D8694FF05A
:10A3E000FF31484010BD00BF00C0014062F30F22A2
:10A3F00062F31F42401810F0030308D0C91A1FD39C
:10A40000DB0748BF00F8012D28BF20F8022D1300FC
:10A4100030B414461546103928BF20E93C00FAD85C
:10A42000490728BF20E90C0048BF40F8042D8900E7
:10A4300028BF20F8022D48BF00F8012D30BC70471E
:10A44000C91818BF00F8012DCB0728BF00F8012D4F
:10A450007047EFF31080C00701D562B672B670473F
:10A460008549262008807047A0F11701682902D38A
:10A470004FF4C0707047804908800020704738B59D
:10A480007E4D7F4C2878800706D401F044F8206088
:10A49000286840F002002860206832BD10B50446EC
:10A4A0007648016821F00201016042F6052001F0C2
:10A4B0009AFB01001CBF002002F0B6FC2046BDE85C
:10A4C000104001F024B838B504465420FDF74CF98B
:10A4D000050001D1002032BD204607F00BF92565AB
:10A4E0002C600020616E41F48031616628626863EF
:10A4F00028652A461720A88120460FF2C901FFF7D8
:10A5000017FD604800684168002205F11400FFF75C
:10A510000FFD0220E861284632BD38B504001CBF9B
:10A52000256D002D28D0002020652A460FF29501C8
:10A530002046FFF70FFD281D01F0FAFC05F1080089
:10A5400001F0F6FC05F11400FFF721FD05F1100004
:10A55000FFF71DFD286B08B1FDF713F9286D18B141
:10A5600005F1500001F0E4FC2846FDF70AF9204609
:10A57000BDE8324007F014B831BD80B5002200922A
:10A580004FF470230068FFF78FFC01BD0068FFF7F0
:10A5900088BC10B50446E069012811D00120E061B3
:10A5A000FDF7D3F860B1216891F82C1001700246D4
:10A5B00004F11400BDE810404FF4C161FFF7B2BCD4
:10A5C00010BD000010B50446521E08461CD040F2D3
:10A5D0000121521A0AD0521E16D040F20641521AD8
:10A5E000012A9CBF2046FFF7D4FF0FE022480188D4
:10A5F0001829A4BF204608F090FF204600F0FFFF76
:10A60000204602F0C5FB01E0FFF787FF002010BDE8
:10A610000846904288BF10461728B8BF17207047D9
:10A6200070B5154E0D463188044608F080FF32881B
:10A6300029462046FFF7ECFFA08170BD38B50446DF
:10A640000D480A4601882046FFF7E2FF0546A5812E
:10A650000420FDF77AF868B1216891F82C10017098
:10A660004580024604F11400BDE8384040F2016123
:10A67000FFF758BC31BD0000580200207C0B0020C1
:10A68000480000209808002080B506F0EFFF00B1D8
:10A69000006D02BD80B5002100B10168084607F0D9
:10A6A0001BF8010003D0086D0028F7D002BD002080
:10A6B00002BDEFF31080C00701D562B672B67047D5
:10A6C000002105E0827A5118427A0068891AC9B2DD
:10A6D0000028F7D108467047C169012902D140F22C
:10A6E00003107047006A08B14FF481707047F8B5E5
:10A6F000170004460D461E460AD1206A072803D0DB
:10A70000082808BF092700E00B27300018BF0D27D5
:10A710000698FFF7D5FF618D0A0009D0A28D8B1A2C
:10A72000834205DA401A1118C9B206A801F04CFD9F
:10A730000C20FDF70AF8020003D106A801F0F8FB8F
:10A74000F1BD206890F82C00107055801771D680EC
:10A7500040F205610698906004F11400FFF7E2FBF7
:10A76000F1BD7CB504460D4616460C20FCF7EDFF06
:10A7700018B901A801F0DCFB73BD216891F82C1019
:10A7800001704580868002460199816004F11400C1
:10A7900040F20661FFF7C6FB73BD016240F209613A
:10A7A000FFF7EBBE38B50D46044640F20961FFF7EE
:10A7B000EDFE002020620820FCF7C7FF68B1216889
:10A7C00091F82C1001704560024604F11400BDE8B8
:10A7D000384040F20761FFF7A5BB31BD09B1030C5A
:10A7E0000B8002B11080704710B50446206B18B181
:10A7F000FCF7C7FF0020206310BDF8B504460D46E6
:10A8000016461F46FFF7F0FF2846FCF79EFF206321
:10A8100010B94FF4C170F2BD1EB13A463146FBF794
:10A820000DFEA7850020F2BD10B504460846FFF7CF
:10A8300047FF628DA18D130002D0521A90420BDAAD
:10A84000A289531E002902BF216A0829131F9BB247
:10A85000984201D1012010BD002010BDF2B51500B5
:10A8600082B004461E4622D10846FFF729FF0700A2
:10A870001DD0206AC01F012802D9C01F04D00BE0E0
:10A88000029800F017FD05E0029BA28D218D204665
:10A89000FFF767FF00200290A08D3A18A28536B11D
:10A8A000218D92B2204608F0ABFE050004D02A4666
:10A8B0000021204600F089FC00F05EFDF7BD2DE987
:10A8C000F042044682B0A0891F46C01EB8420D4621
:10A8D000164605DB204602B0BDE8F04208F0DFBEB8
:10A8E0002585F9B22046FFF788FF5FEA000910D1FD
:10A8F000A089411F8F42A8BF471FBFB200973346B0
:10A90000002200F009F85FEA00091CBF2046FFF7AB
:10A910006BFF4846BDE8F6822946204608F0E6BEB1
:10A9200038B50D460446002108F02EFF256331BDE1
:10A93000F8B5044682B015461846FFF7C1FE074633
:10A9400000F01AFD089EB6B9ED19A08DA9B281429A
:10A9500015D2A189ADB22A46831A4E1FB342B4BFA5
:10A96000401B481F80B20090206B218D8318FFF799
:10A97000D4FF06000FD000F0E1F9314608E000F006
:10A98000DDF90121204608F0FFFE060003D0014654
:10A990002046FFF7C5FFF7BD30B583B00446FFF78B
:10A9A0009BFE050012D14FF6FF72DFF8EC08E2843F
:10A9B00001AB00F0C2F8012102200090204608F00F
:10A9C0005EFE050002D1012100F0A2FA28463EBD3C
:10A9D0002DE9F843089C0546884691461E4604F139
:10A9E0001C00FCF7B2FE070016D0286890F82C0077
:10A9F0003870BC6149EA084078602246314607F168
:10AA00000800FBF71BFD3A4605F11400BDE8F843CA
:10AA100040F20261FFF786BABDE8F1832DE9F24FFB
:10AA2000804682B01E469246504609F078F90746A5
:10AA300000F0DDF8AAF1040B4FF6FF75002456BBB9
:10AA400000F0D5F8814612E00299E3B25FFA8AF28B
:10AA5000384601F034FA7D885FFA8BF000903B1D98
:10AA600039882A464046FFF7B3FF5444A4B24C4508
:10AA7000EADBB8F82620954212D2DFF8200800F071
:10AA80005CF8691C0220009001AB89B2404608F0D6
:10AA9000F6FD060008D040F20A40864208BF0026B4
:10AAA00031464046FFF77EFE00F066FC38469AE0ED
:10AAB000F0B583B000F03FFA07001DD14FF6FF70EC
:10AAC000E08433462A4631462046FFF796FE0700CB
:10AAD00012D1A08D01904FF42053206B00900121E2
:10AAE000E28C204608F048FD070002D000F026F96D
:10AAF00002E0022100F00CFA3846FEBD7CB500F001
:10AB000057F9060017D104F1260204F1280128465E
:10AB1000FFF764FEDFF8880700F00FF801AB0220B2
:10AB20000090E28C218D204608F03FFD060002D106
:10AB3000032100F0EDF9304676BD0088ADF8040041
:10AB400070472DE9F24F04469146484682B0984638
:10AB5000A0F1060B002509F0E2F8B8F1000F4FF65E
:10AB6000FF77064633D100F042F8824608E00090B5
:10AB7000B2887188B31D2046FFF72AFF4D44ADB25D
:10AB8000554517DA0299EBB25FFA89F2304601F0C7
:10AB900096F95FFA8BF037880028E8D1278570880E
:10ABA0006085B088618DA08500F093F95FEA0008A8
:10ABB0000DD115E0E28C97420FD2DFF8E806FFF7DF
:10ABC000BCFF791C00F0B3F85FEA000808D040F23F
:10ABD0000A40804508BF4FF00008414600F01BFACC
:10ABE00000F0CAFB304609F0A3F8BDE8F78F0298E1
:10ABF00066E51CB50446084604F1260201A9FFF7E4
:10AC0000EDFDDFF8A4060088BDF80410ADF80600DD
:10AC10000DF10603022000902046E28C08F0C5FCEE
:10AC200016BD70B500F0C4F8060008D129462046CC
:10AC3000FFF7DFFF060002D1042100F069F930467A
:10AC400070BD2DE9F843089C05460E46914698468E
:10AC500004F11C00FCF779FD070016D0286890F875
:10AC60002C0038707E8087F80490BC6122464146F3
:10AC700007F10800FBF7E2FB3A4605F11400BDE8D6
:10AC8000F84340F20361FFF74DB9BDE8F1832DE9C8
:10AC9000F24F04469346584682B09846461F002716
:10ACA00009F03DF8B8F1000F4FF6FF7A05462FD1B5
:10ACB000FFF79DFF81461BE00299FBB25FFA8BF222
:10ACC000284601F0FCF8B5F800A0206B28B1F6B2D8
:10ACD0003246691DFFF740FB40B9F0B20090AA78F8
:10ACE000B5F803106B1D2046FFF7ABFF5F44BFB202
:10ACF0004F45E1DBE28C924510D2DFF8B005FFF75B
:10AD00001CFF0AF1010100F012F85FEA00080AD006
:10AD100040F20A40804508BF4FF0000800F00EF8EE
:10AD2000414600F078F900F027FB28465BE7022057
:10AD3000009001AB89B2204608F037BC204653E5AD
:10AD40002DE9F04100F00CF95FEA000815D13B460F
:10AD5000324639462046FFF750FD5FEA00080CD125
:10AD600029462046FFF745FF5FEA000802D0FFF7BB
:10AD7000E5FF02E0052100F0CBF8A6E070B500F099
:10AD800017F8060012D14FF6FF70854204D100215A
:10AD900000F041F9002070BDE0840246691C00F01B
:10ADA00035F9060002D1062100F0B2F8304670BD38
:10ADB00004460D4690E42DE9F04104461F460D4639
:10ADC000904607F11800FCF7C0FC060013D020687D
:10ADD00090F82C003070758077613A464146301DFE
:10ADE000FBF72CFB324604F11400BDE8F04140F2C1
:10ADF0000461FFF797B8BDE8F0812DE9F44F012910
:10AE00000CBF02261026B71C8046FFB21D463846EE
:10AE100008F085FF4FF6FF7B002481463DBB00987C
:10AE2000FFF74EFC824614E00099E3B23A464846EA
:10AE300001F045F899F80300B9F800B028281BD0B4
:10AE4000334609F1020259464046FFF7B4FFE419C0
:10AE5000A4B25445E8DBB8F8262093450CD20BF198
:10AE6000010189B2404608F079FB050008D040F2A4
:10AE70000A40854208BF002529464046FFF792FC5C
:10AE800000F088FA484608F053FFBDE8F18F2DE93D
:10AE9000F04100F065F85FEA000816D138000CBFF9
:10AEA0000020B819608525853000A68502D100F004
:10AEB0000FF804E0218D3246204608F0A1FB5FEA3E
:10AEC000000802D1072100F023F84046BDE8F081D8
:10AED0002946204608F07DBB2DE9FC4100F040F8F2
:10AEE0005FEA000813D104F1260201A92846FFF702
:10AEF00075FC0097E28CBDF804103346204608F03C
:10AF000054FB5FEA000802D1082100F001F84FE08D
:10AF1000204642E4F8B500F00EF8070009D1F2B27D
:10AF20002946204608F08BFB070002D10921FFF7D4
:10AF3000EFFF3846F2BD04460D461646FFF7CCBB80
:10AF40002DE9F04100F00CF85FEA000807D100F0AD
:10AF5000DDF85FEA000802D10A21FFF7D9FFB4E764
:10AF600004460D4616461F46FFF7B6BBF8B5FFF779
:10AF7000F7FF40B93B4632462946204601B0BDE8BE
:10AF8000F04008F0A6BBF2BD2DE9F04182B0FFF71A
:10AF9000E7FF5FEA00080BD1089800903B46324675
:10AFA000FFF7BAFC5FEA000802D10C21FFF7B0FFFF
:10AFB0004046BDE8F68170B5FFF7FAFE060008D1FD
:10AFC0002946204608F0E0FB060002D10D21FFF7DC
:10AFD0009FFF304670BDF8B5FFF7ADFF070013D1F6
:10AFE0004FF6FF70854205D140F20A4100F013F898
:10AFF0000020F2BD0246691C266300F007F8070036
:10B0000002D11021FFF784FF3846F2BD89B22046F5
:10B0100008F0A4BA29462046FFF7C4BB2DE9F6473D
:10B02000044601299A460CBF4FF004094FF012095B
:10B030004846002708F073FE4FF6FF78BAF1000F7C
:10B040004546064635D10198FFF73AFB824603E0B4
:10B0500028282CD04F44BFB257451DDA0199FBB2C6
:10B060004A46304600F02BFFF078B17841EA0021E3
:10B0700042F6021235889142EAD10020ADF8000074
:10B080000223206B8DF800006A4629462046FFF710
:10B0900016FC002020630FE0E18C8D4207D2691C72
:10B0A0004246FFF7B3FF5FEA000A02D104E040F234
:10B0B0000A4A5146FFF7AFFF01A800F039FF3046BA
:10B0C00008F036FEBDE8F38770B5FFF771FE0600A5
:10B0D0000AD10020A08560852585FFF7F9FE0600CE
:10B0E00002D10E21FFF714FF304670BD2DE9F0416B
:10B0F000FFF736FF5FEA000807D100F007F85FEAC4
:10B10000000802D10F21FFF703FFDEE63B4632467F
:10B1100029462046FFF7D3BB04B5026A062A02D0AF
:10B12000102A04D007E0009AFFF767FE01BD009ADD
:10B13000FFF774FF01BD2AE12DE9F241044685B015
:10B14000206A022815463AD1084603904FF6FF764A
:10B1500000274DBBFFF7B4FA804612E00399FBB21B
:10B16000042202A800F0ABFEA08DBDF80A60BDF875
:10B170000810C0B200903246236B2046FFF728FC2F
:10B180003F1DB8B24045E9DBE28C964211D2A08D5A
:10B190000190711C206B00904FF4205389B220461F
:10B1A00008F0EAF9050008D040F20A40854208BFDD
:10B1B0000025FFF7C3FDFFF72DFF03A800E005A85A
:10B1C00000F0B6FE06B0BDE8F08172B5150083B0A0
:10B1D000044609D1FFF728FB30B10399012300226F
:10B1E0002046FFF73BFB7FBD206A032806D00728D7
:10B1F00018BF082832D00E2839D049E003980190B2
:10B2000040F21F2638B3EDB9102000900198417A22
:10B21000A28D084400F11003618D2046FFF7D8FB92
:10B22000E28C208D904212D221490988ADF8081095
:10B2300002AB02210091411C89B2204608F0B5F909
:10B24000050006D040F20A40854200D13546FFF79E
:10B25000E1FE01A81DE0002DF4D1F7E7039801906D
:10B260001DB910B100F026F80FE001A80BE003981B
:10B2700000903DB930B10346218D00222046FFF7F2
:10B2800070FA02E0684600F053FEFFF7C3FE7FBD90
:10B2900003A800F04DFE7FBD126600001A66000094
:10B2A00086770000068C0000FAA00000B6A100001E
:10B2B000C27700000090A38D218D00222046FFF769
:10B2C00016BA32B504461546206AC01F012801D9B6
:10B2D000C01F09D12046FFF7A7FA034600992A4666
:10B2E0002046FFF7BBFA31BD00F054F831BD32B54E
:10B2F000044682B0206A092815460DD101913DB956
:10B30000009100230F2200212046FFF7F0F902E010
:10B3100001A800F00DFE5FE02BE032B5044682B0DC
:10B32000206A03281D4606D0042818BF052806D029
:10B33000082808D01DE02046FFF703FC37BD204653
:10B34000FFF7A5FC37BD009105B143E0002031B106
:10B350000846417A009A0844891C008A5172208567
:10B36000002200206085A08520460099FFF72DFF70
:10B3700037BD00F001F837BD02A800F0D9BD02B515
:10B38000016A012903D10099FFF748FB01BD00F0D4
:10B3900001F801BD684600F0CBBD026A0A2A1CBF55
:10B3A0000F2A102A01D1FFF7FDB9704738B50446BE
:10B3B00082B0206A069D0A2803D00C2807D00F28E7
:10B3C00007D1029B00952046FFF7B2FA37BD0093E4
:10B3D00000E0CEE7FFF7DEFF29462046FFF7E2F95F
:10B3E00037BD026A0A2A03D00D2A07D00F2A07D1D7
:10B3F000026B12B1114600220263CEE7FFF7D2B909
:10B40000704780B5009200231B2204E080B5818440
:10B41000009200231D22FFF76AF901BD80B5C169C2
:10B42000012902D140F2031002BD818C11B940F212
:10B43000811002BD0021818408F0DBF9002002BDEB
:10B440000069022818BF102801D101207047002090
:10B45000704770B50E4624490C68022810D1307828
:10B46000717840EA0120002500E06D1CA1688D4242
:10B470001BDAE16831F815108142F6D1A8B270BD2F
:10B48000102812D1002500E06D1C206985420CDADD
:10B4900060691022314600EB0510FEF75DFF0028C1
:10B4A000F2D145F4004080B270BD4FF6FF7070BD20
:10B4B000034608460C4909681A040AD50A69C3F309
:10B4C0000E0393420EDA4969102201EB0311FAF7D9
:10B4D000B5BF8A68934205DAC96831F81330037042
:10B4E000190A417070470000D4080020DFF8D01618
:10B4F00009680A680C23584310440C380088020479
:10B5000001D500207047C96831F810007047DFF896
:10B51000B0160860704738B5DFF8A4462068021DF1
:10B5200004214FF0FF30FEF749FF002507E00968CE
:10B530000C226A430A440221FEF740FF6D1C216879
:10B540004A689542F3DB002506E0C96801EB450235
:10B550000221FEF733FF6D1C21688A689542F4DBF7
:10B56000002505E049694A191021FEF727FF6D1CE7
:10B5700021680A699542F5DB32BD010007D0DFF88A
:10B58000401609684968814201DB012070470020AC
:10B590007047F8B5DFF828660446306800680C2567
:10B5A00000F018F87879012802D1B8680078F2BD67
:10B5B000641EA0B268B130680068A4B200F00AF856
:10B5C0002046FFF793FF42F603018842F0D1B868A6
:10B5D0004078F2BD05FB04F10844A0F10C07704768
:10B5E000DFF8DC15096809680C225043084410F89C
:10B5F000070C072801D1012070470020704710B5C3
:10B60000044600F098F80DD0102304F140020B21FD
:10B6100008F0BAFC00F089F8BDE8104004230C21C2
:10B6200008F0B2BC10BD10B50446641CA0B2FFF710
:10B63000A4FFC0B1A0B2FFF759FF42F60211884241
:10B640000AD1DFF87C0500680068A4B20C216143D0
:10B65000084410F8020C10BDA0B2FFF747FF42F6F5
:10B6600003018842E1D14FF0FF3010BD38B100290D
:10B6700005D44A1001EB92729210102A01DB0020CF
:10B6800070471044A1EB820190F840004900C84087
:10B6900000F00300704770B504000D4644D0002D43
:10B6A00042D4DFF81C050068806985423CDA6810E6
:10B6B00005EB907081100846102835DA2318A5EBA9
:10B6C0008101490093F8403003268E40B343261889
:10B6D000204486F8403002F0030606FA01F11943CF
:10B6E00080F840106AB142F6052000F07CFAFFF7BE
:10B6F0009AFF80B2A84204D1FEF7C1FEE0630125A3
:10B7000000E0002500F017F80ED0102304F14002ED
:10B710000B2108F0F5FB3DB100F007F8BDE87040E3
:10B7200004230C2108F0ECBB70BD206890F9540094
:10B7300004F13C027047206890F9540010F1010FA9
:10B74000704770B50D4604462E46761CB0B2FFF722
:10B7500014FFD8B1B0B2FFF7C9FE42F60211884219
:10B760000DD1DFF85C0400680068B6B20C217143AB
:10B77000084410F8070C072808D1032070BDB0B2A8
:10B78000FFF7B4FE42F603018842DED12846FFF7F8
:10B790004AFF10F1010F01D1002070BD0146204683
:10B7A000BDE8704062E70000DFF81414096809681A
:10B7B0000C22504308440C38417904290DD8DFE8A5
:10B7C00001F00305060A0A00806802E007E08068CD
:10B7D00040680078704702207047002070478068FA
:10B7E0008078704770B504460E4615463046FFF720
:10B7F000C4FE08B9012070BD00F0F8F87143084498
:10B800000C38E90724D54188CA0701D4022070BD4D
:10B81000CA0607D5226812F8453FDB0741D500F07C
:10B8200058F84BD38A0605D500F057F82FD100F011
:10B8300050F843D349060BD500F056F831D592F9AC
:10B840000F1011F1010F33D0517D0279914235D3A0
:10B85000A90702D58178890704D5690704D58178BD
:10B86000490701D4032070BD06210D4228D041882C
:10B87000CA0507D5226812F8453FDB0711D500F04D
:10B8800028F81BD38A0507D500F027F801D005203A
:10B8900070BD00F01EF811D3490511D500F024F851
:10B8A00001D40F2070BD92F90F1011F1010F01D1D9
:10B8B000082070BD517D0279914201D20C2070BDEB
:10B8C000290504D54088000501D4062070BD00205C
:10B8D00070BD527D03799A427047226812F8453F45
:10B8E00003F00303032B7047216801F1450211782F
:10B8F000C90770472DE9F04104460229B8BF00206E
:10B900003BDBAF4DA1F102082968496A03204F00D3
:10B91000B845BCBF28F00107022067B1791C21702F
:10B9200060703A462868016AA01CFAF787FDE019A2
:10B93000841CA8EB07082968C96A07200E01B8F122
:10B94000030FACBFA8F102010021B14205DAC81013
:10B9500001EB10700011060106200EB938460AE00E
:10B96000711C2170607032462868816AA01CFAF749
:10B9700065FDB819801C07B1801CBDE8F08100008E
:10B980002DE9F0411C461646002780460D462760EB
:10B9900037802846FFF7F1FD10B90120206022E032
:10B9A00000F024F8694308440C384179042915D87B
:10B9B000DFE801F00305080C1300806804E08068EC
:10B9C00047680BE080684068471C07E0817A7D4F3C
:10B9D0004046FFF74BFE388000E078A71FB12846AD
:10B9E000FFF7E2FE30803846BDE8F0817448006819
:10B9F00000680C2170472DE9FC4104460D461646AF
:10BA00002846FFF7BAFD18B900F098F8012093E036
:10BA1000DFF8AC81D8F8000000680C2169430844C5
:10BA2000A0F10C07787920B1042806D0072808D0A7
:10BA30000BE000F083F803207EE000F07FF80620A2
:10BA40007AE000F07BF8802076E02846FFF7ACFE35
:10BA5000B04203DA00F072F807206DE07979019ABC
:10BA6000022904BFB86880786AB11346002208E052
:10BA700093F80AE0724493F809E01B68A2EB0E0207
:10BA8000D2B2002BF4D19319984203DA00F056F8A1
:10BA90000D2051E0012904D02CD3032914D006D362
:10BAA00028E0B868406801990023304409E0B9688B
:10BAB0004968901908700023B868406801993044BB
:10BAC000401C00F0FCF915E00198417A827A0844A4
:10BAD000521A103072B1032A0CD20178022A24BF04
:10BAE000407841EA0021387A00EA0102B97A20461A
:10BAF000FFF7D1FD14B900F021F81CE07879032894
:10BB000011D17D7A00F01AF8B97A2046FFF7AEFD20
:10BB10000346D8F80000C06930F81510012220460D
:10BB200000F07DFC07E0019800903346626B2946E7
:10BB3000204600F053FC0020BDE8F68101A800F08B
:10BB4000F7B930B51E4B1B685C688C4202DA21469F
:10BB500000E0401C8CB285B2AC4209D31C6880B2B4
:10BB60000C2545432C4434F80C4C9442F1D130BDA3
:10BB7000002030BD70B5124B1B68401C0C2600E045
:10BB8000401C84B28C4216D25D68A54280B212DBA2
:10BB90001D6874432C4434F80C4C2AB1022A01D09D
:10BBA00002D3EDE7022C03D0002C18BF012CE7D103
:10BBB000401E80B270BD4FF6FF7070BD00000000E7
:10BBC000D40800203214002010B50446FFF7D5FC3D
:10BBD00010B94FF6FF7010BDFFF708FF614308442E
:10BBE00030F80C0C10BD80B58DF800006946000AD5
:10BBF0008DF801000220FFF72CFC024604210120F1
:10BC0000FFF79FFF02BDF8B5044642F60520FFF797
:10BC1000EAFFFFF708FD054629462046FFF726FD07
:10BC2000024604F140000021002300260027CAC07C
:10BC300029462046BDE8F8402DE5EFF3108000F0DE
:10BC400001007047427A8A184272827A891881729A
:10BC5000704780B50120FBF746FDDFF81817801FFD
:10BC6000086001BDF8B5044600200D4600900FE0C5
:10BC7000707AFFB230443A46214600F0F4F9B07AC7
:10BC80003818B0723146684600F026FA3C44ED1B85
:10BC9000E8B288B1EDB22F463C2FA8BF3C2000F09F
:10BCA00065F8060000D1A3E0B07AC0F14501B942C1
:10BCB000DEDAC0F14507DBE70098F2BD2DE9F0417F
:10BCC0000446FEF713FA8046DFF8A806DFF8A85608
:10BCD0000068DFF8A866012C23D13168814225DA9B
:10BCE0000120FBF7E5FC07464046FEF703FA67B381
:10BCF00010213846FEF760FAB86840F00800B860D6
:10BD00000020B872787238607C60B86840084000E3
:10BD1000B8600020012CF8600DD13068401C306004
:10BD200013E0002CDCD129688142D9DB4046FEF7C4
:10BD3000E1F900200AE01CB92868401C286004E0F2
:10BD4000DFF83C060168491C01603846BDE8F08117
:10BD50004521B3E710B545210220FFF7AFFF0400EE
:10BD60001CBF0921FFF76EFF204610BD10B53D280E
:10BD700001DB002010BD00F109010220FFF79EFF4A
:10BD800004001CBF0921FFF75DFF204610BDF8B578
:10BD9000044600200D460090002620E0607A78726C
:10BDA000A07AB872A068B968400860F34101B96030
:10BDB000A068B968800860F38201B960607AA17AEE
:10BDC0000A1A204400F11001787A384400F04BF947
:10BDD000009800B9009706B1376024683E462CB140
:10BDE0002846FFF7B5FF0700D8D101E00098F2BD63
:10BDF000684600F09DF80020F2BD38B5040021D05F
:10BE0000FEF774F90546A068616820F00800012972
:10BE1000A06008BFDFF8641505D000290CBFDFF86B
:10BE20005815DFF85C150A68521E0A60C0072146E3
:10BE30004CBF03200120FBF74CFC2846BDE83240F4
:10BE4000FEF758B931BD30B5DFF83015DFF82835C9
:10BE500045680A681C68012D0AD1C56845B10025EE
:10BE600004E04560C560521E0068641C0028F8D1DB
:10BE70001C600A6030BD10B508E0427A837AC9B20E
:10BE80009C1A8C4205DAC91A006851180028F4D1AE
:10BE900010BD10440844103010BD38B50446154696
:10BEA000A07AC0F14502954288BF154620442A4633
:10BEB00000F0D9F8A07A2818A072284632BD2DE9E2
:10BEC000F0425FEA000918BF00290BD00C46607AE7
:10BED000A17ADBB20F1A9F4206DA591A2468431876
:10BEE000002CF4D1002021E0A67A2118301A194440
:10BEF000C51A1031EDB24E4609EB020705E0607A33
:10BF0000A27A2118151A1031EDB2BE420CD2701966
:10BF100087423CBFBD1BEDB22A463046FAF78EFA87
:10BF200024687619002CEAD1A6EB0900BDE8F0825E
:10BF300038B5044603E00568FFF75FFF2560206819
:10BF40000028F8D131BD00B9704710B5016821B99A
:10BF500000220260084610BD026003681A68002AC9
:10BF6000F6D09468C4F34004002CF5D000241C6083
:10BF7000EFE738B50446607A884202D3401A60720F
:10BF800013E0A27AC2F14503C3188B420FDB121AE9
:10BF90000D1A2318581903F11001103008F01CF87D
:10BFA00000206072A07A2818A072012032BD002003
:10BFB00032BD38B504460D46FFF7DBFF08B1204619
:10BFC00032BDFFF7C5FE28B1046045218172C5F17D
:10BFD0004501417232BDF8B504460D46607AA17A3A
:10BFE0000A1A081A561B8542B6B204DA0020FFF777
:10BFF000AFFE070001D10020F2BD607A2044284442
:10C0000000F11001787A384400F02CF8B87A301832
:10C01000B872A07A801BA072206838602760012067
:10C02000F2BD38B504000D4618BF002D07D0687A60
:10C03000A97AA37A0A1AC3F14501914201DA0020D4
:10C0400032BD284400F11001E01800F00CF8A07A8D
:10C05000A97A0818697A401AA0722846FFF7CDFE1F
:10C06000012032BD32461030FAF7E8B9F8B504467F
:10C070000F4626680020354605E0B07A717A381AF6
:10C080000F1830463668F9B269B166B1B07A717A84
:10C09000FFB2401A8742F0DA39463046FFF79BFF7D
:10C0A0000028EAD1F2BD08B10021016026602846CF
:10C0B000F2BD016821B10A6802600020086001E059
:10C0C0000022026008467047016819B10A680260E0
:10C0D000084692E601607047026812B90160704735
:10C0E000024610680028FBD1116070472DE9F84323
:10C0F0000400884691461CBFB8F1000F5FEA0900B2
:10C1000001D1002021E0274600E0074638680028DA
:10C11000FBD13D464E460DE0324641462846FFF7EC
:10C12000BCFEC0B2361ABD421CBF3D602F46F6B2FF
:10C130008044002536B11DB96068FFF709FE054649
:10C14000002DE9D1A9EB0600C0B2BDE8F28338B5F5
:10C1500005680C4615B9046031BD054628680028FD
:10C16000FBD1206818B1204600F054F803E02846BF
:10C17000FFF757FF00B92C6031BD026802B10A60B9
:10C18000016070470A0001D170471A461368002BFE
:10C19000FBD1036813600160704738B504460D4653
:10C1A00004E06D1A01682160FFF727FEE8B250B184
:10C1B000206840B1427A817A891A89B2EDB28D4203
:10C1C000EFDAA918417231BD70B504460D462068FA
:10C1D00010B970BD00203060E8B2D0B120680028EE
:10C1E00017D0002601E00646084601680029FAD16A
:10C1F000417A827AEDB2531A9D4202DA511B817262
:10C2000070BDAA1A8D18FFF7F8FD002EE2D10020AC
:10C21000206070BD70B5044643E0A17A607AC1F138
:10C2200045021518ADB2002D3AD002000DD00A1A01
:10C23000204400F1100104F1100007F0CDFEA07AB7
:10C24000617A401AA07200206072206840B3816851
:10C25000C1F3400121BB417A827AA37A0844521A81
:10C2600000F11001607A92B22E4695422044C8BF78
:10C2700016461844FFF7F6FEA07A3018A072AD1BE0
:10C280002068417A71184172ADB22068817A427A91
:10C29000891A03D101682160FFF7AFFD002DD4D1C9
:10C2A0002468002CB9D170BD70472DE9F94D82B0DA
:10C2B000002402980094002888464DD006460027A6
:10C2C000A246002526E0A8EB0A0B5FFA8BFB57B9C4
:10C2D000029840684146FFF7F1FC070036D0394626
:10C2E0006846FFF7F9FE707A3044401900F11001FA
:10C2F000787A381850445A46FFF7B5FEB87ADA44CF
:10C3000058445FFA8AFAB8725D44C245EDB204BF80
:10C310000027A246707AB17A0A1A95420FDA521BA8
:10C3200013464245C8BF4346A8EB0A0C6345CADA28
:10C330004245AEBFC346081AA0EB050BC5E73668F9
:10C34000002EBED1009C0020009004E0009810B1A7
:10C350006846FFF7EDFD204604B0BDE8F08D0748C4
:10C3600005490068096840EA01200549096840EA72
:10C37000014070471C000020580500205405002093
:10C380005C050020020003D081429241D20F00E000
:10C39000012210467047F8B500F02DF838B100F0D2
:10C3A00031F8BDE8F84040F20371FDF7BBBDF1BDC7
:10C3B00038B504460D460820FBF7C7F968B1216877
:10C3C00091F82C1001704560024604F11400BDE89C
:10C3D000384040F20571FDF7A5BD31BDF8B500F05C
:10C3E0000AF838B100F00EF8BDE8F84040F20171EB
:10C3F000FDF798BDF1BD04460D4616461F460C20BC
:10C40000FBF7A3B9216891F82C1001700246458012
:10C410000671C7800699816004F114007047F8B571
:10C4200004460D4616461F460820FBF78EF948B114
:10C4300000F05EFA04F11400BDE8F84040F2047127
:10C44000FDF770BDF1BD2DE9F04F8046894693465A
:10C4500085B01F4659464846FFF794FF08B10123AF
:10C4600075E00E993846FEF7F4FF0228ADF8020099
:10C470000ED80221112006F0EBFF01904FF0FF369D
:10C48000B8F80C00801E03904C4603A8078802E011
:10C4900010235CE06C1CA1B28B4552D3BDF8022086
:10C4A0005946A0B2FFF74DFB0028044649D0BDF81D
:10C4B00002205946FFF75EFB05460020ADF800005C
:10C4C00004AB6A4621464046FFF75AFA8246039873
:10C4D000BDF80010001F884203DA0398001FADF872
:10C4E0000000002EBDF800000BD4B04202D1001DA8
:10C4F00087420BDA01994A7A1144301D00F0B7F8EF
:10C50000BAE00646381F8642C8BF0646200A8DF8A4
:10C5100009008DF80840280A8DF80B008DF80A50A4
:10C520000422019802A9FFF7E1FD0198F2B25146F9
:10C53000FFF7DCFDB81B071F4FF6FF708542BFB247
:10C54000A8D116F1010FD5D100F078FA0A234A4696
:10C550001021404606F0D2FFD2E72DE9F04F804689
:10C560000D46914685B01C4649462846FFF70AFF0E
:10C5700008B101232FE00E992046FEF76AFF83469B
:10C580000221092006F064FF01904FF0FF37B8F850
:10C590000C00ADF80C50841EA4B2264600E06D1CC1
:10C5A000A9B289455AD35A464946A8B2FFF7C9FAF3
:10C5B000050053D0012229464046FFF713F90290A7
:10C5C00018B100F03BFA029B05E000F060FA40B1C0
:10C5D00000F034FA80232A460821404606F08EFFF8
:10C5E0001FE0ADF8000002AB6A4629464046FFF75F
:10C5F000C7F98246BDF800102046884288BF084629
:10C60000ADF80000002FBDF800000BD4B84202D1F5
:10C61000801C86420BDA01994A7A1144B81C00F05A
:10C6200026F829E00746B01E8742C8BF0746280AF9
:10C630008DF803008DF80250022201980DF10201DD
:10C64000FFF754FD0198FAB25146FFF74FFDF01B7A
:10C65000861E4FF6FF708542B6B2A0D117F1010FCA
:10C66000D9D100F0EBF9BDF80C200A23B4E74874E7
:10C670004046019906F03BBF05B0BDE8F08F2DE9BB
:10C68000FC4704460F4688B011463846FFF77AFE4D
:10C6900010B101233A4652E00221052006F0D8FEEF
:10C6A00000904FF6FF78A089ADF80470851EADB2FA
:10C6B000C14600E07F1CBDF82000B9B2884236D3E5
:10C6C000B8B2FFF781FA8246C24530D04FF400621B
:10C6D000B9B22046FFF786F80028EBD15FEA0A409E
:10C6E0004CBF10260226C14509D00AF4004009F4C7
:10C6F000004188421BD1B01C854201DA17E0D146C7
:10C700003804000E8DF809008DF808700DF10A014B
:10C710005046FEF7CDFEB21C0098D2B202A9FFF738
:10C72000E5FCA81BBFB2851E4745ADB2C2D1C145CD
:10C730000AD16846FFF7FCFBBDF804200A23042158
:10C74000204606F0DBFE0DE00098417A084400F137
:10C7500010015FEA09404CBF0220012048702046CA
:10C7600006F0CAFE0AB0BDE8F0872DE9FE4F054687
:10C77000180A8DF8010090468DF800300E464146AB
:10C780003046FFF7FFFD3446002708B1012006E0E0
:10C79000284606F007FF5FEA000902D11120019048
:10C7A0002BE069460220FEF754FE824606E0042391
:10C7B00002AA4946284606F039FE012741468C4226
:10C7C0003BD2DFF85C060068029052462046FFF735
:10C7D000B8F9040031D052464146FFF7CBF9834601
:10C7E00001AB0DF1020221462846FFF7C9F8019975
:10C7F00059B12646484606F071FE019B3246062195
:10C80000284606F07BFEBDE8F78FBDF80210BDF8A4
:10C810003420ADF808409142ADF80AB05C46CDD165
:10C82000BDF834200C99FDF797FD0028C6D1494684
:10C83000284606F0EEFD0428B9DA17B90A2001905F
:10C84000D8E74946284606F057FEDCE738B51446D7
:10C850001A46456B00234363049B23B10A462946CD
:10C8600006F04CFE07E00C2D214602D106F0D3FE67
:10C8700001E006F0B8FE002032BDFEB517460026E6
:10C8800004460D46ADF804600122FEF7ABFF0290AE
:10C8900020BB00F0FCF868B1666B0820FAF755FF82
:10C8A00028B300F025F840F2027104F11400FDF7FE
:10C8B00039FBF7BD02AB01AA29462046FFF760F815
:10C8C0000646029850B9BDF80400B84202D20720CB
:10C8D000029003E0C01B3E44ADF8040032460298CB
:10C8E000BDF80430009029462046FFF7AFFFF7BDA2
:10C8F000216891F82C10017045800671C7800246AE
:10C9000070470A2242630022B7E70C234363B4E76F
:10C910002DE9F04F824683B0BAF80C00461E0C4653
:10C920001746304607F0FBF900258346D8460095A8
:10C93000A9462FB107EBD7704010B7EB40000CD0E1
:10C9400004200090009B4A460E21504606F0D6FD7A
:10C95000584607F0EDF9BDE8F78F607814F8021B30
:10C9600041EA0029012249465046BF1EFEF73AFF20
:10C9700000280090E6D14846FEF732FE08B180203C
:10C98000DFE76B4601AA49465046FEF7F9FF0099DA
:10C990000029D7D1BDF80420711B9142B8BFADF872
:10C9A0000410BDF8042001464046F9F747FDBDF8E4
:10C9B00004004519002F8044CFD1AAB259465046F1
:10C9C00006F050FEC4E780B5002343632AB1134646
:10C9D0000A46122106F092FD01E006F06DFE0020ED
:10C9E00002BD76B50446122060630D460222204641
:10C9F000FEF7F8FE060002D000F020F812E00198E1
:10CA00000199407AC01C487200F041F830B1019899
:10CA100000900023122200F037F873BD019B00F054
:10CA200008F8064600F001F873BD32462946204654
:10CA3000C9E7002229462046FEF7DDBF01A8FFF71F
:10CA400077BA34B582B004460D460422FEF7CAFE1A
:10CA500018B102A8FFF76CFA37BD02980299407A24
:10CA6000C01C48725220606300F011F830B1029887
:10CA700000900023522200F007F837BD029BFFF719
:10CA8000D8FF0020606337BD2946204683E428464E
:10CA9000FEF7A6BDF2B504460846497A00F080F8D4
:10CAA0002846FEF76AFD98B901276846FFF740FA65
:10CAB00000F072F83B462A461621204606F01EFD7D
:10CAC000092F04D140F209412046FFF771FCF1BD66
:10CAD000022229462046FEF785FE0700E5D1009890
:10CAE0000121FFF754F908B90927DEE7014604F1EF
:10CAF0005000FFF7F1FA00980099407A401D487203
:10CB00003246009B2946204606F010FEF1BD7CB55A
:10CB1000044600200D461646019026BB04F1500045
:10CB2000FFF711FA0190F0B1417A00F039F8FFF700
:10CB3000AEFF00280198407A09D00199401D487243
:10CB40003346019800901822FFF79EFF22E00199DA
:10CB5000401D48723246019BFFF76CFF06460020DD
:10CB6000002E0190DAD0FFF769FF00F015F80020E1
:10CB7000606346B133462A461821204606F0BEFCC3
:10CB800006F5806103E0204606F009FE00212046FC
:10CB9000FFF70EFC002076BD04F15000FFF7C8B986
:10CBA00008441030B0F80150B0F80360704710B579
:10CBB000044631B9FFF7F0FF2046BDE8104006F00B
:10CBC000EEBD1820606300222046BDE81040002121
:10CBD0009DE738B50446258F280020D042F6052071
:10CBE000FFF701F8A8420BD1FDF749FCE0630423ED
:10CBF000206890F9540004F13C020C2107F080F900
:10CC000040F20A612046FDF7C1FC00F009F8034636
:10CC1000022229462046FFF702FC0020208731BD72
:10CC200029462046FEF78DBD2DE9F04104460D460C
:10CC3000164698462846FEF7ACFC0746FFF7F0FF7D
:10CC4000F90607D5C10705D500F097F806F0B0FD45
:10CC500088B111E0B90611D580070FD5208F68B9CA
:10CC600000F08BF806F0B8FD30B9258740F20A6174
:10CC70002046FDF782FC0020BDE8F08140F28110E3
:10CC8000FAE72DE9F84304460D46904699460026FA
:10CC900000272CB1E069012808BF40F2031029D019
:10CCA0002846FEF776FC3021084208BF4FF4C070DA
:10CCB00020D044B90126002002E000B90127204617
:10CCC000FDF7E8FC044674B1E069012809D04B4641
:10CCD000424629462046FFF7A7FF002EEDD110B1AE
:10CCE00008E0002EEBD187F00100064214BF40F2AD
:10CCF00081100020BDE8F283F8B504460D46E069D6
:10CD0000012816461F4600D13CE0FFF7C0FE00B9DF
:10CD10003BE0606B0A2818BF0C2807D106980090EA
:10CD20003B4600F02BF8FFF791FDF2BD40F2811079
:10CD3000F2BDF8B504460027E06901280D46164605
:10CD400000D11FE0FFF7A3FE00B91EE0606B1228C0
:10CD500004D0182807D0522803D00AE0FFF765FE58
:10CD600005E0676307E000F009F8FFF7D0FE07462B
:10CD700001E040F281173846F2BD4346324629466B
:10CD80002046704740F20310F2BD4FF4C070F2BD70
:10CD90002DE9FC41044642F60520FEF724FF054636
:10CDA00020480088ADF802000DF102010220FEF7D4
:10CDB00050FB0126074624E001AB6A463146204677
:10CDC000FEF7DEFD019901291AD0BDF800100329F4
:10CDD00016DB4178807851EA002811D0A84504D1AB
:10CDE0004146204600F020F850B94146FFF719FFB0
:10CDF000010005D00346012241462046FFF70FFB04
:10CE0000761CB0B2FEF7B9FB38B13A464FF6FF7167
:10CE1000B0B2FEF796FE0600CED1BDE8F381000069
:10CE2000005B0000BEA10000F8B507460025002FFA
:10CE30000CBF012600260120ADF800000C464FF67D
:10CE4000FF70ADF802001EB13846FDF723FC07461F
:10CE5000BFB1FDF714FBF96B884210D03846FEF7DE
:10CE6000D2FE21463846FEF76CFC022807D1042387
:10CE70006A4621463846FFF7D7FE00B96D1C002EE2
:10CE8000E2D1E8B2F2BDFEE7002806D55C4900F029
:10CE90000F00084410F8040C01E05A49085C4009EE
:10CEA000704738B504460D4607F0D2F85649D1E927
:10CEB0000023C4E90023D5E90023C1E90023BDE82C
:10CEC000324007F0C9B810B5044607F0C1F8D4E9FC
:10CED00000234D4906E010B5044607F0B9F8D4E93F
:10CEE00000234A49C1E90023BDE8104007F0B4B867
:10CEF000F8B5074607F0ACF8444ED6E9004507F010
:10CF0000ABF838687968044001EA050220EA0404B5
:10CF100021EA0200210008BF0028054604D0C6E926
:10CF200000453948C0E90045F1BD10B500F00AF8E8
:10CF3000184304E010B500F005F823EA000041F8BA
:10CF4000220010BD421151F82230012400F01F00D0
:10CF500004FA00F0704710B5044607F079F82B4941
:10CF6000D1E90023C4E90023BEE770B5064607F007
:10CF70006FF82649D1E9004507F06EF83068204285
:10CF800005D170682840401E8041C00F70BD002050
:10CF900070BD1E49421151F8221000F01F00C1401F
:10CFA00001F0010080F0010070471949096801EBA8
:10CFB0008000006C7047164A126802EB8000016422
:10CFC0007047F0B5059D069C002603E00FB942F8B6
:10CFD0002650761C9E420FD2270002D08E42F6D2F7
:10CFE00005E052F826708E42F0D2002FF1D150F8B1
:10CFF000267042F82670ECE705480260F0BD00009C
:10D0000018ED00E000E400E080E100E000E100E075
:10D0100008ED00E072B67047002343720174931C60
:10D0200083724274704770B516460D461A1D044649
:10D03000D2B20E21FFF7F0FF00F06EFA0121A0F846
:10D0400003504671817070BD38B50D4604463E21CF
:10D05000FFF7E2FF607A2044857431BD00234372FC
:10D0600081820623837282740F2303740423437422
:10D070000123C3747047816841F00401816007F0A7
:10D0800059B810B50446002350E3DFF8080BFEF74B
:10D090004FBF38B5DFF8FC4A2046FFF70AF8050015
:10D0A00012D0206818B14FF00040FCF741FCA8688E
:10D0B000C0F380000028284602D0BDE8324027E0B7
:10D0C000BDE8324000F0F8BC31BD38B504460EE092
:10D0D00038B500F0BAF9008AC0F30131481EA168E2
:10D0E0008041C00F21F0020141EA4000A060FCF73E
:10D0F000FDFF05462146DFF89C0AFEF7EDFF4FF0E5
:10D100000040FCF715FC2846BDE83240FCF7F2BFB2
:10D1100010B5044640F20641607A2044008A401A65
:10D120004CD040F2FB71401A50D0801E4AD03238A9
:10D1300000F0C7804FF47571401A4BD04FF47F71E7
:10D14000401A00F0968040F6FC31401A46D0401F4D
:10D150004BD0801E4DD0401E4FD0401E51D0401E9F
:10D1600053D0401E55D0401E57D0401E59D0401FAE
:10D170005BD0C01E00F08180401E5AD0401E5CD0A3
:10D18000401E5ED0401E60D0401E62D0801E64D023
:10D19000401E66D0401E68D0C01E72D0801E74D063
:10D1A0004DF6DF31401A00F08080401E71D0401EE5
:10D1B00073D0401E75D0401E7BD07EE02046BDE877
:10D1C000104084E02046BDE810409FE0002240F679
:10D1D000014106E02046BDE81040A2E0002242F2F4
:10D1E00001012046BDE810404BE72046BDE8104055
:10D1F000A6E12046BDE810402BE12046BDE81040E6
:10D20000C8E02046BDE810408AE12046BDE8104055
:10D21000B2E12046BDE81040C9E12046BDE810401B
:10D220004FE22046BDE8104038E22046BDE81040FD
:10D2300005E22046BDE8104094E02046BDE81040DD
:10D2400080E02046BDE81040B1E02046BDE8104037
:10D25000E4E02046BDE81040CFE02046BDE81040A5
:10D26000BCE12046BDE81040C8E12046BDE81040C2
:10D27000D6E12046BDE81040A5E22046BDE81040BA
:10D2800083E22046BDE810405CE22046BDE8104045
:10D2900041E22046BDE81040EFE02046BDE81040E6
:10D2A000F7E02046BDE8104004E12046BDE810400C
:10D2B0008AE32046BDE8104017E1204600F072FCEA
:10D2C00020B92046BDE81040FEF797BD10BDF8B567
:10D2D00000F0BBF810304579B0F8030001F043F9D5
:10D2E00006000BD0FCF702FF07462946304607F040
:10D2F00072FC05463846FCF7FDFE00E00225EAB266
:10D3000040F2064100F0C8F9204601E210B504469B
:10D3100002F093FB2046BDE81040002240F6034196
:10D32000AFE610B504460623002241F20901FFF7DB
:10D330007AFEA07ADFF86018204406220A30F9F756
:10D340007DF8F5E110B504460823002242F21801E9
:10D35000FFF769FEA07A204400F10801082007F0D9
:10D36000A0FEE5E11FB50446694600F0D5F8C21CF1
:10D37000133002F098FC1023002242F2170100F053
:10D38000FBF9A07A102269462044F9F757F800F01B
:10D3900090FB1FBD10B500F069F8012002F058F9AC
:10D3A0002046BDE81040002242F2090169E670B54E
:10D3B00000F04BF8B0F813500220FEF7C9FC06004D
:10D3C00006D1072242F2130100F066F9204613E06D
:10D3D000284601F0C8F820B1214607F040FB02467C
:10D3E00003E02046FEF709FD0222D2B242F2190103
:10D3F0003046FFF733FE304600E210B500F0BEF9CC
:10D4000020B1002107F0B6FB024600E002222046D0
:10D41000BDE81040D2B242F21B0132E638B500F04E
:10D4200014F800F11005B5F8030001F09CF820B1E4
:10D43000691D07F09FFB024600E002222046BDE87E
:10D440003840D2B242F21A011BE60446607A204408
:10D45000704710B500F00AF8002002F0F9F82046F5
:10D46000BDE81040002242F208010AE60446607A54
:10D4700020441030011DC278704710B500F05CF9EF
:10D4800002F0F9F82046BDE8104000224FF60441B2
:10D49000F7E570B500F01FF800280EBF0225D6F89A
:10D4A000051001F0CDFE2A462046BDE870404FF63B
:10D4B0000541E6E570B500F00EF800280EBF022524
:10D4C000D6F8051001F0C3FE2A462046BDE870409C
:10D4D0004FF60641D5E504460025607A204400F168
:10D4E0001006B6F8030001F03EB838B50446002532
:10D4F00000F012F8C178012906D1406800B101207E
:10D50000C0B202F0BBF900B912252A462046BDE898
:10D5100038404FF60741B4E5607A20441030704738
:10D5200010B5FFF792FFC07C02F0BFF8002820463C
:10D53000BDE8104014BF0022072242F20A01A0E514
:10D540001FB500F046F8817B0391417B0291C11D1C
:10D55000019181790091437902794188008802F034
:10D5600056F8010018BF0C200246204604B0BDE862
:10D57000104042F2060184E510B5044682B0607A9C
:10D5800020441330817900914379B0F80320B0F83A
:10D590000110007800F07FFB02B000282046BDE8B3
:10D5A000104014BF00220C2242F20B0169E510B5B5
:10D5B00000F00FF8417801B10121007800B101209D
:10D5C00000F0B4FB2046BDE81040002242F20C01FE
:10D5D00057E50446607A20441330704710B5FFF7D2
:10D5E00034FFC07C07F041FE00282046BDE8104013
:10D5F00014BF00220C2242F21D0142E510B5FFF7D4
:10D60000E8FF82784178007807F0EFFD0028204697
:10D61000BDE8104014BF00220C2242F21E0130E58A
:10D6200038B5044607F05DFE05460223002242F2AB
:10D630001F0100F0A1F8607A2044C58298E02DE92E
:10D64000F041044642F2130600F0B7F8050001D19C
:10D65000022205E00220FEF77BFB070005D107222E
:10D66000314600F019F8204613E0607AC01C607261
:10D67000FCF73CFD80462146284607F007F90446A2
:10D680004046FCF737FDE2B231463846FFF7E6FC8C
:10D690003846BDE8F041EEE42046DFE438B5044604
:10D6A000FCF724FD054600F031FB002814BF0022E2
:10D6B0000C2242F20E012046FFF7E3FC00F013FBC0
:10D6C00021E5F8B5044601F02BFA05460220FEF7E5
:10D6D0003FFB060042F20D0703D065B9FEF78DFB54
:10D6E00003E015B1284601F03EFA07223946FFF75C
:10D6F000D3FF20460CE0607AC01C607229462046A9
:10D7000000F0F4FDC2B239463046FFF7A7FC3046C0
:10D71000BDE8F240AFE410B500F00EF8C0B201F081
:10D7200058FD0023002242F224012046FFF77BFC33
:10D730002046BDE810409EE40446607A2044B0F8DC
:10D740001300704738B500F019F8054602224DB1B4
:10D7500000F0A9F828B10146284607F052F9024620
:10D7600000E007220023D2B242F2220100F004F8C6
:10D770002046BDE832407EE4204654E40446607A08
:10D780002044B0F8130000F0EEBE70B50446022548
:10D7900000F013F8064600F086F80CB9072505E0FE
:10D7A00026B10146304607F0DFF80546EAB22046CA
:10D7B000BDE8704042F2160163E4607A2044B0F89C
:10D7C000130000F0D0BE70B504467F26607A204476
:10D7D000B0F81350284600F0C6FE20B100F060FEFD
:10D7E0000646002200E00222032341F20541FFF732
:10D7F000C3FFFFF791FEC58006722046BDE870406A
:10D8000039E42DE9F04104460D4616461F4600F066
:10D810004AF85FEA000811D00A220321FFF714FC3E
:10D8200098F80900404410300021C1708480C58000
:10D83000068147814046FFF71EFC0120BDE8F081CC
:10D840002DE9F843074688461646994600F02BF81E
:10D85000040008BF002024D013220121FFF7F4FBAD
:10D86000607A204400F110050C98E870AF805FEA00
:10D87000080018BF0120A8714946300018BF0120D8
:10D88000E871062205F10800F8F7D8FD0898E8814C
:10D89000099828820A9868820B98287500F009F97F
:10D8A0000120BDE8F2830120FEF752BA2DE9F041D4
:10D8B00000F071F85FEA000808BF002013D00C22C6
:10D8C0000421FFF7C1FB98F80900404400F110075C
:10D8D0000821BC80B81DFCF76FFCBD71FE7040468E
:10D8E000FFF7C9FB0120BDE8F08170B500F0A4F896
:10D8F000060001D1002070BD04220821FFF78CFB37
:10D90000707A30441030691E8941C90FA0F8034075
:10D91000417185708BE02DE9F04105460E461746B2
:10D920009846FFF7C0FF040008BF002015D00B2267
:10D930000721FFF789FB607A204400F11001A1F86C
:10D940000350A1F80560A1F80770A1F809800698B6
:10D95000A1F80B0000F0ADF80120BDE8F081F8B5AA
:10D9600000F019F8070001D10020F2BD0D220521B9
:10D97000FFF76AFB787A38441030A0F80340A0F82B
:10D980000D5008223146401DF8F758FD3846FFF784
:10D9900072FB0120F2BD04460D4616460120FEF73B
:10D9A000D7B910B5FFF77FFF040001D1002010BDEB
:10D9B0000122FF21FFF730FB617A214400208874A7
:10D9C00000F077F8012010BD10B5044698B0002093
:10D9D00060720220A07248202074684601F07CFC2E
:10D9E000A0826022694604F11600F8F727FDA07CAA
:10D9F00006214843401C6074617CA07A0818A0721C
:10DA000000F057F818B010BD70B500F015F806001A
:10DA100001D1002070BD04220521FFF7FDFA707AC4
:10DA2000304410300021A0F8034045718170304629
:10DA3000FFF721FB012070BD04460D460120FEF7D3
:10DA400087B92DE9FC470D46544991469A46D1E9DC
:10DA50000023CDE900230A9C617A8046A07A461A09
:10DA60000D212046FEF7A5FA607A201800F1100774
:10DA70003E203870062206F10C00787049460220DC
:10DA8000B8700120F8701DF8080038717D71B81D5C
:10DA9000F8F7D4FC3E73A07A201880F810A0A07A82
:10DAA000401CA0722046FEF7B5FB00F002F8BDE86E
:10DAB000F3872046FFF7DFBA2DE9F0470446A06858
:10DAC000400800F00105607A2044067C304600F0F2
:10DAD0004AFD5FEA000904D12046BDE8F047FEF7A1
:10DAE0008CB9A06820F00400A060607A001D60720C
:10DAF000484601F07BFB804625E0A07A617A401A17
:10DB0000C2468045C8BF8246022078725246607A7B
:10DB1000204400F1100107F11200F8F78FFC787A29
:10DB20005044B872607A50446072A068B968400886
:10DB300060F34101B9603946A06820F00200A0609E
:10DB4000484601F0BBFAA07A617A401A804519DA9A
:10DB50000020FEF7FDF80700CFD1607A001F607249
:10DB6000C0B2204430F8101F01F4704131430180ED
:10DB70002146A06865F34100A060BDE8F047054874
:10DB8000FEF700BB21464846BDE8F04701F096BAD3
:10DB900000000000080B0020E4070020A45A000049
:10DBA00006F0E4BA00207047890001EB401000F154
:10DBB0000850026070470122F6E70022F4E70000F7
:10DBC00070B5DFF84868341D0B2806F134054DD8D0
:10DBD000DFE800F0064C1C4927242D2D4C2D2D2A62
:10DBE0002878DFF82C28DFF82C18012301F065FFD6
:10DBF00001F0EAFE07F0A9FB054600F08EF8216867
:10DC0000A5F1C802BDE8704001F0A1BF07F07CFC9F
:10DC1000B0422BD1BDE8704001F0D6BEBDE87040E7
:10DC200006E2BDE87040BFE101F0CEFE1BE000203F
:10DC300000F088F907F08DFBA16881420CDA01F051
:10DC4000C3FE07F082FB044600F067F8A4F1C801A8
:10DC5000BDE8704001F05CBF01F011FFE9694018B8
:10DC60002168401AE861BDE87040B5E070BDDFF89A
:10DC70009C07102101854185C18601870021016330
:10DC80004162DFF89417C16102214161FA2181608C
:10DC9000182101767047F8B5DFF870770C4697F8D1
:10DCA0002410C90715461E4601D50020F2BD28B133
:10DCB000012107F12400FFF77EFF04E0012107F1B5
:10DCC0002400FFF77AFF3C857D853E630120F2BD8D
:10DCD000DFF8380790F8240010F0050F04BF00208B
:10DCE00000F03DBA704710B5FCF700FA0446DFF8C3
:10DCF0001C07416A4A0704D521F004014162FFF77D
:10DD0000E7FF2046BDE81040FCF7F4B9DFF8FC0659
:10DD1000406A800800F001007047DFF8F00690F8D4
:10DD2000240010F0060018BF01207047F8B5DFF896
:10DD3000DC562C1D216A58B9C8074CD5FCF7D6F91A
:10DD40000746206A400840002062FFF7C1FF3DE01F
:10DD5000C80740D4880705F1340612D50220FDF724
:10DD6000F7FF3061B8B3032105F12400FFF725FF69
:10DD7000042105F12400FFF720FF00203076012068
:10DD80007083FCF7B3F90746002105F12400FFF783
:10DD900012FF94F82000400718D40020F06140F2F0
:10DDA000712140F6C410A060E08C801E4843E06002
:10DDB0002520307001F063FE61680818643020602F
:10DDC0003062284607F0E9FA07F06AFB3846BDE8FA
:10DDD000F240FCF78FB9F1BD2DE9F041DFF82C4698
:10DDE000251D0121204607F0F4FA04F13406E98CE0
:10DDF000F06940F27128091F08FB01F1884219D32C
:10DE000001273078A98C401CC0B22828A8BF252043
:10DE10003070306A08FB0100286030620020F06139
:10DE200095F8200000F00400CFB1002814BF322084
:10DE300010200FE001F023FE316A401AE968002744
:10DE4000A1F6C4118842DCD201F019FE00F57A7007
:10DE500028600DE0297D88420AD2481E07E000288C
:10DE6000297D14BF3C202020814201D2481C287506
:10DE7000204607F092FABDE8F04107F011BB2DE90A
:10DE8000FF41FCF733F9DFF884150A6A019200229A
:10DE90000A62FCF72FF902E02046FDF7AEFF019879
:10DEA00010B301A8FEF705F904460622677AE019C7
:10DEB0001030418990F9056001F00F05C1F3801819
:10DEC00000F10C0102A8F8F7B9FA07F1120060722C
:10DED000C0B2A17A8142DFD30094F3B202AA4146D4
:10DEE0002846FFF7AEFDDAE7BDE8FF8170B5DFF841
:10DEF0001C55417A2E6C084400F11004707A628936
:10DF00003044C2F38012018AC1F3C011914206D19C
:10DF1000062204F10C011830FCF71EFA08B10020AB
:10DF200070BD304601F04FFE002001F08FFE2089C9
:10DF3000216801EBC000A864686A40F020006862B4
:10DF4000012070BD38B5DFF8C444616A0A072AD5DC
:10DF5000090901F0010104F14C0558B121B16888AB
:10DF60000228A4BF40086880042104F12400FFF7C0
:10DF700022FE0AE021B96888FF28DCBF40006880E3
:10DF8000042104F12400FFF718FE01F076FD6988F2
:10DF900090FBF1F201FB12002870032104F1240030
:10DFA000BDE8344009E631BD30B5DFF8604494F88F
:10DFB0002400800683B036D5E06B256C697A002397
:10DFC000E3632364294401F110021231128812061E
:10DFD000D20F019201F10C038A1D0092A16C01F293
:10DFE0001532012100F05AFE2846FDF706FF606A4F
:10DFF00020F02400606201F0E7FC94F82400C007E0
:10E0000003D4BDE83E400120A9E01820207607F0A7
:10E010009CF90446FFF781FEA4F1C80103B0BDE8F6
:10E02000304001F075BDBDE83E40012001F0BBBDB0
:10E030002DE9F04782B001F08EFC0024050021D0CC
:10E04000697A681810300279B2B1428902F00F067D
:10E05000100A072E00F03F000ED206280CDB2628FF
:10E060000ADA012E01D10C2806D140180C30002EFE
:10E07000A87201D4072E06D32846FDF7BEFE002065
:10E08000FFF760FF5CE0DFF88483DFF8909308F12E
:10E0900024073878400707D519F82600800703D5EC
:10E0A0002846FFF723FF04463868C10744D5042EED
:10E0B0000CBF4FF0010A4FF0000A210028D1800761
:10E0C00026D55046FFF73EFF19F82600C0071FD59A
:10E0D00098F84C00010003D0401E88F84C0017E06F
:10E0E000687A002128440091032330F81A1FC1F3F5
:10E0F0008012811C386A00F071F8386A01F063FD03
:10E10000012001F0A3FD03213846FFF754FD01244F
:10E11000BAF1000F02D0387880070DD519F8260023
:10E12000400709D5294608F12000FDF7D5FF4FF03B
:10E130008040FBF7FDFB02E02846FDF75EFE64B978
:10E1400001F042FC07F001F90446FFF7E6FDA4F1F7
:10E15000C801BDE8FC4701F0DBBCBDE8F387F0B5C2
:10E16000AA4D0446686C85B018B1FDF746FE002044
:10E170006864E86B18B3296CE1B14A7A114401F183
:10E18000100601F1120700F0FDF9022207F1160155
:10E190000492BB1DCA7A5209039280B28A88029205
:10E1A0004A8801920988009131880906CA0F002126
:10E1B000FFF746FBE86B00F0D6FC0020E863286C14
:10E1C00018B1FDF71AFE002028642146284607F002
:10E1D00000F905B0BDE8F04007F062B970B504463B
:10E1E00000200D46607203F00F01207C049E00F0B9
:10E1F000C000084306F10C01090201F47C510843F8
:10E2000020824FF6BF7108408049096B01B101219E
:10E2100040EA811020824FF67F710840110018BF3C
:10E22000012140EAC110208206227D4904F112003A
:10E23000F8F704F90622294604F11800F8F7FEF869
:10E24000607A30180E30A07270BD80B50421684627
:10E2500001F004FC0098002100F03F023F2A18BFA3
:10E2600010F03F0F03D04008491C1B29F4DB1B2989
:10E27000ECDB0098664948400022002120FA01F3B7
:10E28000DB0748BF521C491C2029B8BF022AF5DB16
:10E29000022ADBDB9DF800009DF80110884201BFD7
:10E2A0009DF8021088429DF803108842CED0009855
:10E2B00000221F2100F00303022B14BF012B521C6C
:10E2C0004008491EF6D1192AC0DA0098800E0022B3
:10E2D000052100F00303022B14BF012B521C400840
:10E2E000491EF6D1022AB1DB009802BD2DE9F041AA
:10E2F000DFF8188108F10405074695F8200040076B
:10E3000088B00C4607D53846FDF777FD204600F06B
:10E310002AFC0C2076E008F134061922B460787AE1
:10E32000384400F1100101A8F8F788F81620009091
:10E3300005239DF809200DF10A013846FFF74EFF2D
:10E34000787A384400F11E04FFF77FFF2060032134
:10E35000201D01F083FB0220E071BDF813006081F5
:10E3600001F08BFB6189491C90FBF1F201FB12006B
:10E370002081FF22BDF81500A0810521BDF81700FE
:10E38000E08104F11000FCF731F8207D00F01F005F
:10E3900020750C21207990FBF1F10C2202FB110079
:10E3A000617D401D60F30401617501F060FC617DD9
:10E3B00001F01F0141EA40106075F760FBF796FE1F
:10E3C0000746286A40F004002862C00716D440F6C9
:10E3D000C410A86040F27121B088801E4843E860F4
:10E3E0002520307001F04BFB696808186430286004
:10E3F0003062404606F0D1FF07F052F83846FBF78E
:10E4000079FE002008B0BDE8F0810000240B002058
:10E41000D6BE898E55555500C1DB0000E45A000078
:10E42000E4070020890001EB401000F10850026071
:10E4300070470122F6E70022F4E750E8002F0A4374
:10E4400040E80023002BF8D1704750E8002F8A43A2
:10E4500040E80023002BF8D170470F31012805D088
:10E4600002280CBF88004FF6FF7000E0C80080B2A1
:10E47000704790FBF1F201FB1200002848BF08181A
:10E48000704710B101F18400704701F1A800704796
:10E49000CC307047006A70472030CEE72030D4E798
:10E4A00090F965007047012904D017D3032906D0DD
:10E4B0000DD313E0818C828E008E120103E0818CDB
:10E4C000008E4FF47A4292FBF0F0401804E0818C09
:10E4D000408E01EB4000C01D80B27047808C7047B9
:10E4E00070B504460D46164600F055FE40F2712107
:10E4F000636801FB06F201FB053194F82030A1EBC3
:10E5000010211B07616006D5216F400000EB02203F
:10E510004018206770BD01EB5200606070BD816FD4
:10E5200000291EBF8968C1F38001002908D1C06F8E
:10E5300000E0006828B18168C1F380010029F8D0AB
:10E540000120704780F86410704710B5044600F051
:10E5500077FA204600F016F8BDE81040012101FAD4
:10E5600000F0FBF7E5B9DFF8801C91F8202090421D
:10E5700006D2496801EB002090F82010C90600D4AB
:10E5800000207047DFF8601C4A68801A001203D42C
:10E5900091F82010884201DB4FF0FF3070472DE9E1
:10E5A000F043044604F1200585B02868DFF8387C84
:10E5B000410204F15C0629D58108C00800F0010978
:10E5C00001F0010800F0D4F80021049104F15E0389
:10E5D000317803914246A98A029180B2698A0191F9
:10E5E000298A490800914946FFF72AF9002835D0C1
:10E5F0004FF4800100F0BAF83878C00706D5002043
:10E60000FDF7A6FB0146204606F0AEF92868C001DA
:10E610000ED500F0ADF8298AAB8A6A8A490880B223
:10E62000FFF7EFF8002819D04FF0807100F09EF846
:10E630002868800108D5204606F003FC00280DD08C
:10E640004FF0007100F092F8286840010BD500F0FF
:10E650008FF8002180B2FFF748F9002879D04FF0F9
:10E66000806100F083F82868C0001ED500F080F8B3
:10E67000B1890022C9B280B2FFF718F9002868D02A
:10E680004FF0805100F072F897F821001C280CDB45
:10E690000521204600F06EFE38B10020FDF758FB42
:10E6A00018B10146204606F0ACF9286880001AD55A
:10E6B000D4F8FC00F17A00F092FC0746D4F8FC0094
:10E6C000B17A00F08CFC804600F052F80097F37AA3
:10E6D000B17A424680B2FFF71EF9002839D04FF0D8
:10E6E000005100F043F82868002810D500F040F8E9
:10E6F000D4F8FC10337A090A01F00F02114680B2F7
:10E7000006F012FF28B34FF0004100F02FF8286800
:10E7100000010AD500F02CF8317A80B2FFF7E5F855
:10E72000B8B14FF0006100F021F82868400006D52C
:10E730004FF0804100F01AF8204606F059FC286896
:10E7400000020FD500F014F8317A80B2FFF75CF9BF
:10E7500008B9002007E04FF4000100F007F8204658
:10E7600000F001FA012005B0BDE8F08328466CE610
:10E77000204607E710B50B280C4624D8DFE800F048
:10E78000062312211B171F1F1F1F1F1F204600F0EB
:10E790005CF9204600F014FB6168BDE810400120E0
:10E7A00001F03ABA06F0B0FEA0420CD136E02046A5
:10E7B000BDE8104008E1204600F027F932E00121D1
:10E7C00000E0002134E010BD10B50B280C4624D821
:10E7D000DFE800F0062312211B171F1F1F1F1F1F3A
:10E7E000204600F032F96168206FBDE8104001EB6F
:10E7F0001022012001F0ABB906F086FEA0420CD138
:10E800000CE0204600F0E0F80CE02046BDE81040A7
:10E81000FBE0012100E000210AE010BDBDE810404E
:10E8200001F0D2B8BDE810400521DFF8080B02E680
:10E830002046BDE8104058E0DFF8AC190A7E5206C9
:10E8400009D590F82020120705D54969891E416035
:10E850004FF400610167704770B50446002594F8D5
:10E86000200000070DD5606FE18C4843216F420006
:10E87000050A02F580725118080A00F548702167F0
:10E88000E06040F27126208E401E7043206101211D
:10E89000204606F09EFD218EE28C6068514306FB07
:10E8A0000100401B6060204606F077FDBDE8704027
:10E8B00006F0F6BD00F118018A8B0B8B120392FB58
:10E8C000F3F2222392FBF3F230F86C3FC06810B1F0
:10E8D00003EBD3704308180290FBF2F0C0F1400044
:10E8E0001E28B8BF1E20087070472DE9F0475FEA68
:10E8F0000109804604D001F067F84046FFF79CFF0D
:10E9000008F120054046A988DFF8DC4805F05EFCE8
:10E91000B9F1000F824608F15B0608F16C0705D0DB
:10E92000207E800702D500F066F909E0388838B902
:10E930002868C0054CBF08203E2070724FF0000AC6
:10E940004046FFF7B7FFBAF1000F0CD14FF40001BA
:10E950004046FFF7FAFD0121404606F03AFDBDE8CA
:10E96000F04706F09DBDB9F1000F18D028680107E7
:10E9700015D5698A99B110F4C02F10D1207E800777
:10E980000DD5386958B9A988404606F0C2FA698A97
:10E99000012802DB4A1C904202DB481C00E00120F7
:10E9A000E880A988E8884118A9803988091A39803F
:10E9B00025213378B27858438018FFF75AFDB0709C
:10E9C0004046BDE8F04747E738B5044600F0C3FFCE
:10E9D00040B10146204600F032FA0121204600F005
:10E9E000CBFA18B12046BDE834402CE0DFF8F80738
:10E9F0008569204600F0E4F9280ABDE8324000F0BD
:10EA0000010080F0010001F021B910B504464FF477
:10EA1000803100F015F80021204600F0ADFA18B161
:10EA20002046BDE810400EE0DFF8BC078069000A10
:10EA3000BDE8104000F0010080F0010001F0B3B823
:10EA400004F12000F9E401214FE710B5DFF8E418E4
:10EA500000228A7220220A6000F12801D0F8FC20EE
:10EA600090F85D40C2F303230A684968204490F897
:10EA70003600BDE8104001F020B870B50446210210
:10EA80000023012289B20520F8F7E0FDDFF858578E
:10EA900085F820400520F8F70BFE68602102F7F7A3
:10EAA000B9FD00204FF4807603E08B1833448B507F
:10EAB000401C0202631E69689842F6DB0020885001
:10EAC0006868A86070BD10B5DFF81C47E068B0B991
:10EAD0000220FDF73DF9E06002218172E068427A90
:10EAE000817A1044891A1030FBF766FBE068417A9E
:10EAF0000844012130F8102F61F30102028004F173
:10EB00001000FDF715FA1B2084F821001120207752
:10EB10000120E16960F30B210020E161206010BD5C
:10EB200038B5FBF7E3FADFF8C046A5680DB12968F0
:10EB3000A160FBF7DFFA0DB9002032BD4FF4807100
:10EB40002846F7F767FD05F165001B2141708170CC
:10EB50007F2101700320686100202862E069C5F808
:10EB6000FC00284632BD10B5044606F029FA04F12F
:10EB70007C00FDF7DDF904F18000FDF7D9F9A06F05
:10EB800018B1FDF73AF90020A067FBF7AFFADFF8FC
:10EB900058168A6822608C60FBF7ACFA002020626D
:10EBA00010BDF8B5044604F120054800298A002666
:10EBB00087B2B9421CBF28820126688A90421CBFD6
:10EBC0006A820126A88A98421CBFAB820126287857
:10EBD000000704F16C0705D5298A204600F0DBFA0E
:10EBE000B8603EB100F007F84FF080712046BDE8F4
:10EBF000F440AAE4F1BDA88A298A000190FBF1F053
:10EC00003880704730B5002100220125931002EBB7
:10EC10005373DB10C45CA2EBC30305FA03F31C427D
:10EC200004D0491C022901D1012030BD521C252AE3
:10EC3000ECDB002030BDF0B58AB000220025AC101E
:10EC400005EB5474E610012400F021F81CBF0DF808
:10EC50000250521C6D1C252DF1DB0025AE1005EB7A
:10EC60005676F61000F013F803D0461986F83650A1
:10EC700008E095FBF2F602FB165647191DF80660F0
:10EC800087F836606D1C252DE8DB0AB0F0BD8F5D7E
:10EC9000A5EBC60604FA06F6374270472DE9F047A1
:10ECA0001E46824630680AF104070D467862904697
:10ECB00006F110015046FFF7BEFF0322311D0AF195
:10ECC0002C00F7F7BBFB089906220AF15E00F7F764
:10ECD000B5FB099810B1042100F06EF8102100F086
:10ECE0006BF84FF480015046FFF72FFC717D0AF15D
:10ECF0005B0001F01F0101700AF16C047189490089
:10ED0000B98540F27129B189F985F1893986717D1A
:10ED1000490941700021398401217984717D01F014
:10ED20001F018170052020805046FFF7C3FD46205B
:10ED3000786030894000811C09FB0180386040F216
:10ED4000E2485DB1DFF8F015B961F17918FB01F126
:10ED500000EB510038604FF4487022E0504600F05C
:10ED60001AFA00F500753868A0EB15203860082104
:10ED7000DFF8C805B86100F01FF84FF4003100F06B
:10ED80001BF8F07918FB00F0690001EB00206060CF
:10ED90005046B98D00F0FFF9A0606068000A00F5E8
:10EDA0004870B8607089401E09FB00F0F86050465A
:10EDB000BDE8F04706F0F1BA0AF12000FFF73DBBCD
:10EDC00070B50646B06F38B9306AC00304D406F196
:10EDD0007C00FDF76EF9B067B56FDFF80C4405B93C
:10EDE000E568402106F12000FFF72FFBF06F00B12E
:10EDF00001206B7A316A2B4401F0010233F8106F65
:10EE0000490801F0010162F3820632461E8061F377
:10EE1000C30211461A8060F30411198028B103213E
:10EE200004F11800FFF705FB04E0032104F11800CA
:10EE3000FFF701FB2846BDE8704000F0C4BE2DE995
:10EE4000F0410D460446687ADFF89C83284408F1B7
:10EE5000140600F110073079400605D43868001F09
:10EE60003060062100F084F87068397931B9C00645
:10EE70004CBF0721042100F07BF85DE020F010007A
:10EE800070600321787984F86500B87A084253D01D
:10EE9000012100F06DF84FF48071FFF7D1FD788902
:10EEA000C0F3001018B1022100F062F804E0022162
:10EEB00008F11800FFF7BFFA216A7889490801F0C4
:10EEC0000101C0F3800081F00101884220D14FF49C
:10EED000003104F12000FFF7B8FA4FF4803104F15B
:10EEE0002000FFF7B2FAA06F60B18168C1F3800122
:10EEF00021B9B4F86A10491CA4F86A10FCF77DFF28
:10EF00000020A067206A80F002002062002001E05B
:10EF1000B07B401CB0737989206AC1F3C00100F056
:10EF20000102914208D180F001002062687A2844F1
:10EF300030F81A1F080A04D12846BDE8F041FCF752
:10EF40005CBF01F00300032806D14021FFF778FDE4
:10EF50004FF40031FFF774FDEC60294608F1100012
:10EF6000FDF7BAF8BDE8F0414FF00050FAF7E0BC09
:10EF700008F11800FFF75DBAF8B5DFF8B8530C4692
:10EF800029688A0625D411F4C07F26D1016ACE08EB
:10EF9000A97A032907DB84F0010106F001020A4285
:10EFA0001BD1114319D0D0F8FC002A2100F017F82A
:10EFB000074606F0CEF9B8420FD3287810F01C0FA0
:10EFC00007D106F00100204205D008212846FFF7AE
:10EFD00030FA0020F2BD204300D00120F2BDC0F382
:10EFE0000320FFF73ABA2DE9F04782B0FBF77EF82D
:10EFF0007D490A69009200220A61FBF77BF807E06D
:10F00000A06840F00400A0602146284605F002F9FF
:10F010000098002850D06846FDF74BF80446607A07
:10F02000E56821180C3001F11007B97A607201F01F
:10F030000306286A000405D532462146284600F01A
:10F040000AFF20B1032EDBD0286AC00407D5204672
:10F05000FCF7D3FE3D21284605F0FEFDD8E7A06869
:10F0600020F00400A06097F90500BE79A17A7F899D
:10F070005FFA80F8607AA1EB0009801F6072FFB22E
:10F08000C0B2204400F1100A2846FFF77BFA4CF684
:10F09000FF71084040EA0730C0F30D00AAF80200F3
:10F0A0008AF800805FFA89F0AAF804008AF8016003
:10F0B0002046FEF775FDABE7BDE8F387F8B50D46D2
:10F0C0000446A868C0F3800171B1687A216A2844B7
:10F0D00003261030090519D500781F2807DA98494A
:10F0E000C140C80712D402E0216A090508D5FAF721
:10F0F000FDFF0646294604F18000FCF7EDFF45E0E0
:10F10000C0F34000002814BF02260126206A4004F4
:10F1100004D532462946204600F071FEA87A697A65
:10F12000471A02212846FCF744FF687A284406F073
:10F13000030210F8101F01F0FC011143FFB241EA75
:10F1400007214FF61F7211400180FAF7CFFF0646E4
:10F15000294604F17C00FCF7BFFF94F8200000076B
:10F1600006D5E08C022811DB204600F079F80DE08E
:10F1700000F085FC61680D1A06F0C6F9A04205D1C1
:10F18000B5F57A7FC4BF2046FFF71AFE3046BDE8CA
:10F19000F240FAF7AFBF38B504460D4600F067FD00
:10F1A000684994F85C3051F8200051F8231040F27F
:10F1B00071226A43521C081801B0A0FB0201BDE88D
:10F1C0003040090241EA106100025F4A002302F068
:10F1D000EFB8054A1C2882F8210003DB0121104604
:10F1E000FFF72BB970470000C809002090F86600AF
:10F1F000704710B500F166031C788C4204BF5C7840
:10F20000944207D05A7019704FF00051BDE8104079
:10F21000FFF79BB910BD38B504460D46206A0003C0
:10F220000DD44FF400212046FFF736F9A4F86850BA
:10F230002046BDE834404FF08051FFF786B931BD1C
:10F24000C90744BF4FF48021FFF726B97047C907AB
:10F2500044BF4FF48021FFF721B97047FC3070475D
:10F260002DE9F8430446FAF741FF804600F007FC19
:10F27000261D3168081AB0F5FA7028D4B18D40F215
:10F28000712909FB01F1B0FBF1F5308CADB2401BE7
:10F29000308404F15B07B8783A78252105FB120029
:10F2A000FFF7E7F8B8700021B4F86C00401BA4F831
:10F2B0006C00204606F08DF8B18D3068694309FB7B
:10F2C00011003060204606F068F806F0E9F8404684
:10F2D000BDE8F243FAF70EBFF8B50446FAF706FFA9
:10F2E0000025002219490AE04B6803EB022393F83A
:10F2F0002030DB0644BF24F815206D1C521C91F809
:10F3000020309A42F0DB00220DE04B6834F81260A6
:10F3100003EB06235719B3F86A6024F81760521CF0
:10F320000026A3F86A60AA42EFDBFAF7E3FEE8B230
:10F33000F2BD0000E009002075E70000C9E7000009
:10F340007C2C0200C05A000040420F00C809002077
:10F3500010B504464FF4C051FFF7A0F803E0014692
:10F360002046FFF7ABFE04F18000FCF7A2FE002868
:10F37000F5D110BD026A120309D5B0F86800012268
:10F3800002FA01F1084018BF0120C0B27047012005
:10F390007047FEE70A431040884201D101207047C0
:10F3A00000207047F0B5DFF88C64341D0B2883B063
:10F3B00006F12C051FD8DFE800F0067D1B252D394E
:10F3C0007A7A7D7A7A23FF2086F82B0000F073F892
:10F3D000286800F0F8FBE0690C220021FFF7DAFF53
:10F3E000216803B0BDE8F04080F0010000F014BCDB
:10F3F00006F08AF8B0425DD1BDE8F74000F0E4BA0B
:10F4000000F0E2FA207D20283CBF401C2075BDE8BA
:10F41000F740ADE0207F10F0810F02D000F0D4FA69
:10F4200045E0BDE8FE40012000F0BDBB00F093FACE
:10F430000600F3D000F0BDF9032825D0052832D10D
:10F44000707AAF68304400F110040020A86000F02A
:10F45000BBFA012000F07BF8628920892168C2F3A1
:10F460008012019204F1180304F10C02009201EBE6
:10F47000C00200213846FFF711FC3046FCF7BDFC06
:10F48000BDE8F74006F00CB83046FCF7B6FCE06982
:10F4900040F08000E061686800F095FBBDE8FE4048
:10F4A000002000F0D3BB3046FCF7A7FCB6E7BDE870
:10F4B000F7401EE0F7BD10B5DFF87C03016821F0CE
:10F4C00080010160C17A4C1CC472E4B2032C01D1EA
:10F4D000002010BD817A0122A2401142F2D004F135
:10F4E00025000123D54AD649C0B200F0E6FA012032
:10F4F00010BD10B5FFF7DFFFCE4C68B1E06A00F039
:10F5000062FB206A0C220021FFF744FFBDE8104097
:10F5100080F0010000F06CBB206AC1050FD5218D81
:10F52000491E218589B251B920F4807020620120E2
:10F5300000F00DF805F0B4FFBDE81040B1E0207E0A
:10F54000112824BF401E2076BDE8104010E010B501
:10F55000B84C216A21F0100121620146204605F0D5
:10F5600038FF606B18B1FFF7FEFA0020606310BD32
:10F5700038B500F082FAC5B2AE4C0121204605F044
:10F5800028FF112295FBF2F202EB0212A18C6068B7
:10F59000AA1AD2B2511840F2712202FB0100606037
:10F5A000204605F0FAFEBDE8314005F079BF10B500
:10F5B000A048A44A00F1080100F12C044A6140F27D
:10F5C00053724A608A6050220A600222CA6018227E
:10F5D0000A744FF400628A83CA83072280F82A20C3
:10F5E0000020E0600C2088610220FCF7B1FB206065
:10F5F0000220FCF7ADFB606000220021002000F03B
:10F60000B3F8BDE81040002200210120ACE038B57D
:10F61000894C2378DB0601D5012032BDA2618A4DD9
:10F620002368AA5CA0801B090698A07242EA031214
:10F630002260E1804FF0FF32E068002100F069F8BD
:10F6400020694FF0FF32012100F063F8002032BD45
:10F65000F8B504460D461646FAF748FD0746200061
:10F6600018BF01203246294600F07EF83846BDE832
:10F67000F240FAF73FBD10B50446FAF737FD6D4981
:10F680000A6A0C8542F480720A62BDE81040FAF7FB
:10F6900031BD80B5FEF785F910B9BDE8024000E044
:10F6A00001BD4FF08050FAF743B938B5614C216A7B
:10F6B000CA0607D558BBFAF719FD05460020FFF723
:10F6C00046FF1FE018B3080705D5606B18B9FFF7B0
:10F6D00027FA6063E0B1206AA18C40F0100020623C
:10F6E000E08C401A40F2712148432061FAF7FEFC99
:10F6F000054600F0C4F9A16808186430606020462F
:10F7000005F04BFE05F0CCFE2846FAF7F3FC01208D
:10F7100032BD38B51446427A104400F11005454810
:10F72000002911BF04214949826B895C2A8802F4AF
:10F730007D5201F00F01114329804FF6BF72006A1C
:10F740008009114000F0010041EA80102880062263
:10F750003F49A81CF6F772FE002C04D42988A01D8E
:10F7600060F30D21298031BDF8B51546314A02EB11
:10F7700080070C460128F86A427A024402F110061A
:10F780000CBF012100212A46FFF7C3FFF86A328827
:10F79000417A120A02F03F025118891C81723CB171
:10F7A0002A46214606F10800BDE8F840F6F746BEB5
:10F7B000F1BD38B51F4CE16A4A7A1144427A831888
:10F7C00003F1100512312B79002B30D0AB79253B9A
:10F7D000032B2CD26B891B0A03F03F039A180C32BF
:10F7E0008272A87A00F00F00032818D194F8200044
:10F7F00040071CD50C2B1AD1062205F11200FAF78E
:10F80000ABFDA0B9E06A417A08446989008AC0F377
:10F810008010C1F3C011884209D1032032BD0528F0
:10F8200005D194F82000000701D5052032BD4FF026
:10F83000FF3032BD8C090020AC090020D6BE898E75
:10F8400055555500A5F30000945A00009C5A00003D
:10F85000E4070020890001EB401000F1085002602D
:10F8600070470122F6E70022F4E710B5044605F0E0
:10F8700083FE001BC00F80F0010010BD38B5DFF81B
:10F88000F45329788842044601D1002032BD20007B
:10F8900007D005F0F0FD01214FF0004006F096F989
:10F8A00004E006F0B9F9002005F0E5FD2C70012018
:10F8B00032BDDFF8C4130A7A52074CBF042200227B
:10F8C0000A6100684860042005F017BEDFF8A8232D
:10F8D00000211161800744BF082005F00EBE70476B
:10F8E00010B5DFF894130A7A92074CBF0322002266
:10F8F0000A61427A024452F8103F148903EBC403B0
:10F900004B6000F11003097B9171117901F0010145
:10F9100011710021417202F10A011289C91A5118AC
:10F9200081720520BDE8104005F0E7BDDFF84823EF
:10F93000002110F4407F116118BF0A2006D1C106D2
:10F9400048BF072002D4800602D5092005F0D5BDA6
:10F9500070477047704738B5C74C25680120FCF7E1
:10F96000F7F9206008B9256032BD284632BD10B5D0
:10F970000024C14A30B1022102F10800FFF771FFF3
:10F98000012404E0022102F10800FFF76CFF204689
:10F99000BDE81040002106F081BA10B50024B64A37
:10F9A00030B1012102F10800FFF75BFF022404E0FF
:10F9B000012102F10800FFF756FF2046BDE8104084
:10F9C0000122002106F07EBA80B5AB490020086113
:10F9D0000121022006F018FA0020FFF7C8FFBDE859
:10F9E00002400020D9E738B5A34C78B10088010067
:10F9F00008BF012009D0A1490A4600E0121D136882
:10FA00000BB19842FAD3501A801020759C4806F02A
:10FA1000E1F901214FF44C7006F06DFA994805F0B8
:10FA2000B2FD0546206818B90120FCF791F9206065
:10FA300006F078FAE8B232BD704780B5FFF7C4FF30
:10FA4000BDE802400020CEE78B4800687047704751
:10FA5000427A1044084410307047704738B5044665
:10FA60000D4606E0EDB22946204605F0A7FD044408
:10FA70002D1AE8B20028F5D131BD06F09DBA05F087
:10FA80007BBD0A46002808BF06F0C6B80021104614
:10FA900006F09CB805F03BBD70B5044676480D46AF
:10FAA00016460473447306F048FA22463146284647
:10FAB000BDE87040012306F061BA70B504460D46FA
:10FAC0006D4821460B2C16460473B8BF611C0DDB34
:10FAD000252CB8BFA11C09DB08BF002106D0262CAD
:10FAE00008BF0C2102D0272C18BFFF21012B417326
:10FAF00004D0022B08BF06F033FA01E006F01DFA2D
:10FB0000224631462846BDE87040002306F036BA4A
:10FB100070B500F03EF886B00D4605F02DFD281AB0
:10FB20003C2810DB3046FFF738FF58B900900295AB
:10FB30000120019069460020039001208DF81000FB
:10FB400000F02CF808B100F050F806B070BDF0B528
:10FB500000F01FF80F4685B0154607F13C00FFF78F
:10FB600084FE88B93046FFF718FF68B9A7F13C005A
:10FB700000900295002001900390694601208DF8C5
:10FB80001000002000F00AF808B100F02EF805B0CF
:10FB9000F0BD0646384C0120206170478DF81100F9
:10FBA000607B06F0AAB910B5044633480121016113
:10FBB00040688A30FFF759FE10B92046FFF7EDFE86
:10FBC00000B124E010BD00B583B0417A014410318A
:10FBD0000091817A407A081AADF80400684601F075
:10FBE00029FA08B100F001F807BD0B2005F085BC2B
:10FBF00010B5214C02212161FFF7B9FE20B9607BCD
:10FC00000022002101F01BFA00B100E010BDBDE8A8
:10FC100010400B2005F071BC7CB50446164E022046
:10FC200030610D4605F13C00FFF71FFE50B920463C
:10FC3000FFF79DFE30B9019000956A46707B12492E
:10FC400001F0FDF908B1FFF7D0FF73BD10B5044610
:10FC500009480221016140688C30FFF706FE10B9A7
:10FC60002046FFF784FE00B1D1E710BDF6E602485A
:10FC7000007D7047451400200C0B0020C05A000086
:10FC8000AC5A0000B85A0000ED5A0100002848BFE5
:10FC900001F0FAB9C0B201F0EEB970477047704791
:10FCA000854806F08FB970B588B00C46002104AEC7
:10FCB0004B42D5180344ED7B7554DB7B0DF80130C6
:10FCC000491C1029F4DB06F0E2F9802204A906F0B1
:10FCD000F7F906F0DCF96B466A46012106F001FAF5
:10FCE0000028F0D142420DEB0201C97B2154401C97
:10FCF0001028F7DB08B070BDF8B50C4615461E4657
:10FD0000FEF7C6FB074674B108222946F6F796FBB4
:10FD10000422314607F12500F6F790FB0422314614
:10FD200007F115000FE00822294607F10800F6F751
:10FD300085FB0422314607F12900F6F77FFB0422F8
:10FD4000314607F11900BDE8F840F6F777BB38B542
:10FD50000546FEF79DFB04464FF420512846FEF76A
:10FD60009BFB002044F8100F20712061207528466D
:10FD7000FEF790FB000702D58020207131BD802066
:10FD8000207531BD10B50446FFF7E2FA2046BDE804
:10FD900010404FF08061FEF7D8BB10B504464FF419
:10FDA0006041FEF77BFB2046BDE81040FFF7D0BA6C
:10FDB000F0B585B006460F46FEF76AFB0446FAF733
:10FDC00095F905464FF440413046FEF765FB4FF488
:10FDD00000513046FEF762FB3A4669462046FFF77F
:10FDE00062FF002042421DF800102244401C1028EF
:10FDF000D173F7DB2846FAF77DF905B0F0BDF0B511
:10FE000083B00C461546FEF743FB0646A07A617A9E
:10FE1000401A1FD0284F802332460221384606F070
:10FE2000E5F8A17A607A00956218103201922036C6
:10FE30000A1A204400F110013346384606F0F2F861
:10FE4000A07A001DA0723068401C306002D1307969
:10FE5000401C3071F7BDF0B583B00D461646FEF775
:10FE600017FB0446A87A697A411A052918DB001F96
:10FE7000A8728023104F22460221384606F0B6F8B9
:10FE8000A97A687A00966A181032019204F1100378
:10FE90000A1A284400F11001384606F0D3F808B1D8
:10FEA0000020FEBD2069401C206102D1207D401C45
:10FEB00020750120FEBD0000EC09002000B970474C
:10FEC00010B5046C230003D013460A460021A04756
:10FED00010BD00224FF00111F0E700224FF48031F5
:10FEE000ECE70A460849E9E768B1016419B1074936
:10FEF000074A084B01E00022002301614361002111
:10FF0000C26081604160704703000100DBFE0000B9
:10FF1000D3FE0000E3FE000010B50446F6F78EFAAB
:10FF2000204610BD890001EB401000F184400260C2
:10FF3000704710B5040030D00121354806F054F95F
:10FF400001213448F6F7C8FC334960684860F8225C
:10FF500032488260227A637C42EA0322637E42EA6C
:10FF6000034242602268CAB902220A600721016086
:10FF70000023217E6069042200F09EFC94F820108A
:10FF8000E0690023042200F097FC217CE068BDE8D2
:10FF900010400123042200F08FBC10BD012A03D1C0
:10FFA0000A6005210160E9E7022A04D105220A60FE
:10FFB00001210160E9E7032AE7D100220A6002601B
:10FFC00010BDF8B5164C144E25687068002748B16E
:10FFD0000F4806F01FF9716800EB5100B0FBF1F01B
:10FFE000401E070200F007F830680E492940084318
:10FFF00038432060F1BD0122FFE71E210A4891E746
:020000040001F9
:1000000009490968002944BF084908607047000091
:100010000034060000250800B808002074000840DD
:100020007C000840FC00FFFF94400840800008402E
:1000300080B5012A03D100F02FF8012002BD002075
:1000400002BD38B504461D4D1D4900222846F9F76A
:100050006FFF74B1002004F027F8044606F042F95F
:10006000E061C4612846BDE8384000220121F9F76B
:1000700059BF012004F018F8124C13490022204601
:10008000F9F756FF002203212046F9F74BFFBDE8A0
:1000900032400120F9F743BE10B50C4C102200216C
:1000A0002046F7F771FB2046FAF728F8BDE8104024
:1000B000002205490348F9F73BBF0000D0080020A3
:1000C0003100010098080020E7000100C00800206E
:1000D00038B504460D462278611C2846FFF71CFF00
:1000E0002078286131BD2DE9F84317461C4606F0FB
:1000F00077F9DFF89455DFF89485D5F800C0DFF87C
:100100009065FF1E3CD07F1E5BD0FF1F00F0FF807C
:10011000FC3F00F0B2807F1E00F0F2807F1E00F0F6
:10012000CB80F83F56D0BF1E64D0FF1E00F07E800B
:100130007F1E00F0DC80FB3F14D040F2FF403F1AEE
:1001400000F023817F1E00F0FC807F1E00F0028102
:100150007F1E00F009817F1E00F00C813F1F00F020
:1001600023812CE12068B0800023A088F080002249
:10017000DFF8200530603146012000900820C4E0FF
:1001800006F0ADFC40B10120706000234FF4946094
:1001900000F044F9082010E10220B0800023012083
:1001A000F0803081002240F29B6070813146002057
:1001B000B0810120F081DFF8E00400F00DF910209B
:1001C000FBE02068B0800023DFF8D00400F026F9BF
:1001D00006209AE000F01CF9070026D02068C069CC
:1001E00010281FD06068B080002397F83E0000F010
:1001F000FEF817E000F00CF9070016D007F120090F
:10020000D9F81000802810D16068B080002399F8D8
:100210001E0000F0ECF8D9F80000C0B201F026FA98
:10022000F9F7A8FF3846F8F74DFEC8E0206890F8C7
:100230002C0006F0D9FD0700F7D0206800F114016A
:100240000622301DFFF768FE2068C069B072314693
:100250002068C06B012818BF0020F072002397F8B7
:100260003E0030730022206890F854007073DFF86D
:10027000300400F0B1F80E209FE0207830710622A3
:1002800060787071A11CB01DFFF746FE207A3073B4
:1002900004F10B03607A7073A07AB0730B30010223
:1002A00041EA102040F4403040F0A00000F094F803
:1002B0003146B27B0F2080E000F08AF8002819D088
:1002C00090F83E00307100236088A6F805000022F7
:1002D000A088A6F807003146E088A6F80900207A31
:1002E000F072DFF8C00300F077F80C2065E000F052
:1002F0006FF8002863D000F065F8DFF8AC0359E030
:10030000DFF8A80300F07DF80420E04757E000F094
:100310005FF8070053D0207801F0A8F900281CBF2F
:10032000C06910284BD097F83E00307100236078E8
:1003300070710022A078B0713146DFF8740330602C
:100340002EE000F045F8002839D000F03BF8DFF847
:1003500064032FE000F068F830710023DFF85803E1
:1003600000F05CF8052028E000F05EF800F038F8B6
:10037000D24804E000F058F800F032F8D04830607D
:10038000314601200090092017E000F04DF830714F
:1003900000236068A6F805000022CA483060314694
:1003A00001200090072008E000F03EF830716068FE
:1003B0007071C54800F025F806202C68A047002081
:1003C000BDE8F28390F83E0030716078707170473C
:1003D00021788020F8F760BE3060012000907047DF
:1003E000307100236068C6F8050000227047B071C4
:1003F000C6F800800120009000222C6831460720BA
:1004000020473060002301200090002231467047D1
:10041000206890F82C108020F8F73EBE3060002253
:100420000120009031467047207806F002BD80B56B
:1004300006F098FD06F0C8FDBDE8014006F0EEBEEE
:10044000704710B5044682B0207806F000FDFF2802
:1004500008BF4FF4C0700AD0B4F807100091B4F888
:100460000530B4F80320B4F8011002F0E7F900F009
:1004700034F8964829E010B582B00078844C06F034
:10048000E6FCF9F785FEA080214691482060012016
:100490007D4C24680090002300221BE010B5044628
:1004A00082B0207806F0D3FCFF2808BF4FF4C0705C
:1004B00008D0617819B1012102F04CFA02E0012163
:1004C00002F054FA00F009F8824808600120009018
:1004D000002224680620A04713BD6D496A4C88801D
:1004E0000023704710B5044682B0207806F0AFFCB8
:1004F000FF280EBF4FF4C070617802F046FAFFF794
:10050000ECFF7548E1E7F0B5044683B000F096F8DB
:10051000050008BF4FF4C07037D005F12406307EC7
:1005200040071BD53768CFB100E007463868002880
:10053000FBD1B87A6278C0F1450191420EDB3844B4
:10054000A11C1030FFF7E8FCB87A61780818B8727F
:100550006178306940183061002016E02846F8F7CD
:10056000C3FC10B94FF4C7700FE06178A01CFBF713
:1005700079FB019020B101A92846F8F734FD20B19C
:100580000198FBF73AFC4FF4C17000F04FF8534864
:1005900000F025F8F7BD38B5044600F04FF80546E1
:1005A0006078F8F786FD002D14BF00284FF4C07264
:1005B0000AD0E9690022814206D0E86195F83C0042
:1005C00040F0010085F83C00002331498A80002278
:1005D00020782D4C8871424800F001F831BD086048
:1005E0000120009007202468204710B5044682B0FF
:1005F00000F024F810B94FF4C07011E000F12001B0
:100600000A7FD20609D40A69802A06D10868C0B2D6
:1006100001F02CF8F9F7AEFD01E0F8F753FC0020EB
:1006200000F004F82F48FFF7DAFF13BD184988805F
:1006300000232078144C8871002270472078F8F746
:1006400038BD7047704770B5044682B0FFF7F6FFBB
:100650000025002600280E490FBF4FF4C070856B9F
:10066000466B0020888000232078074C8871C1F8F1
:100670000760C1F80B5000221B4808600120009061
:100680000F202468A04773BD50050020A003080177
:10069000FC070020A0040E00A00C0100A002010530
:1006A000A00A0800A0080802A0020804A000030194
:1006B000A0030803A0020F03A0010F01A0050F0073
:1006C000A0050F02A0030F04A0020F0920020800DA
:1006D00020020801200208022002080320030B0068
:1006E00020030B0120030B02200B0B0549010028FE
:1006F00006D5054A00F00F00104400F8041C7047AE
:10070000024A11547047000018ED00E000E400E0D8
:1007100080B504210B20FFF7E9FF04210C20FFF72F
:10072000E5FF04211320FFF7E1FF04211420FFF768
:10073000DDFF04211520FFF7D9FF04210D20FFF76D
:10074000D5FF04211620FFF7D1FF04210E20FFF76B
:10075000CDFF04211020FFF7C9FF04210920FFF776
:10076000C5FF04211120FFF7C1FF04210A20FFF774
:10077000BDFF04211220FFF7B9FF04211820FFF765
:10078000B5FF04211A20FFF7B1FF01211D20FFF75B
:10079000ADFF04211720FFF7A9FF01210120FFF77A
:1007A000A5FF01210320FFF7A1FF01210420FFF78E
:1007B0009DFF01210520FFF799FF01210620FFF78A
:1007C00095FF01210720FFF791FF01211B20FFF773
:1007D0008DFF01211C20FFF789FFBDE804400221A5
:1007E0006FF0010082E7FEE780B501211C48F6F7B3
:1007F00073F81C4806F049FE1B484FF0FF31416377
:1008000040F2FF7101604168C90AC90241600120DC
:10081000164906F023FE16494FF0005008601549AE
:10082000086000201449086001BD14480168CA0727
:1008300003D5114A13685B1C13608160704710B5C3
:100840000D490A680E4B1B680C68A242F9D1D1030E
:1008500041EAD3310160C3F30E01818010BD000075
:1008600080091200445A0000202004405C5A000015
:1008700080E200E000E100E0D808002018200440F9
:1008800008200440890001EB401000F18440026020
:10089000704710B53024224B6043BDE81040184427
:1008A000002207E010B530241D4B6043BDE8104026
:1008B000184401220C30E5E7F8B5160004460D4651
:1008C0001F4605D017B1FFF7EDFF01E0FFF7E1FF8D
:1008D00030211348614308440F21082D05D2AA0096
:1008E000436800F015F8416006E0A5F108029200A7
:1008F000836800F00DF881604EB9002F294620462C
:1009000002D0BDE8F440CDE7BDE8F440C1E7F1BD59
:10091000914023EA010106FA02F2114370470000F8
:1009200000A00040890001EB401000F1844002600B
:10093000704710B504003BD006F008FFDFF87005E3
:100940000021002200230EC02068DFF8681502286D
:100950001BD1086880022BD410222146DFF85805ED
:10096000F5F76CFDA08900F0FCF900F030F8B4F95F
:10097000080000F024F8DFF844050168C908C90040
:10098000016000F073FA012010BD012804D108684D
:1009900010F4400F0CD1DFE7DFF824050068096888
:1009A00000F0010080F0010001F480010843D3D081
:1009B000002010BDDFF80C05B0F90C00704780B5C1
:1009C00000F02AF9DFF8FC04B0F90C0002BDDFF8F2
:1009D000F4044068022808BF00F053B8012808BF9B
:1009E00000F028B8DFF8C814DFF8DC2408681040ED
:1009F0000860DFF8D8040268D208D20002600A68F2
:100A000042F0804242F014020A60016841F00401A1
:100A10000160C168C908C900C160C16841F0050131
:100A2000C160816821F0C0018160816841F081016D
:100A300081607047DFF87814DFF88C240868104074
:100A40000860DFF888040268D208D20002600A68F1
:100A500042F003020A600168DFF8742441F00301E8
:100A60000160C168C908C900C160C16841F00601E0
:100A7000C160816811408160416821F4404141605A
:100A80007047DFF82C04DFF8402401681140016052
:100A900041F0804141F020010160DFF838044168F5
:100AA00021F4EE414160416841F48A4141600168AE
:100AB00041F001010160704730B5DFF8F413DFF851
:100AC0001C340A681A400A60C0F3431342F47C5293
:100AD00042F0C8020A6000F01F04C01300F00102D7
:100AE000DFF8D0030068C04300F4FE10B0FA80F0D5
:100AF000C0F1130098423CBF03461F240BB90123E9
:100B000000E004B9012401259D406D1E0868AD0375
:100B100005F47F1528430860002A086840EA04604D
:100B2000086044EA4310DFF8B8130A6805D042F4BD
:100B300080020A6040F4004030BD22F480020A6066
:100B400030BDB1F900208242B8BF1046A0F1C80202
:100B50006FF0270392FBF3F2082AA8BF072201EBEC
:100B6000C201091D01284B68B1F9021000FB0131D7
:100B7000A8BF01F5FA714FF47A70B1FBF0F0072AC3
:100B80001FBFDFF840134968022940F40040704756
:100B9000012231F83230834202D3521C082AF8D3A2
:100BA000521E01EBC20120F400404FF47A72504310
:100BB0004A68B1F90210801A0128A8BF00F5FA703E
:100BC00090FBF1F0704710B5B94AC64B1168194057
:100BD000116083281368C2490EDA1C0A04F47F549A
:100BE00023431F2813600CDA0A68520852000A6077
:100BF0008A69520852000BE043F47C5343F0C80367
:100C000013600A6842F001020A608A6942F0010238
:100C10008A61BDE810403CE038B5AA4CB4F90E102A
:100C200040186168012917D1A149AB4B0A681A40E5
:100C30000A6006220FF2EC3333F91250A84201DAAF
:100C4000521EF9D133F912500868521C40EA026072
:100C500008600868606115E0A26801B1921C442335
:100C60000FF2B0215A438D182946FFF76AFFFFF7AC
:100C700023FF212808BFB5F9025003D0291DFFF733
:100C800087FF05462846FFF79EFFE089281AA081C6
:100C900031BD38B58B4C227801469348CAB17929C9
:100CA00017DB026F914B1A4002679339904A15681F
:100CB0002B401360052391FBF3F109318900036F89
:100CC00041F457410B430367136819431160012234
:100CD00000E000220321FFF725FE754908686061E6
:100CE00031BD38B57248794D0168490801F4FE14E8
:100CF000016821F47F1101602143016007F0C0F811
:100D000028B1286820F47F102043286004E0A869F7
:100D100020F47F102043A8614FF0007075490860EF
:100D200031BD68496248496901607348016821F032
:100D300080610160704738B507F0A2F86F4C634DD1
:100D400018B128682040286002E0A8692040A86106
:100D50006948016821F00061016031BD5948008A8D
:100D600070477CB5574C06466068022808BF962538
:100D700003D001280CBF3225B425E6B1F6F74CFDAF
:100D80004FF47A71B0FBF1F07043B0FBF5F0400125
:100D9000B0FBF1F04FF0FF3101E04008491C0028A2
:100DA000FBD149B21029A8BF4FF4706005DA0029C1
:100DB00058BF080201D54FF480700FF25011D1E9ED
:100DC0000023CDE90023009028040190684600F03C
:100DD00010F800F01AF80546F6F71EFD6421B0FB86
:100DE000F1F042F210716943B1FBF0F02082208AE9
:100DF00076BD434942684A600A68120B12030A60D2
:100E00000A68006810430860704730B53C494A687A
:100E100048684B680C680D68D2B2000404F00F04F7
:100E2000000E096802FA04F4821AC5F303151B02C6
:100E3000AA401B0E090A5211181A01F00F0102EB09
:100E40006412884002EB601030BD03012D4A03F4A8
:100E5000F87300F00700184310600A012A4802F4F2
:100E6000F87201F0070111430160704780B506F088
:100E7000F6FF401E06D0801E01280CD9801E0128D6
:100E80000CD90EE00F484068012819BF042100204A
:100E90000421042007E00021002004E003210320B6
:100EA00001E00A210F20BDE80440CEE70000000069
:100EB000E80F002188410E403400002058410840CE
:100EC000D481E00F30000020E8FFFFBF0041084060
:100ED0003EFFBFFF204108403F00C0E0FF3FC0E0B1
:100EE0000841084037C0FFFF944008408220FFFFC0
:100EF0001C4108401C40084020400840FFFFDF7FA5
:100F000068600840F00F0021EC0F00210000000095
:100F100000000000C800FCFE1F811D0B6ABDFBFF26
:100F2000B0807F054A32FFFF74801603EA4B000051
:100F30005180B50127B200003F80490184C50000FF
:100F40003280D100F0C300002880740034B4000067
:100F500028004B00EAB500008C00FCFEFFFF0000FB
:100F6000000000001F8158114C42FAFFA180CA0501
:100F70000197FFFF5D806A024CA400004180570189
:100F8000A7CC00003480E000BECA00002A808C009C
:100F9000CABC000029005200B5B90000C800FCFE20
:100FA0001F01C80B7D30FBFFAB001C05035BFFFF7F
:100FB0007300FD02DC5500005300D501BEAF0000F8
:100FC0003F001901E4C800003300AC0090C70000E6
:100FD0002C006C00B1BC00002700430046AF0000AD
:100FE0009600FCFEFFFF0000000000001F016D0FD7
:100FF000A182FAFF7E00C103791F00005500E401C1
:10100000F4B1000041003701C7C900003300C0003F
:10101000CAC700002B006E00F7B900002600380098
:101020008AA8000083FFBFFFE2FFF1FFF9FFFEFF88
:101030000000000080B504F015FDC0B202BD1346EB
:101040000A460021F8B504460D4616461F4604F030
:10105000D1FC08B90220F2BD204604F0E4FE08B13C
:10106000C0B2F2BD3B4632462946204601B0BDE83B
:10107000F04004F047BD10B504F0D5FE040008BFF1
:1010800004F012FEE0B210BD80B5FFE704F005FEEB
:10109000002002BD04F0F0BD012100F01F029140CC
:1010A000DFF8C822400942F820107047890001EBA0
:1010B000401000F184400260704738B5DFF8B0524C
:1010C0000121284605F090F8DFF8A842DFF8A802D1
:1010D0002060284605F09EF84FF47A71B0FBF1F0DD
:1010E000400200F5FA70B0FBF1F0A0F58071090A3A
:1010F000C0B240EA0120A0624FF0FF3000F011F9C9
:10110000401E206331BD80B51C20FFF7C5FFDFF80E
:101110006C124FF0805008600122BDE808400021A9
:101120000CE080B51C20FFF7B7FFDFF854124FF03A
:10113000805008600122BDE8084002219148B5E7CF
:101140009148006871E09148002101604160816030
:1011500070478F4A13680A1A3CBF581C8218104601
:10116000704710B504468B480022002100EB0410A4
:10117000FFF79CFF4FF480708749A040086010BDC6
:101180002DE9F84F054616460C4602F061FF8046F1
:101190002846FFF7E6FF0027012EDFF8009224D152
:1011A000D9F80000401C0419D9F818A0A2453CBF8A
:1011B000A4EB0A00441E280176490A18D4601122C3
:1011C0000A502046D9F800B05946FFF7C2FF4FEA4F
:1011D0009A0181420CD3D9F848004FF48071A9409C
:1011E0000840401E8041C00F03E0022EDCD10CE01D
:1011F00000207F1C012E07EB0B0409D1062F07D21C
:101200000028D8D1404602F027FF0120BDE8F28F28
:101210000028F7D02846FFF7A4FF404602F01CFF45
:101220000020F3E75B490001085800F00100704717
:1012300001F46001574A000141F003011150704769
:10124000F8B504460D46164606F09EFC00F069F817
:1012500007462046FFF785FF012E03D1BD4238BF68
:10126000002100D3E91B04F1090000024C4A40F0C0
:101270000100106032462046BDE8F84080E748494A
:1012800000200860704770B500F028F806F0F5FC03
:1012900000F047F8012E03D1854238BF002100D36A
:1012A000291A04F1090000023E4A40F001101060C2
:1012B00032460FE070B500F011F83A483A4A01683A
:1012C000114004F1090241EA026141F480310160F8
:1012D000324629462046BDE8704051E704460D4697
:1012E00016463EE72F493148086070472B48006892
:1012F0007047284901EB0010C068704780B5222074
:10130000FEF77EFEBDE808400122122116E71E48C6
:10131000006810F0060018BF01207047C10F4000A0
:10132000704700F0010101EB500070472DE9F843D0
:10133000154CE568FFF7F5FF0646606A4708206828
:10134000C00701D40FE0361AB046BE4288BFB84687
:10135000D4F80C9049462846FFF7FBFE4045F7D3EA
:10136000B0424D46EFD3BDE8F183000080E200E0DB
:1013700000040600005008400011010000E100E0F8
:1013800080E100E0045008400C5008401050084034
:1013900030500840745008406450084018500840CD
:1013A000705008406C500840FFFFE0E00000010171
:1013B0001B4213D1094236D12AB18446B0FBF2F068
:1013C00002FB10C2704706F081BEFCD3002200234E
:1013D00070470B000200002100207047904271EB23
:1013E000030CF6D370B5B1FA81F4B3FA83F52C1B74
:1013F000A340C4F1200532FA05F63343A2405FF062
:101400000046E64002E05B085FEA3202841A71EBB4
:10141000030524BF204629467641F4D302000B0081
:101420003000002170BD012ACFD970B5140C20D036
:10143000B1FA81F4B2FA82F5C4F120046419B4F16E
:101440002006D6D3B2405FF00044F440002502E00D
:1014500052085FEA3303C61A71EB020E24BF30460E
:10146000714664416D41F3D302000B002000290056
:1014700070BD0C46B1FBF2F102FB11452D0445EAAB
:101480001045B5FBF2F402FB145580B240EA054565
:10149000B5FBF2F002FB105240EA044070BDFEE7DB
:1014A0001B4901200860704730B51A481A4B016883
:1014B0000020002203EBC204184D64682D686D07FC
:1014C0000FD453F83250B5F5007F18BFB5F5806FD3
:1014D00005D0B5F5006F18BFB5F5803F01D144F4D4
:1014E00080740F4D2D68ED0553F8325048BF24F03D
:1014F0001C04294202D0214208BF2843521C092A59
:10150000D8D3C10348BF20F01C0030BD000000004C
:1015100008500E4004500E40FC590000E841E00F16
:1015200088300E40014800210170704746140020A9
:101530007047FEE770B505460E460220F6F7B8F88C
:10154000040028D06821F8F737FEE6610622294614
:1015500004F11400F4F772FF4FF0FF3084F85400E8
:1015600000206349401C0A68C0B204E092F82C30A5
:101570009842F7D09268002AF8D104F12C0210703A
:1015800040F6FF705080002050610868A0600C6039
:10159000204600F0AFF8204670BD00B1C18570470D
:1015A00010B504003ED094F904000128A4BF401EE9
:1015B000207194F90400012809D1207B800706D509
:1015C000206900281EBF0128204600F0C3FB94F9C3
:1015D0000400012826DA204600F097FB04F13000D1
:1015E000FAF7A6FC04F14C00FAF7A2FC404908689F
:1015F00058B1844203D1A068086006E008468168BB
:1016000019B1A142FAD1A168816000220FF219013B
:101610002046F8F78DFC2046BDE81040002201214D
:10162000F8F780BC10BD000010B5012A0C4602D0AE
:10163000022A07D004E0002202212046F8F772FCBB
:10164000002010BD2046F8F7A2FC21460220F6F744
:1016500040F8012010BD2649096800E0896800298A
:101660001CBFCA8D8242F9D10846704720490968DB
:1016700000E0896800291CBF91F82C208242F8D133
:101680000846704770B50446194806680D4600E0E4
:10169000B66856B1F069A842FAD10622214606F191
:1016A0001400F8F759FE0028F2D1304670BD38B565
:1016B00004460F48056800E0AD685DB1286904285C
:1016C000FAD13CB10322214605F11700F8F744FE98
:1016D0000028F1D1284632BD10B90548006870478E
:1016E00080687047024900200860704700000000D1
:1016F000DC08002010B10179491C01717047FEE738
:101700000188491C8AB202B9012101800088704712
:1017100010B50446012000F0ECFADFF8B8080460C8
:101720000020BDE81040E4E2DFF8A80800210160D5
:10173000C1610162C16281624FF6FF7101870021C0
:1017400081608181016181827047DFF88818C278E9
:101750004A6042F2130382889A4200D0704700B573
:1017600083B082788DF802208088ADF8040001F102
:101770003800FFF7C5FFADF800006A460621DFF824
:101780005808F8F71CFC07BD70B505468CB0DFF8AB
:101790004468A878DFF840487060B5F80300103856
:1017A00039D04FF47E71401A35D040F2FB71401AA7
:1017B00031D040F2FE31401A16D0001F26D0001F53
:1017C0002AD04FF47F71401A5CD040F6FD31401AA8
:1017D00000F07E800C381ED0093842D0401E2FD039
:1017E000401F02285FD978E00A20F5F7AEFFB5F870
:1017F000071041800246A9790170697A0171A989AF
:1018000001816989C1804FF4837115E0B5F8090041
:10181000B060E888B0817FE00622A91D06F13000A3
:10182000F4F70CFE0620F5F790FF06460622A91DE8
:10183000F4F704FE324608212046F8F773FB6BE00C
:1018400008208DF80E000822A91D0DF10F00F4F7F5
:10185000F5FD00F063F8ADF80C0003AA40F60801AE
:1018600057E010208DF81A001022A91D0DF11B0061
:10187000F4F7E4FD00F052F8ADF8180006AA40F6BF
:10188000070146E068798DF80900E888FFF7E3FE74
:1018900008B190F82C008DF8080002AA287A8DF87B
:1018A0000A000B2135E06879010014BF40F4007094
:1018B0000020009042F21F01B5F8030088420CBFDF
:1018C000E8880020ADF804006A4640F2023120E0CA
:1018D000287A3061E888B0821EE068798DF80200CD
:1018E00040F66D41B5F80300ADF80400B5F803000B
:1018F000401A06D041F29931401A02D0801E0428C5
:1019000002D800F00BF800E0308FADF800006A4616
:1019100006212046F8F753FB0CB070BD06F13800E5
:10192000EEE68078002808BF01F009B870472DE97D
:10193000F8460446A07801286AD002280BD0032874
:1019400051D0052800F09F80062800F0A9800C28BF
:1019500000F0B480BCE0E5784FF0000A11E000F040
:10196000B9F85FFA80F9FFB2AF42F8DB0AEB090081
:1019700020440AF1010A90F904003070304600F06A
:1019800000FFAA45E6DA2A20F5F7DFFE0600E1D0DF
:1019900004EB0A0006220079707000270AEB0500AC
:1019A000204400793072680002FB0A002044011DC7
:1019B000B01CF4F743FD0AEBC50020440079B07277
:1019C00005EBC50001E000F085F85FFA80F9FFB291
:1019D0005745F8DB04EB0900B27A011D06F10B0054
:1019E000F4F72CFDBFE7A088FFF735FE05006FD0A8
:1019F000E07800286CD105F16000E1880180618900
:101A00004180218981802846BDE8F24600F03CBE35
:101A1000A079E179002808D101B1012104F1080081
:101A2000FFF730FE05000CD152E004F10800FFF78B
:101A300081FD05004CD00220E86300F0C4FA0020CC
:101A4000A862E07878B9A1882846FFF7A6FD05F1DD
:101A50006000E1890180618A4180218A8180284675
:101A6000BDE8F446C1E000202861E078010014BF21
:101A700040F400710021284601F026F92846BDE80F
:101A8000F246FFF78DBDB4F80300FFF7E4FD050053
:101A90001ED0B4F80D10621DBDE8F84606F056BF22
:101AA000B4F80B000090B4F80930B4F80720B4F88B
:101AB0000510B4F8030000F0ECFB09E0A088FFF784
:101AC000CAFD050004D0A179BDE8F44600F0FBBDD5
:101AD000BDE8F18607EBC50020447F1C007948442F
:101AE000704738B505462878032848D0052833D0F4
:101AF000082817D00E2808D00F280AD030280CD07C
:101B00003E2869D0FF2863D031BD2846BDE8324069
:101B10003AE62846BDE8324017E600F062F80400D5
:101B20005ED00EE000F05DF8040059D0697994F8B9
:101B30004500002914BF40F0010000F0FE0084F8C9
:101B40004500A878010014BF40F400710021204630
:101B5000BDE8344001F00DB900F043F804003FD077
:101B60000020206140F6FF70E0856879010014BF15
:101B700040F400710021204601F091F823E010218B
:101B8000681DFFF77FFD04002AD0A87880B9B5F85A
:101B900003102046FFF701FDE87A28B194F84500CC
:101BA00040F0010084F845002046BDE834401CE0C8
:101BB00000202061A878010014BF40F400710021CA
:101BC000204601F081F82046BDE83240FFF7E8BC2E
:101BD0002846BDE83240A4E62846BDE83240A6E6E5
:101BE00031BDB5F80300FFF736BD002101F06CB838
:101BF0000146DFF8E803FAF76FBADFF8D803C169E6
:101C0000002906BF806A002801207047DFF8C4134E
:101C1000CA69002022B110461268CA610021016021
:101C2000704710B509F094F8040008D004F11000D2
:101C3000FFF757FF2046BDE8104009F06AB8FFF7EC
:101C4000E5FF18B1BDE8104000F054BC10BD80B5F0
:101C500009F054F818B141F2090100F013BB6AE22F
:101C600080B510B102281AD001BD182009F050F833
:101C700088B142F2240101822A22042100F0FEFAF6
:101C80000A804FF6FF724A8004F084FBBDE80240F0
:101C900002202EE001BDBDE80240012038E509F038
:101CA00057F80028F6D0017C0E29F3D1817CDFF8AB
:101CB000242301295160EDDB09F02BF8EBE710B18B
:101CC000022801D07047C2E722E580B510B1022892
:101CD0000CD001BD00220321DFF8FC02F8F722F945
:101CE000DFF8FC1209680120887301BDBDE80140DE
:101CF00097E7DFF8E022DFF8EC12126851F82210C3
:101D000008470220F5E70020F3E7F8B5B14D044697
:101D1000A88A00280CBF05F1200605F1240603E07F
:101D20000768FAF76AF83760306820B1C168A142E5
:101D3000F6D00646F8E794F83900A98A19B129695E
:101D40004018286102E0A9684018A860002084F8C3
:101D50003900F1BD10B504462069002818BF0128DC
:101D600002D140F2811010BD032802D100F040F9E9
:101D70000AE000F0D6F938B140F2064100F008F868
:101D800013228A7004F006FB01202061002010BDA0
:101D900001820321817400F11301E28D0A807047F2
:101DA00032B504460120E18D40F6FF72914207D121
:101DB0006846FAF7BDF831BDFAF78EF900950020B4
:101DC0000099A9B10D68009A002111600099CC60BA
:101DD0000099896821F0020141EA40000099886079
:101DE0007C48818A0029009914BF24302030E3E721
:101DF00004F090FA31BDBDE8024004F0CBBA2DE901
:101E0000F8430746884616469946232008F080FF87
:101E10000024050006D042F20600288205F11304D2
:101E20000F20A8742780A4F80280267184F80590FA
:101E3000012E0898A07118BF032E04D1099906221B
:101E4000E01DF4F7FBFA0A9860730B98A07328461C
:101E500004F0A0FABDE8F2436DE070B500F011F8AF
:101E6000060002D042F2080055E0002070BD70B5B7
:101E700000F007F8060002D042F209004BE0002013
:101E800070BD04460D46342008F042BF38B5044604
:101E9000152008F03DFF002530B142F20A01018211
:101EA00000F11305012181742C7004F073FABDE870
:101EB000324040E02DE9F04104460D4690461F4671
:101EC0001B2008F025FF002630B142F20B010182F1
:101ED00000F11306072181743470A6F80150A6F8AA
:101EE000038077710699B17104F054FABDE8F041AE
:101EF00021E070B504460D46162008F009FF0026C3
:101F000030B142F20C01018200F11306022181740A
:101F1000347075700BE030821F222020B074294687
:101F200006F1130000F8014BF4F788FA304604F08C
:101F300031FABDE870402D48FFF7E2BB2DE9F843C8
:101F400005460320286188461446994600F03BF870
:101F50000020A8620120E8630A9A09992846F7F749
:101F6000E7FF2D2008F0D4FE060028D042F20D0035
:101F7000308206F113071920B0740622C820388079
:101F8000788005F1140100203871E8697871B81D76
:101F9000F4F754FA00203873A7F80D80A7F80F4023
:101FA000A7F811900898A7F81300A7F81740002089
:101FB000A7F81500304604F0EDF9002001E04FF4D9
:101FC000C170BDE8F2830622074905F12000F4F74D
:101FD00045BA0000800B0020980800209C0B0020D0
:101FE0009C080020045B0000B00B0020B60B002012
:101FF00080B508F083FE18B142F20E0100F001F83E
:10200000F9E60182002181747047BDE8F24004F0D6
:10201000C1B9F8B500F05EF950B142F2130100F019
:1020200047F9E18D118000F049F9BDE8F24082E7FF
:10203000F2BD018200F113050221817470472DE980
:10204000F8430446884615469946302008F060FE5D
:10205000070019D042F21900388207F113061C203C
:10206000B8740822E08D30804146B01CF4F7E6F9E0
:1020700075811022494606F10C00F4F7DFF9384665
:1020800004F088F9002001E04FF4C170BDE8F2834C
:10209000F8B50D0004460BD1162008F039FE0025D6
:1020A00018B142F21B01FFF7C4FFE18D298014E053
:1020B000262008F02DFE0026070006D042F21A0066
:1020C000388207F113061220B8741022E08D308098
:1020D0002946B01CF4F7B2F9384696E710B5044625
:1020E000152008F015FE28B142F21D010182C474CA
:1020F000012189E06DE070B504460D46164600F0FA
:1021000010F858B142F21E01018200F0B6F80C70CE
:102110004D708E7004F03EF9002070BD4FF4C17018
:1021200070BD172008F0F4BD80B508F0E7FD10B1D0
:1021300042F21F01A6E04FF4C17002BDF8B504469B
:102140000D4616461F461A2008F0E2FD88B142F2FD
:102150003201018200F1130206218174E18D1180A8
:102160009570D67017710699517104F013F900201B
:10217000F2BD4FF4C170F2BD80B508F0BFFD40B1B3
:1021800042F21801FFF73DFF04F004F9BDE80240F8
:10219000D1E602BDF8B5FFF774FE060017D042F293
:1021A0001700308206F113072020B0741022214658
:1021B00007F11000F4F742F9102229463846F4F7E7
:1021C0003DF9304604F0E6F8BDE8F240B3E6002001
:1021D000F2BD4FF4C17010BD10B500F005F810B19C
:1021E00041F205410CE0F4E70446162008F090BDEA
:1021F00010B5FFF7F9FF10B14FF6044100E0E8E732
:102200000182A0F813400221817404F0C3F8002079
:1022100010BD38B500F00FF810B14FF605410FE0D2
:102220004FF4C17032BD38B500F005F810B14FF66B
:10223000064105E0F4E704460D461A2008F068BDA3
:102240000182062100F01AF80C80C1F8025004F057
:10225000A1F8002032BD38B504460D46192008F01B
:1022600057FD48B14FF607410182052100F006F8FD
:102270000C70C1F80150EAE7D2E70321817400F144
:102280001301704701820021817404F083F800205B
:1022900002BDF8B500F01EF848B142F2200100F08E
:1022A00007F8148000F00AF8BDE8F24043E6F2BDFA
:1022B000018200F113020E218174704755809680CF
:1022C000D78006991181002151814FF6FF719181CC
:1022D00004F060B804460D4616461F46222008F05A
:1022E00017BDFEE7427A8A184272827A8918817293
:1022F0007047002105E0827A5118427A0068891AF5
:10230000C9B20028F7D10846704780B500220FF205
:102310003511DFF8D801F7F70BFEDFF8D4114020B4
:10232000488001BD76B504460D461046FFF7E1FF33
:10233000064601980421F9F73CFE28B901A8F9F7EF
:10234000F7FD4FF4C17076BD0190417A084410301A
:102350004580068020460199FFF722FD002076BDCA
:10236000164699460020F9F7F3BC2DE9F84380465C
:102370005F480D4601784F1C0770FFF7F1FF04001E
:1023800008BF4FF4C1701FD00421FFF7ABFF607A84
:10239000201800F11001052048800C200880122030
:1023A00008714F710820C8800D814E81A1F80C90F2
:1023B0000898C8810988A07A091D0818A0722146CA
:1023C0004046FFF7EDFC0020BDE8F283F8B500F0D1
:1023D0000AF8070000D123E00421FFF783FF00F093
:1023E00015F813211FE004460D4616460020F9F7A4
:1023F000AFBCF8B5FFF7F7FF070000D110E00421EC
:10240000FFF770FF00F002F801210CE0787A384401
:1024100010300521418045710621018006817047F9
:102420004FF4C170F2BD01710221C1800088B97AF8
:10243000001D4018B87239462046FFF7B1FC002055
:10244000F2BD000080B5062A01BF294801891A881B
:1024500091420AD1002101819A7802B10122018AB8
:10246000C068FFF7B3FF012002BD002002BDF8B530
:102470000D4604462879122802D013282BD02DE0CF
:10248000E06B02282AD0298940F67B408A1F8242CD
:102490003EBF6A89931F834213D28A4211D3AB890C
:1024A000B3F5FA7F0DDAE889A0F10A0640F677471E
:1024B000BE4206D200902046FFF7ABFD0C490881D2
:1024C00028B969792046BDE8F84001227EE7CC6052
:1024D00068790882F1BDE06B012805D16979204651
:1024E000BDE8F840002284E7F1BD00009808002014
:1024F000BC0B002070B50546687A284400F1100630
:102500003088C0F30B00FFF7A6F8040004D128467A
:10251000BDE87040F9F771BCEC60308800F44051C0
:10252000C0F30B00B1F5805F308003D1A86820F0C4
:10253000020006E004F13000F9F7FAFCA86840F068
:102540000200A8602946687A001D687204F1300014
:10255000F9F7C2FD206B0146002201E00968521C18
:102560000029FBD1D2B2022AA8BFF9F753FE206B93
:10257000FFF7BFFE04282CD3206B417A014401F100
:102580001005FFF7B6FE2988091D814221D1688810
:1025900004280DD017D3062805D014D2294620468A
:1025A000FFF765FF0FE0216B204606F0FEFB07E01A
:1025B000206B417A091D4172206D216B01F010FAE8
:1025C0000020206370BD04F13000BDE87040F9F7D1
:1025D000AFBC70BD0A431040884201D10120704752
:1025E00000207047012802BF487900F0C000402851
:1025F00001D1012070470020704770B51546202D8D
:10260000044602DB4FF4C07070BDDFF87C69200027
:1026100014BF06F1500006F13000F3F70FFF2CB1A4
:10262000F06A86F86F5040F0200004E0F06A86F807
:102630004F5040F01000F06200F016FA002070BD1C
:10264000DFF84409002101604160816000226421BB
:102650008182C821C1820021018364214183A0219C
:1026600081834FF4A071C183072180F820101021CD
:1026700041848184002180F826100167DFF80C096D
:102680000FF6D501F7F754BC10B504460A20F5F74C
:102690005CF804F12C010A7802704A7E02F0030211
:1026A000012A03D0032A0CBF0222002202728A8E62
:1026B0004280CA8EC2800246098F818040F2091191
:1026C000BDE810400EE038B504460D460220F5F78F
:1026D0003CF894F82C10017045700246BDE8384073
:1026E00040F20721DFF8A408F7F71CBC70B50546D7
:1026F000DFF894480846216FD9B14D72606F00B180
:102700004572E06ADFF88458226F20F00200E06230
:1027100040F2071631462846F7F704FC0020626FA6
:10272000206792B131462846F7F7FCFB002060672E
:102730000BE0FEF7BCFF40B1C16880F8545041F097
:102740000101C160002100F0BFFA0020FEF7AFFFD9
:1027500020B1BDE87040143008F063BB70BD30B5E7
:10276000921E002300E01B199A4208DBCC18647803
:10277000844201D1C81830BDCC5C2500F3D10020C3
:1027800030BD38B50446DFF8005860780428E86AA0
:102790002BD040084000E86204F10B01A27A01202E
:1027A000FFF7DDFF002100B181782868012802D001
:1027B000022807D009E0C80707D42046BDE8324008
:1027C000F4F7DFBF11F0030FF7D0207AA11CFFF759
:1027D00009FF90B1A01C08F024FB0028EDD0E86AA6
:1027E0002C6740F00200E86231BDC10701D48107C7
:1027F000E3D5800701D56C6731BD207A010003D194
:102800000622A11C002009E0012802BFE07900F0A7
:10281000C000C02805D10622A11C012001F086FBC2
:1028200000E0FF2060722246E96A012060F30101A6
:10283000E96240F20711BDE8384053E7F8B50D46AC
:102840001746AF421E4639D3A91F40F67B4291423C
:1028500034D2B7F5486F31DCB6F5FA7F2EDA069C34
:10286000A4F10A0340F677418B4227D2721C07FB82
:1028700002F1B1EB840F21DAFF2807D1DFF8080756
:102880008582C782068344830020F2BDFEF7EEFEF8
:1028900000281CBFC169102910D0C16B0094012908
:1028A00033463A46294606D1FFF7B3FB0028EBD161
:1028B00040F28110F2BDFFF758FDF2BD4FF4C07039
:1028C000F2BD30B5039C2025234307D0DFF8C03686
:1028D00053F82430022B14BF032BA025A84228BF95
:1028E000A9420AD344F201039942B8BF984204DADC
:1028F000814202D3082A00DA0AB9002030BD012043
:1029000030BDF8B5DFF880460546A068C0B200903B
:102910000E466068C3B217462846FFF7D2FF00B9DB
:10292000CCE707F0070084F82000A583E683E06A7F
:1029300040F00400E06200F097F80020F2BDDFF8FC
:10294000480600214160816000224FF48471C9E68D
:10295000FFF74EBC10B50C46FEF788FE00B911E03B
:10296000C08D2146BDE81040FFF753BC10B50C46A2
:10297000FEF77CFE00B905E0C08D2146BDE81040A1
:10298000FFF751BC4FF4C07010BD10B50C0082B001
:1029900004D0032C02DAFEF769FE10B94FF4C070C0
:1029A00016BD0121621E01FA02F400210091E3B27A
:1029B000E2B2FFF7C3FB16BD10B543F6FD73041F6B
:1029C0009C423CBF0C1F9C4201D2884200D2D9E7F6
:1029D000DFF8B43503F12204208061802271D86AC7
:1029E00040F4C070D86200F03FF8002010BD70B510
:1029F0000546052DBCBF0E46042E82B00ADADFF86C
:102A0000884594F8202000910346E18BA08BFFF7C6
:102A100058FF10B94FF4C07076BD6068854204BF9E
:102A2000A06886421ED0E06A40F00C00042D65606C
:102A3000A660E06214D0012D02D0022D02D003E086
:102A4000012002E0022000E00020216909B940F0E5
:102A50000400002100F02DFAE06A40F03000E0624E
:102A600000F002F8002076BD70B5DFF81C4504F1D7
:102A7000260586B06888002840F09580E66A002226
:102A8000442100F092F8C0B100200390002394F894
:102A90002000A168029004A8019000200090DFF8B7
:102AA000F00450F82100E18BC2B2A08BFFF7A7F928
:102AB0006880E06A20F0040061E04022082100F014
:102AC00074F838B10020FFF7E1F96880E06A40F05F
:102AD000400054E00022102100F067F850B194F853
:102AE0004F0004F13001FFF7B8F96880E06A20F088
:102AF000100044E00022202100F057F850B194F873
:102B00006F0004F15001FFF7B2F96880E06A20F02D
:102B1000200034E00022482100F047F860B126F0A0
:102B20004800E062A068002804BF6068002803D065
:102B30000120FFF7ABF935E0E66A00224FF420717F
:102B400000F033F860B100200090A28C618C2878EE
:102B50000023FFF7AFF96880E06A20F080000EE004
:102B60004FF400724FF4807100F01FF848B100215B
:102B70000020FFF7BEF96880E06A40F40070E06270
:102B800011E000224FF4407100F00FF800281FBF41
:102B900026F44070E0622068002804D00021012063
:102BA000FFF7A7F9688006B070BD304612E580B522
:102BB000032802DB4FF4C07002BDDFF8CC130A68B3
:102BC00002B11AE0DFF8CC2352F820000860C86A8E
:102BD00040F4C070C862FFF747FF002002BD80B517
:102BE000DFF8A4030168491E022906D8002101600C
:102BF000C16A41F48071C162EDE740F2811002BD0B
:102C00002DE9F04784B080460C9CDF4F0020206007
:102C10000D46F86A40051646994602D540F28110E5
:102C20000AE005B1012529464046FEF783FC5FEA2C
:102C3000000A03D14FF4C170206017E0062241461C
:102C40000AF11400F3F7FAFBCAF81C50CDF808900B
:102C50000196788B00903B8BFA8AB98A5046FFF731
:102C60006DF9206020B15046FEF79AFC00200AE082
:102C7000F86A40F48060F862504606F03DF850462D
:102C8000FEF738FD504604B0BDE8F08710B50446A5
:102C9000FFF760F82046FEF783FC002010BD30B53A
:102CA000044683B0206904280DD0019140F2032529
:102CB00000946A462946B548F7F781F96A462946DD
:102CC0002046F7F77CF937BD38B504460D46207B22
:102CD000C00712D4E06904F11401FFF783FC60B16E
:102CE00094F9540010F1010F07D10420206104F180
:102CF0001400BDE8324008F094B815B92046F7F743
:102D0000E2FBE16BA048012911D1C16A21F4806185
:102D1000C162A5B10820F4F718FD024645600460C1
:102D20002046BDE8384040F20121F7F7FBB800210A
:102D3000002D81604160ECD1204605F0DDFF0220CE
:102D400020610420F4F701FD024640F206211460E0
:102D50008E48F7F7E7F80420F4F7F7FC0246046022
:102D600040F202212046F7F7DDF82046BDE8324068
:102D70008AE470B504460D460C20F4F7E6FC060024
:102D80001CD004F145003460017811F0010131716B
:102D90001CBF017801F0020171712946C07BB0713E
:102DA000B560204600F08EF932464FF4017120469E
:102DB000F7F7B8F82046BDE8704065E470BDFEB591
:102DC0000F46032F0546164634DB089C8C4228BF6D
:102DD0000C4602A90220F8F73CFB00F064F8010061
:102DE00028D00021ADF8001001AB01466A46002052
:102DF000F8F7C6FDBDF800202146914288BF114674
:102E0000ADF800100199A9B9BDF8001091B1891C65
:102E10008F420FDBBDF80010491C29706E7001460F
:102E2000BDF80020A81CF3F709FBBDF80000801CCA
:102E3000C0B2FEBD0020FEBDDCB50E46032E04462A
:102E40002FDB55480088ADF802000DF10201022089
:102E5000F8F7FFFA00F027F8010022D00020ADF8C3
:102E6000000001AB6A46F8F78BFDBDF8002009278A
:102E7000B11E914204DA082E13DBADF800100827CA
:102E8000BDF8001069B1491C217067700146BDF89A
:102E90000020A01CF3F7D2FABDF80000801CC0B2DD
:102EA000D6BD0020D6BD02464FF6FF710120F8F7CF
:102EB00048BE38B5344C04F130050021E97784F878
:102EC0006F10A87002212970032001216970009100
:102ED000E877C0F11F01204442F607230A22303070
:102EE000FFF76DFF00F033F80421009142F6042350
:102EF000C0F11F01C0B220441222C9B23030FFF726
:102F00005EFF00F024F8C0B2C0F11F012044303051
:102F1000F8F7F0FC00F01BF8C0F11F01C0B220442C
:102F2000C9B23030FFF788FF70B994F86F00C0F174
:102F30001F012044C9B25030FFF77EFF94F86F1094
:102F4000401884F86F0031BD00F001F831BDE97F11
:102F50004018E8777047000080B5062A09D040F68F
:102F60000700824203D11888D91C07F03EFF0020D9
:102F700002BD05481A88018D9142F8D100210185D2
:102F8000FFF772FD012002BD1409002098080020FF
:102F9000785A0000885A0000B264000080B503F03F
:102FA00073F8A549A54802F08DF805F09CFC0022B5
:102FB0000321002000F025F8A14900200871BDE898
:102FC000014000F0E5BE05F088BC01009C4818BF38
:102FD0000121017170479A48017919B9806800068A
:102FE000400E01E00120704700F001007047944856
:102FF000007A00F0020070479148007A00F0080063
:10300000704710B5044608460528A8BF0320E1070D
:1030100004D5032802D14FF4C07010BD0428884B9A
:103020000CBF0121014619609C6004F0040304F008
:10303000010105F0A9FB002010BD05F0CABB05F099
:1030400029BC05F0E1BB02B5FEF710FB40B16B46B1
:1030500045F21902002105F08FFE08B1002002BDE3
:1030600013E002B5FEF702FB78B1009911F1010FF0
:1030700002D0744A914208D26B4645F218020021F0
:1030800005F07AFE08B1002002BD4FF4C07002BD09
:1030900080B510F1010F02D06A49884203D205F0D1
:1030A00088FB002002BDF0E702B5FEF7DFFA40B171
:1030B0006B4645F21D02002105F05EFE08B10020BE
:1030C00002BDE2E738B50D4604462B4645F21B0229
:1030D000002105F051FE28B925B129462046BDE85A
:1030E000344057E031BD30B587B0FEF7BFFA040079
:1030F00008BF4FF4C07037D004F13C0528680128A0
:1031000026D195F9180010F1010F21D0697AC9076D
:103110001ED4102303AA032100F036FFC0B195F995
:1031200018000A236A46022100F02EFF18B90A216E
:103130006846F3F76FFA9DF800009DF8011040EA29
:10314000012203AB0DF102012046FEF778FF0BE0F0
:10315000002345F217020021204605F00DFE00284D
:1031600014BF002040F2811007B030BD10B50446F6
:103170000220F4F7EAFA60B104F12C010A78027037
:10318000024691F82810417040F60201BDE8104057
:103190000CE010BD38B500F01EF830B100F015F8A5
:1031A000BDE8384040F6010100E031BD2648F6F7A1
:1031B000B9BE38B500F00FF830B100F006F8BDE840
:1031C000384040F60501F1E731BD94F82C1001704C
:1031D00045600246704704460D460820F4F7B5BA2C
:1031E00032B5044645F2180582B16946042007F05D
:1031F00033FE0098134A0146B1FBF2F102FB1100C5
:1032000000906B462A460021204602E06B462A4683
:10321000002105F0B1FD0820F4F797FA50B194F8B9
:103220002C10017002460099416040F604010648E6
:10323000F6F778FE31BD0000EFBEADDEBEBAFECAC5
:10324000D00B002040420F009808002010B5044623
:103250000120F4F77AFA40B194F82C10017002467C
:10326000BDE8104040F60301A0E710BD38B5FFF7F8
:10327000B2FF30B1FFF7A9FFBDE8384040F60901C1
:1032800094E731BD0749086808B100207047064837
:10329000C008C00008600549C908C900091A0160D2
:1032A000704700BF2414002057140020502F002026
:1032B000DFF800F049020020DFF800F0DD01002017
:1032C0004449096809070AD5017842788378C078AB
:1032D0001B0443EA006040EA02200843704700688C
:1032E000704707F0C9BD00002DE9F04104460020F9
:1032F00014F0030682B015460F464FF0FF382CD06D
:103300000846FFF7DDFF0090F1008840C6F1040198
:10331000C90028FA01F210430090C6F1040085426A
:1033200008D2A9190098C90008FA01F108430090D1
:10333000002501E0301F45197042044400F031F8C7
:10334000714239440F1D241D07E03846FFF7B8FFCE
:1033500000F026F8241D3F1D2D1FADB2042D01D312
:103360000028F2D029000AD048B93846FFF7A8FF54
:103370000090E90008FA01F1084300F011F8001D7F
:1033800004280AD8DFE800F00309090507001248FD
:1033900004E0124802E0002000E01148BDE8F68198
:1033A0000090042269462046FFF782BF80B5FFF7F0
:1033B00083FF001D04280AD8DFE800F0030909058F
:1033C0000700054802BD054802BD002002BD0448B3
:1033D00002BD000014ED00E0023000F0013000F00A
:1033E000073000F0427A8A184272827A8918817214
:1033F0007047002105E0827A5118427A0068891AE4
:10340000C9B20028F7D108467047417A0844103005
:10341000704710B50446A1F11800FFF7EAFFA18933
:10342000081A01D5002010BD80B210BD70B50C4641
:1034300015461E46FFF7EDFFB04201D2002070BDD9
:10344000F2B22946A4F11800F8F750FE012070BD31
:1034500070B505460E460020F8F77AFC040001D14D
:10346000002070BD0821FFF7BDFFA07A3018A072C0
:103470002046FFF7CAFF05F0FF0200F029F82046BA
:1034800070BD80B5FFF7E4FF10B1BDE80240BCE7B6
:1034900002BD2DE9F04104460D4690461F4600202E
:1034A000F8F756FC060011D00821FFF79BFFB07A11
:1034B0002818B072FAB241463046F8F717FE304687
:1034C000FFF7A3FF04F0FF0200F002F8BDE8F0816F
:1034D0000168090A42EA01210160704700B970479A
:1034E00080B5183800906846F8F722FD01BD0A46FD
:1034F00000680421FEF716BF1839F8E7F8B504464E
:103500000D4616461F4605210120FFF7BAFF00B9F8
:1035100017E04570468007713FE038B504460D4618
:1035200003210220FFF7ADFF00B922E00FE038B51C
:1035300004460D4603210320FFF7A3FF00B900E076
:1035400005E00121DFF8880707F0ACFC00BFA0F818
:10355000015001462046BDE83440CDE770B5044631
:103560000D46164605210420FFF78BFF00B92DE01C
:1035700023E04FF4C17032BDF8B516461F4604462D
:103580000D46079B069A07210620FFF782FF00B928
:10359000F7E000F0C6F8A0F8057001462046BDE847
:1035A000F440A9E7012107206BE770B500F070F83F
:1035B0000820FFF76EFF00B908E0A0F80150A0F85E
:1035C000036001462046BDE8704095E74FF4C170A6
:1035D00070BD38B504460D4603210A20FFF751FFA0
:1035E00000B9C6E7B3E738B500F022F888BF2B462C
:1035F0000A4601210B20FFF74CFF00B9A1E7A8E71D
:1036000070B504460D46164605210C20FFF739FF1C
:1036100000B9DBE7D1E738B500F00AF888BF2B46E0
:103620000A4601210D20FFF734FF00B989E790E732
:1036300004461546A089401E83B2AB42704710B5C0
:1036400004464FF6FE73A089401E1840904238BFD2
:103650000246D3B20A4601210E20FFF71AFF00B935
:10366000D0E031E038B5FFF7E3FF88BF2B460A46CC
:1036700001210F20FFF70DFF00B962E769E770B580
:1036800000F006F81020FFF704FF00B99EE794E76A
:1036900016461A4604460D46049B0521704738B568
:1036A00000F093F888BF1846034603211220FFF765
:1036B000F0FE00B95DE74AE710B50446012113208A
:1036C000FFF7DFFE00B93CE701462046BDE81040A9
:1036D00012E738B500F079F888BF18460346032191
:1036E0005220FFF7D6FE00B943E730E77CB5044629
:1036F0000D46A0891646411F1A4606988BB2834292
:1037000088BF034605211620FFF7C3FE10B94FF40A
:10371000C17076BD00F005F801462046BDE87C404A
:10372000EAE6A0F80150A0F803607047F8B5044637
:103730000D46A0891646471F1846FFF75AFEBFB22E
:10374000874205DA0099897AC91B40180099887266
:1037500005210098F8F72DFC010003D16846F8F721
:10376000E7FB0EE0487A084450F8102F120A1202C4
:1037700042F017020260FFF7D4FF2046FFF7B7FEC2
:10378000F2BD4FF4C170F2BD38B504460D460221BA
:103790001820FFF776FE00B9EBE64570D9E610B5C4
:1037A000044601211920FFF76CFE00B9C9E68BE73A
:1037B00038B500F00AF888BF1846034603211B20DD
:1037C000FFF767FE00B9D4E6C1E604460D46A089BE
:1037D000C11E88B29842704738B5FFF7F6FF88BF20
:1037E0001846034603211D20FFF753FE00B9C0E62B
:1037F000ADE610B5044601211E20FFF742FE00B9D8
:1038000000E061E74FF4C17010BD80B50A790AB1DC
:1038100002F580624978022914D0042917D00629BC
:103820001CD008291FD00A2924D00C292CD00E29FD
:1038300025D010292DD0122932D0162935D018299B
:103840003AD001BDBDE804401721F6F7F7BEBDE848
:103850000050134600220021F7F75EBCBDE8084087
:103860000021F7F769BCBDE8005013460022002193
:10387000F7F753BDBDE808400021F7F7A6BCBDE847
:1038800008400021F7F733BDBDE808400021F7F7F5
:1038900018BDBDE80050134600220021F7F76FBDA8
:1038A0001146BDE80440F7F778BD009200230022DE
:1038B0000021F7F77BFD01BD1146BDE80440F7F795
:1038C00090BD10B5417A014401F11004FFF791FD5C
:1038D000401E216880B2421E01F0FF01012960D024
:1038E000022918BF03295AD004295AD005292ED0FD
:1038F000062952D0072939D008294AD009293CD0B5
:103900000A294CD00B2963D00C294AD00D295FD04D
:103910000E2948D00F295BD010293AD0112930D078
:10392000122948D0132951D0162918BF172947D07A
:10393000182948D0192949D01B2918BF1D293AD068
:103940001E2943D0522936D0D22936D00CE058B1A6
:103950006078022808BF102002D0012804D102207C
:10396000801C00F037F833D0002010BD410800EB78
:1039700091718908B0EB810026E00028F4D06078CE
:1039800004E00028F0D060780428EDDB00F022F895
:103990001AE006281CD0142816E0062811E0022898
:1039A00012E0042810E00428DEDB00EBD0714908A7
:1039B000B0EB410008E0022803E00E28D4DB07E06A
:1039C0000428D1D304E00128CED101E00028CBD1D6
:1039D000012010BD92FBF0F100FB11200028704780
:1039E0002DE9F241040083B007D1002918BF012955
:1039F0002BD003A8F8F79CFA27E0DFF8D4824046E2
:103A000007F046FAC8B1022811D0032812D0039853
:103A1000417A014448690399C00754BF04F1080082
:103A2000201DF8F7AFFB002004B0BDE8F0810020B6
:103A3000039004E0012003900CE0039840B9201D9E
:103A4000F8F781FA03900398A8B94FF4C070EBE738
:103A5000012802D104F10800F2E7417A0144086923
:103A6000C0074CBF201D04F10800016819B103997B
:103A7000F8F732FBD7E70398417A084400F11006C3
:103A8000306800F0FF070398FFF7B3FC0500B0D0E3
:103A90000398FFF716FF68B9F807AAD4522F1CBF86
:103AA000D22F1E2FA5D00423002239462046FFF72F
:103AB00025FD9EE7681F3946012942D0022900F002
:103AC0009780032942D0042900F0A980052942D01B
:103AD000062900F0AB80072949D0082900F096801C
:103AE000092949D00A2900F0AF800B2949D00C29B7
:103AF00000F0AF800D2949D00E2900F0B1800F29C8
:103B000049D0102979D011294AD0122900F0AE806D
:103B100013294AD0162900F0B38017294AD0182952
:103B200000F0B380192954D01B2957D01D295AD031
:103B30001E2900F0AF80522900F09D80D22904D0C8
:103B4000ACE031462046FFF760FEACE000F0D2F872
:103B5000F6F774FDA7E003980399407A801C487239
:103B6000039A717800232046F7F7D6FA9EE000F01A
:103B7000C5F8F7F7E1FA99E000F0ACF8F7F7CDFBFC
:103B800094E000F0BBF8F7F720FB8FE000F0B6F808
:103B9000F7F797FB8AE000F0B1F8F7F7A8FB85E0AC
:103BA00000F098F8F7F7EBFB80E000212046F7F7EC
:103BB000F4FB78E003980399407A401D4872002096
:103BC0000090039BB6F8032000F094F8F7F7EEFBA3
:103BD0006CE000212046F7F704FC64E000F084F874
:103BE000F7F70FFC62E000F07FF8F7F70FFC5DE0FD
:103BF00000F080F8F6F714FD55E010280CBF1023F4
:103C0000022300F084F8F8F71EFC4CE010280CBFEB
:103C10001023022300F07BF8F8F79FFC43E0B6F88E
:103C2000032000F067F8F8F72AFD3CE0E81F80B2B7
:103C30000190F01D0090B6F80530B6F8032000F0B2
:103C400059F8F8F792FD2EE000F054F8F8F759FE15
:103C500029E0B6F8032000F04DF8F8F756FE22E010
:103C60006A1E711C2046F8F753FE1CE000F041F874
:103C7000F8F7B7FE1AE000F03CF8F8F7E2FE15E0BE
:103C800003992046F8F706FF10E071782046F8F710
:103C90008EFF08E02046F8F79CFF04E00623002290
:103CA0002046FFF72BFC03A8F8F742F9F80704D5E4
:103CB0006068002803D0022104E0A06800283FF4D7
:103CC000B2AE0321404607F0EDF800BF000000004F
:103CD0004804002003980399407A801C4872727847
:103CE000039900232046704703980399407AC01C2B
:103CF0004872039AB6F8011020467047039803995A
:103D0000407A401C48720022039920467047701D7B
:103D10000090B6F80320B6F801102046704780B531
:103D2000F6F74EFA009008B907F0C8F8009802BDFF
:103D3000F6F79EBA002803D492490A79904201DB33
:103D4000002070470968012202FA00F0084018BFFD
:103D500001207047F0B583B04FF0FF3500260027F3
:103D6000884C10E02068F840C0070BD508236A464D
:103D7000082178B200F008F920B10198A8423CBFB0
:103D800005463E467F1C20798742EBD370B2FEBDCC
:103D900030B583B000257B4C05E00198A1688142D5
:103DA00038BFA0606D1C207985420FD22068E840A2
:103DB000C007F7D508236A46082168B200F0E4F886
:103DC0000028EAD168B200F071F8EBE737BD6D4921
:103DD00009680020002903E0CA0748BF401C4908C1
:103DE000FAD1704770B5040008BF012402D00D2C31
:103DF000A8BF0C24634D29798C4208D2264603E0E3
:103E000070B200F053F8761C28798642F8DB2C71EA
:103E10002A46BDE8704001E05A4A50710C2143F631
:103E2000FF7007F01BB81CB56A4601A943F6FF7086
:103E300007F019F8534C28B900990C222046F2F7E4
:103E4000FDFA13BD002020600C202071002060715D
:103E5000A06013BD4B4800687047F8B50446FFF7F3
:103E6000B6FF484D2979884205DB6879D8B1FFF75C
:103E700071FF00F01BF828680026012101FA06F7FF
:103E800038420DD1384300F034F818B12868B843EF
:103E9000286008E0A868401CA860206070B2F2BDED
:103EA000761C0C2EEADB4FF0FF30F2BD38B510F176
:103EB000010F0446334D06D14FF40041084606F089
:103EC000D9FF002011E0FFF735FF10B94FF4C9709A
:103ED00032BD200240F400404FF47F4180B206F032
:103EE000C9FF28680121A140884300F002F80020A2
:103EF00032BD28602A460C2143F6FF7006F0AEBFA3
:103F0000F8B504460D4616461F46FFF713FF10B9D5
:103F100040F21220F2BD3246394645EA0420BDE89F
:103F2000F84040F4004080B206F098BF2DE9FC4113
:103F300004460D4690460027124E30680121B940D4
:103F4000084217D044EA072040F400406A4601A91D
:103F500080B206F088FF002804BF9DF804004045A9
:103F600008D1009830B142462946F6F7F5F908B96C
:103F700078B204E07F1C0C2FDFDB4FF0FF30BDE890
:103F8000F6810000DC0B0020F0B583B006460F463A
:103F900014461D46FFF7CEFE80B147EA062040F4E6
:103FA000004001AA694680B206F05DFF30B99DF875
:103FB000000000281CBF0198002801D10020FEBD90
:103FC0009DF800108D4288BF0D4601462A462046C6
:103FD000F2F734FA2846FEBD81423ABF53189842A0
:103FE000F2F72CBA8018990707D0521E24BF13F895
:103FF000011D00F8011DF6D8704781071CD1103A49
:1040000007D330B433E93210103A20E93210F9D234
:1040100030BC1032121F24BF53F8041D40F8041D99
:10402000F8D838BF121D521E24BF13F8011D00F826
:10403000011DF8D8704700BF083A07D333E90210D2
:10404000083A40F804CD40F8041DF7D20832EAE7F8
:10405000EFF3108072B6704700B962B67047FEE7A2
:1040600080B53F4800682430F8F723F858B18168DC
:10407000C1F3800119B9BDE80240F9F729B8BDE8DC
:104080000240F9F722B801BD80B5B2F5803F06D0F5
:10409000B2F1011F06D1FFF7E3FF012002BD00F0DE
:1040A0001DF8FAE7002002BD38B50446F4F759FEC2
:1040B0002B4D2C492860FBF717FF2968062081F853
:1040C0003C000320296881F83E000020296808622E
:1040D0002C712868F4F785FE286832BD38B5204C6D
:1040E0002068806A28B3204D286810B906F006FEC3
:1040F00028602868E8B1F5F7F9FF05462068283000
:10410000F7F7D7FF00902846F5F7F4FF009880688E
:10411000C0F3800020B900980099407A801C487252
:1041200069462068C069F4F75EFF10B10098F7F7A0
:1041300064FE31BD70B5040010D0F5F7D7FF084E0E
:104140000546306821462830F7F7C6FF2846F5F7C0
:10415000D1FF3068BDE87040F4F767BD70BD000066
:10416000F80E002089400100000F0020002818BF31
:10417000FFF7E0BF7047FEE70A431040884201D1D5
:10418000012070470020704750E8002F0A4340E8A4
:104190000023002BF8D1704750E8002F8A4340E8F5
:1041A0000023002BF8D17047012802D0022802D04A
:1041B00003E0C8007047880070474FF0FF30704739
:1041C00080B50F31FFF7F0FF80B202BDF8B50446AD
:1041D0000F4601250026012002E0701E8041C00F1D
:1041E0002146FAF74EF9836819000ED0028A9742E9
:1041F00002D10022012104E00078C00705D5002289
:1042000000212046984700B90025761C022EE4DBE9
:104210002846F2BD38B500F007FC000729462046C5
:1042200002D5BDE8344052E1BDE83440E1E02DE97B
:10423000F0410D4682B000F084FD317802290FD0A4
:10424000072959D0092900F098800C291CD00D2984
:1042500046D0112930D014295CD0152974D0A7E09C
:10426000717800F0EEFC202100F0F0FC00F0C5FABF
:1042700000F0EFFC0120009000230FF201622146C4
:10428000002000F000FE7FE000F091FB80057BD471
:10429000022068724FF4007100F0D8FC687A28445C
:1042A0000C2100F8101F052240F2FF214180082157
:1042B0004170012181807FE07778B67800F074FB4F
:1042C000162F07D13246204602B0BDE8F041032147
:1042D00006F0F7BD00F06BFB00F083F8836806E0A2
:1042E00000F065FB00F07DF800F05CFBBB68180097
:1042F00068D03246032108E000F0E5F800F052FBF8
:10430000BB6818005ED032460421204602B0BDE8EA
:10431000F041184700F058F800F05BF88046386824
:10432000F288B18800F059F80646802100F08EFC32
:10433000324641462046FAF75CFF2A4615212046C0
:1043400000F05FF9082237E000F0BDF80FF281417C
:104350008068884218D1687A284400F035F800F067
:1043600038F880463868F288B18800F036F802469E
:1043700041462046FAF73DFF12E000F0A4F80FF2A4
:1043800035418068884204D02846BDE8F641F7F7F9
:1043900034BDD6F8010000F02D012046FAF73BFFAE
:1043A00000F002FB2146BDE8FC41012000F091BD78
:1043B00007203070717001222946204602B0BDE806
:1043C000F04114E1BDE8F38100F111062046FAF74F
:1043D00045BF07463868728831882A23C0F3032016
:1043E0002EE1C00800F00100214680F00100FAF73C
:1043F00048B838B50D460446687A2844007C04283D
:104400000BD0052818D0062827D00B282ED00E2830
:1044100020464DD1BDE8344028E100F015FC687A13
:104420002844103000F10903421C00F006FD284624
:10443000BDE83240F7F7E1BC00F045F800F11201A9
:104440002046FBF7B5FC0621284600F02EFA294647
:104450002046BDE838400022C9E000F0A5FA00F08F
:10446000CCF92046BDE83240FBF78CBC00F0ECFBF9
:104470004FF440412046FAF711F800F092F800F0AE
:1044800022F80546E86880B1417A0844103000F10E
:10449000130300F10B02012100F0D0FC2046FBF7D2
:1044A00056FCE968162200F0CAFB0020E86031BD26
:1044B00000F0C1FD20B929462046BDE83440B6E6EB
:1044C00031BD04460D4621460120F9F7DABFF8B5A3
:1044D0000D460446687A2844017C61B1012914D054
:1044E00003292BD0062943D0082909D00A292BD02B
:1044F0000B2934D04AE029462046BDE8F440D2E3F7
:1045000029462046BDE8F440B0E000F11006204600
:10451000F18800F0B6FB0746701CFAF773FB002821
:1045200018BF002F01D100F012BC00F006FC0FF202
:10453000911200F07DFCF38800F0FCBB2946204678
:10454000BDE8F44000F008BC0B21017400F029F82C
:104550004FF4C05100F07AFB4FF4004103E000F04B
:1045600023FA4FF480412046BDE8F440F9F796BFA6
:10457000284600F09AF900F014F82046FBF702FCF8
:104580002146BDE8F440002000F0A3BC29462046A7
:1045900006F099FC20B929462046BDE8F44046E6DD
:1045A000F1BD00222946204621E02DE9F0410D46CB
:1045B0008046687A284400F1100416461F4640469B
:1045C000F9F768FF00030AD502214046FAF7D2FE48
:1045D00028B11120207067700222A67003E00D2020
:1045E00020700122667029464046BDE8F0414B7AB2
:1045F000D218521C8A728A6842F004028A60FAF762
:104600005DBD38B50446104600F04FF9054620461A
:10461000FAF724FE04462A20A5F801002A2100F01A
:104620000BF8A5F803002A212A20A5F8050000F0C0
:1046300003F8A5F8070031BD2068C0F30320BFE5EB
:1046400070B50C4615461E460121FFF7ADFDB5FBC2
:10465000F0F00F3880B2A042B8BF0446A642B8BFFF
:1046600034461B2CB8BF1B24E0B270BD70B50D469C
:104670000446687A2918D1F8110000F02D06314659
:104680002046FAF7C8FD02206872C5F813600920B9
:10469000A87429460020C5F8170008222046BDE866
:1046A0007040A4E780B5012904D12221F9F74AFF1F
:1046B000002002BDF9F733FF00B1012002BD000068
:1046C00070B504460D4600F038FB012D064602D0B9
:1046D000022D11D015E0F068417A084400F1110173
:1046E0002046FAF7A8FAF068F7F787FB0020F06099
:1046F000214600F0EEFB04E0F068F7F77EFB0020B7
:10470000F060012070BD2DE9F04182B000F08CF91D
:1047100000F0A8F80746012DF868417A014401F13C
:10472000100602D0022D11D014E07078420070887B
:10473000410089B22046F9F7D3FE00F07AFB738975
:104740000FF21902404600F09EFB03E0F7F755FB1D
:104750000020F8600120BDE8F6810000F8B500F007
:1047600063F9C00800F0010080F0010721463846D7
:10477000F9F787FE0646F068417A01441031012DB1
:1047800002D0022D10D013E00B89CA8889882046F8
:10479000FAF707FAF068F7F730FB0020F0602146DF
:1047A000384600F096FB03E0F7F727FB0020F060A7
:1047B0000120F2BD10B50129044606D0042902BF2C
:1047C0002146012000F04DFB00E00FE0012010BD6C
:1047D00010B50129044606D0042902BF2146012054
:1047E00000F03FFB00E001E0012010BD2221F9F7BD
:1047F000A9FE00F002F8002010BD2146012030E3A0
:104800002DE9F04104460D461646F9F743FE00F047
:1048100029F8012D074602D0032D0CD01FE02046B9
:10482000FBF7BBFA222100F00CFA2146404600F0CB
:1048300018FB002014E0F868F7F7DFFA0020F860B2
:104840002046FBF7AAFAF1B200F0FBF94FF0006145
:104850002046F9F77AFE2146404600F002FB01208F
:10486000BDE8F081C00800F0010080F00108214699
:104870004046F9F706BE00207047000080B5F9F702
:1048800009FE10F0400018BF012002BD38B500F04D
:10489000CBF800F03800102800D0F0E02946204680
:1048A000BDE838400FF21D025DE3022282724272BF
:1048B000826842F0040282600222104400F8101F55
:1048C000704700002DE9F041804686B00D4600F0AB
:1048D0007FF9060008BF072040D0687A284400F11D
:1048E00010010E2201A8F1F7A9FD00213046FFF7C3
:1048F000DCFF074602214046F9F7D5FD7881BDF877
:104900000A00F880BDF80C003881BDF80840BC8072
:10491000FBF7B3F8611C90FBF1F201FB1200788009
:1049200017220220787006F1100105F11000F1F74E
:1049300095FD707A68724146FFF7C6FDDFF8D8240E
:10494000C5600020009041467889431E9BB201203B
:1049500000F099FA0B2200F004F8002006B0BDE840
:10496000F0813146404642E670B5FFF7AAFD0646A3
:1049700000F01DF8000307D500F016F84FF0805145
:104980002046F9F7E2FD04E03078400703D500F057
:104990000BF8002070BD29462046BDE870400FF29C
:1049A0001502E0E2074676782846F7F726BA204651
:1049B000F9F770BD38B5FFF784FD016841F00401D7
:1049C0000160FFF7F4FF00074CBF0E2108212846C5
:1049D000FFF76BFF0021C0F8051008222D21C0F859
:1049E000011020462946FFF702FE00F006F80346B4
:1049F00000F01FFADFF824242CE003212046F9F709
:104A000052BD38B500F010F8000603D5FFF7CCFF13
:104A1000002032BD802100F019F929462046BDE86A
:104A200038400FF20D029EE204460D46F9F732BD02
:104A300038B50D4604462A461421FFF7E2FD082248
:104A400000F0FCF8FFF7D9FF002100910346DFF8E2
:104A5000D0232146012000F016FA002032BD38B5DF
:104A6000FFF7E2FF08221021FFF786FB00B906E0FE
:104A700029462046BDE838400FF20D0273E2FFF7E9
:104A800093FF0C2032BD00002DE9FF4180460D460A
:104A9000F9F700FD00224FF44041FFF76DFB0026BF
:104AA00028B100F095F8060008BF07205FD0414606
:104AB000FFF70AFD0746687A284400F11F0110221B
:104AC00007F11200F1F7BAFC687A001D687200F174
:104AD0000A01C0B2284400F11004A972032020701A
:104AE00001A90C2000F0DDFA082201A904F10B0055
:104AF000F1F7A4FC042203A904F11300F1F79EFCD2
:104B0000A6B10220B07270720221B06840F00400B9
:104B1000B06031440A2008740022FFF722FFFD60D4
:104B20004FF400614046F9F7B7FC13E00020F7F7B7
:104B300064F904F1130304F10B0201214046FBF771
:104B4000DBF816222946FFF70DFF0020F8604046EB
:104B5000FBF7FDF803214046F9F7A5FC03460020CA
:104B600000904146AF4A012000F08DF9002004B0CA
:104B7000BDE8F081F8B5FFF757FF800401D40C20A1
:104B8000F2BD00F025F8060001D10720F2BDF5F7CF
:104B9000ADFA074665B105213046FFF786FE0022D3
:104BA000314600F04CF829462046FBF701F90AE0AF
:104BB0000323062231462046FFF7F7FC2046FBF789
:104BC000ECF800F046F83846F5F794FA0020F2BD0C
:104BD0000220F7F7BDB870B582B0FFF725FF0226B7
:104BE00000F03000102827D1FFF7F2FF08B90720A6
:104BF00076BD816841F0040181600222417A01445E
:104C0000002601F8102F4D700146012200F017F820
:104C1000162100F016F8202100F018F8FFF7EDFD3E
:104C200000F017F80121FFF7E9FE0346012000908C
:104C300021467D4A00F027F9304676BD29462046B8
:104C4000D5E42046F9F77EBC4FF480512046F9F7B1
:104C500023BC2146002004E138B50D46044620213E
:104C6000F9F71AFC2946FFF7ECFFFFF7C6FDFFF73F
:104C7000F0FF0120009000236C4A214600F003F968
:104C800031BD10B50446F9F705FC800604D400F0E8
:104C900054F80068022801D1002010BD0021FFF760
:104CA000ADFE012010BDF8B50D4600F04AF82046D3
:104CB0007189FFF7E6FFB28873881146994238BFC1
:104CC000002008234F1E092FA8BF531E77789BB2E0
:104CD000BB4238BF002007B90020921F40F67B433B
:104CE0009A423289F38828BF0020D70097FBF1F75A
:104CF0007F1EBFB2B7F5FA7FC8BF4FF4FA779F4265
:104D000038BF00205F1C79434900C91DC9080A2922
:104D100038BF0A218A4203D3B2F5486F00DC00B9DC
:104D200015E000F00AF83C4A00F082F87089431E52
:104D30009BB2002000F0A7F8F1BD21460020F9F752
:104D4000A0BB0446687A284400F110067047284644
:104D5000BDE8F240F7F751B870B588B0FFF764FED0
:104D6000800602D5FFF720FE53E0687A284400F160
:104D7000100606F1090001A902780A7042784A700B
:104D8000711C082202A8F1F759FB06F1130306F182
:104D90000B02012100F052F80220687204A90420DD
:104DA000A8740C2000F07DF9082204A905F1130075
:104DB000F1F744FB042206A905F11B00F1F73EFBC5
:104DC00005F11B0305F1130200F037F8FFF7B5FFFB
:104DD00001A9123000F108020B7813704B78537060
:104DE000082202A9F1F72AFB4FF000712046F9F7DB
:104DF000ACFBFFF729FF2046FAF7A9FF0C22FFF7CB
:104E00001DFFFFF7FAFD034600F013F8054A00F016
:104E10003AF808B070BD000007470100B54701002F
:104E2000D147010001480100A54601007748010073
:104E3000C560002000902146704700212046FAF707
:104E40005BBF38B50446FFF778FF00F11205204636
:104E5000F9F798FB29892A46BDE8384080B2F8F76F
:104E60007EBD38B504460D46F9F70BFB8368180084
:104E700008D0002202212846984729462046BDE84E
:104E8000344026E031BDF8B514461D46F9F7F9FA6D
:104E90000646F5F72BF90746069820B10121304662
:104EA000FFF772F903E001213046FFF775F92000A2
:104EB00004D002213046FFF767F903E002213046B3
:104EC000FFF76AF9B46035823846BDE8F240F5F77D
:104ED00011B970B582B004460D46F9F7D2FA06460C
:104EE000002000900023002229462046FFF7CBFF38
:104EF000002C1CBF706800280AD04FF08041284663
:104F0000F9F723FB3046BDE87C400221FFF73CB9AE
:104F100073BDF8B506460C463146FFF7D5FA05468F
:104F200031460020F9F7ADFA01462B680A6842EADB
:104F30000300C00701D50120F2BD4FF6FF763046D1
:104F40009B0744BF288A001B3746920744BF098A43
:104F50000F1BBFB280B2B842C8BF3846B04208BFCC
:104F60004FF0FF30F2BD2DE9F04180460C4682B093
:104F700017464146FFF7A8FA0546F5F7B7F8064683
:104F80002878800714D504212046F6F7F2FF009711
:104F90000422607A204469461030F1F74FFA214626
:104FA000281DF7F799F83046F5F7A4F8002005E03A
:104FB0003046F5F79FF821464046B847BDE8F681F0
:104FC00038B50446FFF77FFA054605F10C00F6F701
:104FD000AFFF281DF6F7ACFFFFF7AFFE044604F164
:104FE0000C00F6F7A5FF201DBDE83240F6F7A0BF84
:104FF00070B5044682B0FFF766FA0546281DF7F73C
:1050000058F8060016D002212846FFF7C5F8757A31
:10501000701900F1100104226846F1F70FFA281DFB
:1050200070723146009A20469047072804BF3046E8
:10503000F6F7E3FE73BD00207047FEE73EB5044679
:10504000274D01F024F88022294601F039F801F0BB
:105050001EF805F1100100910294019405F110036E
:105060000022102101F063F80028EAD137BD30B5E5
:1050700089B004460D466846FFF7E0FF2A466946B8
:105080002046F1F7DBF96846FFF7D8FF04A8FFF7E1
:10509000D5FF69463CC912483CC03CC93CC009B078
:1050A00030BD70B504000D4605E0F1B22846FFF7AB
:1050B000DEFF3544A41B04D0112C2CBF102626463D
:1050C000F3E770BD10B5064C10212046FAF7CEFD6F
:1050D00004F11000BDE810401021FAF7C7BD000030
:1050E000E80B002010B5744A946A00236372831C95
:1050F000946AA372926A537A1A4402F110031970E7
:10510000587061B1022901D002D310BD552200E0D0
:105110000F22BDE810400146981CF5F767B9BDE8BD
:10512000104002466549981CF1F788B910B500F0A7
:1051300098F8400706D5FAF7A2FC2169BDE81040AF
:1051400009184FE00121204600F043F9606800F2A1
:1051500071206060204600F020F9BDE8104000F0AA
:105160009FB9000010B50B28534C3AD8DFE800F087
:1051700006391F27362A363639393627E06A504A2B
:105180005049C0B2FAF788FC94F82000800708D58F
:10519000A06AFAF718FD6168BDE810400020FAF730
:1051A0003BBD00F0D2F8BDE8104001461AE000F027
:1051B000ABF9A04215D1BDE81040FAF705BCFAF7EB
:1051C00003FC0BE0FAF7C7FB40B1417A0144097DCB
:1051D00011B1A18C491CA184F6F70FFEBDE8104067
:1051E000A4E710BD0020FAF793BCF8B505460E46BB
:1051F000282DB8BF2F2E174608DA00F032F8C00766
:1052000004D40120F6F7A4FDA06208B90020F2BD85
:1052100039463046FFF766FF0320032F2062E56220
:1052200005D11320206268B2FAF730FD17E0264856
:10523000E061032060614FF49670E0604FF4C87045
:1052400020616420A060F4F751FF0546FAF717FCCF
:1052500000F040F800F024F92846F4F74BFF012055
:10526000F2BD154C94F82000704738B5282804DAB0
:10527000114C94F82010C90701D5002032BDE0621E
:1052800005210020A084216210480F49E060E161FF
:1052900003210F48206161616420A060F4F726FFBC
:1052A0000546FAF7ECFB00F015F800F0F9F828468F
:1052B000F4F720FF012032BD64130020485C000099
:1052C000294176715555550065510100C0C62D0024
:1052D00000093D00A168081864306060204600F0B5
:1052E0005CB870B5FFF7BDFFC00607D5002020628F
:1052F0004FF0FF30FAF7CAFC002070BDF4F7F6FE5D
:105300000546002020620021204600F062F800F0EF
:10531000C7F8FAF759FBA06A18B1F6F76EFD00203E
:10532000A0620020A68CA0842846F4F7E3FE304655
:1053300070BDFEE7890001EB401000F108500260EB
:1053400070470122F6E70022F4E77648C068DC38AF
:10535000704780B5FAF793FB7249C968081ADC38C0
:1053600002BD10B56F4C2168CA0607D521F01001A7
:10537000216018B9A168CA69022090470020A06086
:105380002068810708D520F0020020600021BDE8D8
:1053900010400020FAF775BB10BD38B50446002058
:1053A000206063685F48051D00E00D46296871B103
:1053B0004A68D21AF9D4216080682968884206D1E7
:1053C000087E217E88423CBF0020FFF7CAFF2C6088
:1053D00031BD38B50446534D0846A968A14208BFFF
:1053E000FFF7BFFF281D00E00846016819B1A14280
:1053F000FAD10968016031BDF8B54A4C6568002DE5
:1054000037D0FAF73CFBAB686E6895F814C02A6990
:10541000F71A3F1A5FEACC7C11460AD4002F08D550
:10542000D219EF68D71B04D4711818186860091ACC
:1054300001E0002F13D4286801E0114600686A6873
:10544000531890B142689A1A012A0EDBEB688A1A47
:10545000DC339A42F1D22A7E037E9A42EED2EA6986
:105460002946032090470020F2BD03F1DC00E060F4
:10547000A5600120F2BD10B52A4C28B102212046BA
:10548000FFF75FFF022006E002212046FFF75BFFE7
:10549000A06818B10320BDE810402EE0BDE8104020
:1054A00038B5204C2078400726D4A06820BB0221C4
:1054B0002046FFF746FFFFF79FFF0028FBD00221A1
:1054C0002046FFF740FFA568B5B1A86838B120684D
:1054D00040F0100020602946EA6900209047287DAE
:1054E000800709D4206840F002002060012069682C
:1054F000BDE83440FAF7C5BA31BD0A4989680029C8
:105500001CBFCA6910477047064880687047054845
:10551000016821F0020141F0100101600120ECE777
:1055200000000000381200200120704780B502F012
:1055300038F91F4901200870002002BD10B504464B
:1055400000F06EFC20684168806802F0B3FC02F055
:1055500097FC002814BF1748174802F07AFD14483A
:10556000017829B1002101704FF4803005F0BAFCB8
:1055700020680088C0B210BD80B5FBF7B7FEBDE85B
:105580000240FBF7CBBE10B50446208802F05DFB5D
:105590002080608802F046FB6080A08802F0DFFA7D
:1055A000A080E08802F006FBE080002010BD000033
:1055B00048140020C0CF6A00E067350005F0B3BC96
:1055C000890001EB401000F184400260704780B513
:1055D00006F083F8FBF7A2FE00906846FAF769F937
:1055E00001BD2DE9F04788B002F0D8F9824601A844
:1055F00002F00AFABDF8045000264FF6FF7085420B
:1056000079D0A5EB0A05ADB205F10C00FAF71CFA4A
:1056100081461BE006F10A08AC1B00946A4641462D
:105620004846FAF715FA0746009808B9002700948B
:105630003846009989B205F06AFF8619B6B207B9F3
:105640000020024641464846FAF707FAAE42E1DB3F
:1056500002A9504605F06BFF0C2000906A4600211D
:105660004846FAF7F5F9060002D000980C2801D256
:10567000002236E0DFF8AC0635814168DFF8A81675
:1056800009683279C90901F0010181F0010102F0D4
:10569000FD0242EA4101317101220721FFF790FF2B
:1056A00030799DF80E2000F0FE0002B10122104377
:1056B00030719DF80D0070719DF806103079C908A1
:1056C00000F0FB0001F0010140EA810030719DF81B
:1056D0000700B0710598FBF721FE30600C22002016
:1056E000F07100214846FAF7B8F94846FAF7F8F899
:1056F0004846FAF7ACF908B0BDE8F08780B501225A
:105700000721DFF82006FFF75BFFBDE8024010200D
:10571000FAF70CB92020FAF709B910B5DFF80C0632
:10572000046800221821FFF74BFFE001BDE810409C
:1057300054BF4FF480604020FAF7F8B8DFF8F01556
:105740008968012806D002280AD1C80508D54FF477
